:100000000C94A40A0C94D50A0C94D50A0C94D50A25
:100010000C94D50A0C94D50A0C94D50A0C94D50AE4
:100020000C94D50A0C94D50A0C94D50A0C94D50AD4
:100030000C94D50A0C949D570C94D50A0C94D50AAF
:100040000C94D50A0C94D50A0C94D50A0C94D50AB4
:100050000C94D50A0C94D50A0C94D50A0C94BD992D
:100060000C94D50A0C94B04E0C94874E0C94D50A7F
:100070000C94D50A0C94D50A0C94D50A0C94D50A84
:100080000C94D50A0C94D50A0C94D50A0C94D50A74
:100090000C945D4E0C94344E0C94D50A0C94B158CB
:1000A0000C94D50A0C94D50A0C94D50A0C94D50A54
:1000B0000C94D50A0C94D50A0C94D50A0C94D50A44
:1000C0000C94D50A0C94D50A0C94D50A0C940A4EBB
:1000D0000C94E14D0C94D50A0C94B74D0C948E4DB4
:1000E0000C94D50AF11BD81C401C391C091CF91BA7
:1000F000D81CF51BD81CD81CD81CD81CD81C610BCC
:10010000CA0B520C8F0D970D710F25104311E5127C
:10011000E11337144C145014D81C92149614011681
:10012000BC17D617FD1860193F1ABF1AC61AB21BA2
:100130000C40A540B740C040C940D240E440ED402B
:100140001C412E41374140414941E441ED41F641D6
:100150003F844284318435843B84798446844A8454
:100160005084548458845E846284668479846C8468
:1001700070847484084AD73B3BCE016E84BCBFFDBB
:10018000C12F3D6C74319ABD56833DDA3D00C77F67
:1001900011BED9E4BB4C3E916BAAAABE0000008000
:1001A0003F07634236B79BD8A71A39685618AEBACC
:1001B000AB558C1D3CB7CC5763BD6DEDFD753EF660
:1001C000177231BF000000803F08000000BE92247B
:1001D00049123EABAAAA2ABECDCCCC4C3E000000B0
:1001E00080BEABAAAAAA3E00000000BF00000080AB
:1001F0003F0000000000084178D3BB4387D1133D86
:10020000190E3CC3BD4282AD2B3E68EC8276BED94E
:100210008FE1A93E4C80EFFFBE01C4FF7F3F00008D
:10022000000000004E414E494E495459494E46CDBA
:10023000CCCC3D0AD7233C17B7D13877CC2B32959D
:1002400095E6241FB14F0A000020410000C842007B
:10025000401C4620BCBE4CCA1B0E5AAEC59D740045
:10026000407A10F35A00A0724E18090010A5D4E885
:100270000000E87648170000E40B54020000CA9A18
:100280003B000000E1F5050000809698000000406A
:10029000420F000000A086010000001027000000AF
:1002A00000E803000000006400000000000A0000F5
:1002B0000000000100000000002C76D888DC674FA9
:1002C0000823DFC1DFAE59E1B1B796E5E3E453C6D9
:1002D0003AE651997696E8E6C28426EB898C9B62D1
:1002E000ED407C6FFCEFBC9C9F40F2BAA56FA5F47B
:1002F00090055A2AF75C936B6CF9676DC11BFCE0A3
:10030000E40D47FEF520E6B500D0ED902E030094F5
:100310003577050080841E080000204E0A0000008A
:10032000C80C333333330F986E12831141EF8D2194
:1003300014893BE65516CFFEE6DB18D1844B381BFB
:10034000F77C1D901DA4BBE424203284725E2281C0
:1003500000C9F124ECA1E53D274D6F74696F6E0073
:10036000555620496E742E00555620496E74656EA0
:1003700073697479004F3220436F6E6300434F32CC
:1003800020436F6E630053656E736F7220657272E7
:100390006F722100234E6F2073656E736F722100A0
:1003A000434F3220436F6E63004D65617375726910
:1003B0006E6700234E6F2073656E736F7220666FD9
:1003C0007220504D21004E6F2073656E736F722145
:1003D00000206E672F4C00504D313A322E353A31A5
:1003E00030004D6561737572696E672E2E00234E65
:1003F0006F2054422073656E736F723F00234E6FFF
:100400002073656E736F722100536F756E64204C9C
:100410006576656C004D6561737572696E672E2E29
:1004200000234E6F2073656E736F722100536F75DA
:100430006E64204C6576656C00234E6F2073656E8C
:10044000736F7220666F722074656D70202620684D
:10045000756D696469747921004E6F2053656E7300
:100460006F72210020666F722074656D70202620E7
:1004700068756D696469747921002353656E736FC3
:1004800072204572726F72200053656E736F722016
:100490004572726F7221002357726F6E6720736509
:1004A0006E736F7220666F722074656D70202620E7
:1004B00068756D6964697479210057726F6E672081
:1004C00053656E736F72210054656D702048756DB1
:1004D0006964697479004C6967687420496E746551
:1004E0006E7369747900466C616D652049520048ED
:1004F0002D6669656C6400536561726368204469A8
:1005000072656374696F6E00234E6F2070482073AC
:10051000656E736F72210070482076616C7565009E
:1005200023496E76616C6964206B65792100204DEA
:10053000756C746973656E736F7273004D756C744E
:100540006973656E736F72730044697361626C6581
:1005500000456E61626C65005265626F6F74696E12
:10056000672E2E2E002344413A2D3233002372652C
:10057000706C6965733D002353657474696E6773AD
:10058000206F6620616C6C2073656E736F72733AB6
:10059000002353697A65206F66206865616465721F
:1005A000202B20616C6C2073656E736F72733A2020
:1005B000002353697A65206F6620686561646572FF
:1005C0003A20002320616E64207265616479207492
:1005D0006F207573652100206D6F62696C65206CFA
:1005E0006F6767657220737461727465642000437D
:1005F000616C6962726174696F6E205072657373A9
:100600007572653D00536561206C6576656C2050A0
:100610002863616C63293D00234572726F723A70E2
:100620007265737375726520424D503038352C20D9
:10063000636865636B20776972696E672100495250
:100640002054656D702073656E736F7220666F75D0
:100650006E6400504D322E352073656E736F7220BC
:100660006C696B656C7920666F756E6400206D6FC8
:1006700062696C65206C6F67676572207374617264
:10068000746564202E2E2E2000576946692049503B
:100690003A002357694669204950206164647265B5
:1006A00073733A2000456455484B205345534C6FB3
:1006B000676765720053656E736F7220736C6F7439
:1006C00020616E6420747970653A0057656C636FC1
:1006D0006D6520746F20456455484B0023456E645A
:1006E000206F66204D756C746973656E736F722030
:1006F0004379636C6523002354696D6520647572CA
:100700006174696F6E3D002354696D6520696E7474
:10071000657276616C3D00576946692049503A0020
:10072000234D5320456E61626C656400234D532058
:1007300044697361626C6564002352657374207050
:100740006172616D657465727320746F2064656693
:1007500061756C742076616C756573004C6F6767AA
:100760006572204E616D653A200067657453656C53
:10077000665465737442697428293A200069734984
:100780006E74657272757074456E61626C65642812
:1007900031293A2000676574496E7465727275700C
:1007A000744D617070696E672831293A2000676561
:1007B00074496E74657272757074536F7572636587
:1007C0002831293A2000676574496E746572727524
:1007D0007074536F7572636528293A2000676574D9
:1007E0005261746528293A20332E31343135393F2E
:1007F00000616363656C2E69734C6F77506F77652A
:100800007228293A2000616363656C2E6973417315
:100810006C65657028293A2000616363656C2E69F8
:1008200073546170536F757263654F6E5A28293A1D
:100830002000616363656C2E6973546170536F753A
:100840007263654F6E5928293A2000616363656CB5
:100850002E6973546170536F757263654F6E5828BB
:10086000293A2000616363656C2E69734163746982
:1008700076697479536F757263654F6E5A28293A99
:100880002000616363656C2E6973416374697669E6
:100890007479536F757263654F6E5928293A200039
:1008A00069734163746976697479536F75726365AE
:1008B0004F6E5828293A200069735461704465745A
:1008C000656374696F6E4F6E5A28293B2066616CB0
:1008D00073653F2000697354617044657465637487
:1008E000696F6E4F6E5A28293B20747275653F20E0
:1008F000006973546170446574656374696F6E4F09
:100900006E5928293B2066616C73653F200069732E
:10091000546170446574656374696F6E4F6E5928D5
:10092000293B20747275653F2000697354617044DF
:100930006574656374696F6E4F6E5828293B206635
:10094000616C73653F200069735461704465746520
:100950006374696F6E4F6E5828293B2074727565F9
:100960003F200067657453757070726573734269D8
:100970007428293B2066616C73653F2000676574AD
:10098000537570707265737342697428293B2074C3
:100990007275653F20006973416374697669747983
:1009A000416328293A20006973496E61637469764E
:1009B0006974795A456E61626C656428293A200031
:1009C0006973496E616374697669747959456E61BA
:1009D000626C656428293A20006973496E6163740A
:1009E000697669747958456E61626C656428293A44
:1009F0002000697341637469766974795A456E6140
:100A0000626C656428293A200069734163746976D1
:100A100069747959456E61626C656428293A2000D1
:100A20006973416374697669747958456E61626C63
:100A3000656428293A2000676574467265654661D9
:100A40006C6C4475726174696F6E28293A20006776
:100A500065744672656546616C6C5468726573684E
:100A60006F6C6428293A200067657454696D654984
:100A70006E616374697669747928293A2000676524
:100A800074496E61637469766974795468726573C8
:100A9000686F6C6428292000676574416374697607
:100AA0006974795468726573686F6C6428292000D2
:100AB000676574446F75626C6554617057696E64E4
:100AC0006F7728292000676574446F75626C6554E0
:100AD00061704C6174656E637928293A20006765FE
:100AE000745461704475726174696F6E28293A207C
:100AF00000676574417869734F666673657428266C
:100B0000782C2026792C20267A293A2000676574D3
:100B10005461705468726573686F6C6428293A2058
:100B20000058595A2047733A200058595A20434FC9
:100B3000554E54533A2000736574206761696E7393
:100B40005B5D3A006761696E735F6F7269675B5DD9
:100B50003A00696E7075742044535463616C696225
:100B6000726174653A0020766F6C746167653D0050
:100B70002354757262696469747920557070657266
:100B8000204C696D69743A200020766F6C7461673F
:100B9000653D0023547572626964697479204C6FF5
:100BA000776572204C696D69743A20002354757220
:100BB000626964697479204C6F776572204C696D45
:100BC00069742056696E663A20004D617820726122
:100BD0006E67653D0023566F6C74616765207365B1
:100BE0006E736F723A00342D32306D4100414353C1
:100BF000373132204D61783D004143533731322047
:100C00004D61783D3541002343757272656E7420E5
:100C100073656E736F723A00234453205468657293
:100C20006D6F6D657465722063616C696272617469
:100C3000656420666F72202300234E6F206E656509
:100C40006420746F2063616C6962726174652063F3
:100C5000757272656E742073656E736F72210023F6
:100C60004143533731322063757272656E7420735D
:100C7000656E736F72206F666673657420563D00F3
:100C8000235556207A65726F20766F6C74616765A4
:100C9000203D00234F3220766F6C253D00234F32DC
:100CA0002063616C6962726174696F6E3A2000231F
:100CB000566F6C746167652870483D3130293A0081
:100CC00023566F6C746167652870483D34293A007B
:100CD000232D2D2D2D2D2D2D2D2D2D2D2D2D2D2D4E
:100CE0002D2D2D2D2D2D2D2D2D2D2D2D2D2D2D2D34
:100CF0002D2D2D2D2D00235265736F6C7574696F2A
:100D00006E3A20202000234D696E2056616C756577
:100D10003A2020202000234D61782056616C7565B3
:100D20003A202020200023556E69717565204944C2
:100D30003A2020202000234472697665722056658F
:100D4000723A202020002353656E736F723A202080
:100D5000202020202000232D2D2D2D204D61676E79
:100D6000657469632053656E736F72202D2D2D2D70
:100D70002D2D2D2D2D2D2D2D2D2D2D2D2D2D2D2DA3
:100D800000482D6669656C643A20280020202020E8
:100D90002020202020202020202020002020202073
:100DA000202020202020202020202000233A5368CB
:100DB0006F772F48696465204C4344002A3A546891
:100DC00069732048656C700044233A43616C696222
:100DD000726174696F6E00442A3A53657474696E67
:100DE00067730044423A5265736574204C6F6767BD
:100DF00065720044433A436C656172204C43440081
:100E000044443A4D756C746953656E736F72730028
:100E100044393A43757272656E7400566F6C746132
:100E200067652B43757272656E740044383A456C81
:100E30006563747269630044373A4D6F74696F6E0D
:100E40000044363A44532054656D700044353A5599
:100E50005620496E74656E736974790044343A4F54
:100E60003220636F6E632E0044333A434F32206367
:100E70006F6E632E0044323A504D28313A322E358F
:100E80003A3130290044323A504D28313A322E3529
:100E90003A3130292A0044313A54757262696469E2
:100EA00074790044303A566F6C7461676500393A62
:100EB0006F7220334420616363656C2E00393A49B8
:100EC0006E636C2E20616E672E00383A7048207673
:100ED000616C756500373A49522054656D70003772
:100EE0003A49522054656D702A00363A4D61676E5A
:100EF00065746963206669656C6400353A4761739F
:100F0000204C6576656C00343A495220466C616D20
:100F10006500333A4C6967687420496E742E00325C
:100F20003A616E642048656967687400323A5465B6
:100F30006D7020507265737375726500313A546537
:100F40006D702048756D696469747900303A536F2B
:100F5000756E64204C6576656C00303A536F756E23
:100F600064204C6576656C2A0054696D65206C615F
:100F70007073653A00576946692049503A00005E2F
:100F8000BCE2613FDD83C29C7E20A3FD1F41009D2A
:100F900023BE46DB65F88C11AF32CA57E974697419
:100FA00065726174696F6E3D0073656E736F722355
:100FB0003D0043757272656E74207374617475734D
:100FC0003A206379636C653D006E6379636C653DBF
:100FD000006E73656E736F72733D006D61786E7332
:100FE000656E736F72733D00656E61626C65643D22
:100FF00000234D756C746973656E736F7273206D29
:101000006561737572656D656E742073657474695E
:101010006E67733A0046696E64696E672057694669
:1010200069204950007365703D006976616C3D0030
:101030006E697465723D00230043616C2E20466129
:10104000696C65640043616C2E20446F6E65004ED0
:101050006F206E6565642100496E76616C6964205D
:101060005028506129005365614C6576656C2050AD
:10107000285061293A0043616C696272617465208D
:1010800050004453542054656D702073656E736F27
:10109000720043757272656E742073656E736F7241
:1010A000004F322073656E736F7200555620736562
:1010B0006E736F720043616C6962726174650046A1
:1010C00061696C65640054422063616C2E20646F1A
:1010D0006E65005570706572204C696D69743A3E9A
:1010E000004C6F776572204C696D69743A3E00540C
:1010F0007572626964697479004661696C6564003F
:1011000070482063616C2E20646F6E6500704831FA
:101110003020507265737320420070483420507242
:1011200065737320410043616C696272617465008C
:10113000416E676C65732F003E6128782C792C7A9C
:10114000292F673A004E6F2073656E736F7221000E
:1011500049522054656D7065726174757265004DF9
:101160006561737572696E672E2E004E6F20736510
:101170006E736F723F0049522054656D70657261E5
:1011800074757265004D6561737572696E672E2E98
:10119000004F6666206169722D636F6E642100499D
:1011A00074277320746F6F20636F6F6C2100546518
:1011B0006D702069732066696E6521004973206136
:1011C00069722D636F6E64206F6E3F0049742773E0
:1011D00020717569746520686F74210049742773E4
:1011E000207665727920686F742120004F66662032
:1011F0006169722D636F6E642100497427732074D6
:101200006F6F20636F6F6C210054656D7020697380
:101210002066696E6521004973206169722D636FD4
:101220006E64206F6E3F0049742773207175697476
:101230006520686F74210049742773207665727980
:1012400020686F74210054656D702048756D696465
:10125000697479004E6F2053656E736F7221004E72
:101260006F20445320546865726D6F6D65746572AC
:101270002100445320546865726D2E004D6F7469CF
:101280006F6E00556E6B6E6F776E00496E6475738E
:10129000747269616C20342D32306D4100414353CA
:1012A000373132204D61783D3541002343757272EC
:1012B000656E742073656E736F723A0000002100D2
:1012C000240027002A002D00300033000101000017
:1012D000040107010A0100002200250028002B005C
:1012E0002E003100340002010000050108010B014D
:1012F000000020002300260029002C002F003200CF
:1013000000010000030106010901050505050705A7
:1013100008080808020202020A0A08080404040471
:10132000010101010101010103030303030303039D
:10133000040707070C0C0C0C0C0C0C0C020202022C
:1013400006060606060606060B0B0B0B0B0B0B0B15
:1013500001021020200808102040102040800201C7
:1013600002010804020101020408102040808040AC
:1013700020100804020180040201804020100804AB
:101380000201080402010102040810204080010249
:1013900004081020408000000A0B02090C0D0E0802
:1013A000070304010000000000000000000000002E
:1013B000000000000000000000000000000000002D
:1013C00000001211100000000000000000000000EA
:1013D000000000000000000000000000496E76617F
:1013E0006C6964206B65792100202020202020205A
:1013F000202020202020202020002020202020200D
:1014000020202020202020202020002020202020FC
:1014100020202020202020202020200020202020EC
:10142000202020202020202020202020004E455455
:101430003D426C7565746F6F7468204C45004E4575
:10144000543D426C7565746F6F7468004E45543D31
:10145000576946690053657474696E67204661690F
:101460006C65640053657474696E6720446F6E65C3
:10147000004368616E6765204E6574776F726B3EDE
:1014800000547970653A0042542F57694669204EDE
:101490006574776F726B004368616E676520536592
:1014A0006E736F723E0043757272656E7420536581
:1014B0006E736F72004F7468657200496E642E20FF
:1014C000342D32306D4100414353373132203C33AB
:1014D000304100414353373132203C3230410041EA
:1014E0004353373132203C3541003E4D6178205620
:1014F0006F6C743A3E004368616E676520766F6C6E
:10150000746167653E00547970652000566F6C7495
:101510006167652053656E736F72004368616E6723
:1015200065207479706520746F0053656E736F72F7
:101530003D4448540054656D702048756D69646978
:10154000747900002CA7FCA611241FBECFEFD1E2B6
:10155000DEBFCDBF00E00CBF1BE0A0E0B2E0E2E9DF
:10156000FCE601E00BBF02C007900D92AA3EB10756
:10157000D9F723E1AAEEBBE001C01D92AF39B20753
:10158000E1F71AE0C3EADAE000E006C021970109BA
:10159000802FFE010E946FB3C23AD10780E0080796
:1015A000A9F70E944C9A0C9438B60C9400002F9224
:1015B0003F924F925F926F927F928F929F92AF92E3
:1015C000BF92CF92DF92EF92FF920F931F93CF9330
:1015D000DF93CDB7DEB7C554D1090FB6F894DEBF9F
:1015E0000FBECDBF8C01E090090CF0900A0C8091E9
:1015F0009713882349F06DE675E080E19FE00E9433
:10160000C24CC8010E947951680125E0C20ED11C6C
:1016100035E0C316D10420F18091090C90910A0C99
:101620000817190729F10E94DC3E0E944A760C3EF9
:101630004FEF140724F010930A0C0093090CB80123
:10164000CE0101960E947C50BE016F5F7F4F8CE2FD
:1016500092E10E940F4BCE0101960E94F24B08C00E
:101660000E3F5FEF150721F40E945A760C94CC1DB3
:101670006FEB79E080E292E10E94C84BF5E0CF1673
:10168000D10490F068ED7BE0CE0101960E94564CAB
:101690004AE050E06FEF7FEFCE0101960E9460902C
:1016A000CE0101960E94F24BF8017C96E632F105DC
:1016B00010F00C94D81C8827EE58FF4F8F4F0C94D5
:1016C0006FB30E94DC3E89E390E00E94257120E028
:1016D00030E04AE754E40E940AAFAB01BC0121E0CC
:1016E000CE0101960E94F74B60E178E0CE01809632
:1016F0000E94564CBE016F5F7F4FCE0180960E94C4
:10170000724B61EC75E00E945B4BBC0180E292E1A0
:101710000E94DD4BCE0180960E94F24BCE010196D5
:101720000E94F24B65EC75E08AE192E10E94C84BA1
:101730006AE172E1CE0101960E944E4C4AE050E00F
:1017400068E070E0CE0101960E94BB8FCE01019649
:101750000E94F24B60E272E1CE0101960E944E4C73
:101760004AE050E06FEF7FEFCE0101960E94738D4B
:10177000CE0101960E94F24B6AE172E180E292E1B1
:101780000E94094B8091450C882311F40C940A1D8A
:101790000C945117C090B902D090BA020E94DC3E5E
:1017A00089E390E00E94257120E030E04AE754E4AC
:1017B0000E940AAF0E9494B1CE0101960E947C5013
:1017C00060E178E0CE0180960E94564CBE016F5FCA
:1017D0007F4FCE0180960E94724B61EC75E00E94B3
:1017E0005B4BBC0180E292E10E94DD4BCE01809612
:1017F0000E94F24BCE0101960E94F24B809124127E
:1018000090912512099718F423E0F22E02C092E07D
:10181000F92E8091B7108330E4F4C6010E94B378AA
:101820004B015C016091B8107091B910072E000C4B
:10183000880B990B0E94ABAEA50194010E940AAFE0
:1018400020E030EC4FE754E40E94FBB0AB01BC0158
:1018500003C040E050E0BA012F2DCE0101960E9456
:10186000F74B6AEF75E0CE0180960E94564CBE01A0
:101870006F5F7F4FCE0180960E94724B6DEC75E0DA
:101880000E945B4BBC0180E292E10E94094BCE01B9
:1018900080960E94F24BCE0101960E94F24B60EDC1
:1018A00075E042CF8091450C882309F42CC186ED68
:1018B0009DE00E940D8E61E0809102020E94A5854C
:1018C00060E0809100020E94A5850E949A970E9484
:1018D000E05B0E94FD5BAB01BC0123E0CE01809682
:1018E0000E94F74BBE01605E7F4FCE0101960E94C1
:1018F0004E4C67EF75E0CE0101960E945B4BBC0138
:101900008AE192E10E94DD4BCE0101960E94F24BEA
:10191000CE0180960E94F24B6BEF79E0CE010196EA
:101920000E94564C6AE172E1CE0101960E94724B10
:10193000BC0180E292E10E94DD4BCE0101960E9443
:10194000F24B0E94FD5B6B017C010E9406864B01FD
:101950005C016EE170E080E090E00E942B860E94C6
:10196000FD5B2B013C010E9406869B01AC012819FE
:1019700039094A095B0949015A0131ED831637E0FB
:101980009306A104B1040CF441C0A7019601C30160
:10199000B2010E9434B06B017C0120E030E0A9016B
:1019A0000E94EAB118165CF426EA3BE944EC5BE3DA
:1019B000C701B6010E94A5AE87FF0BC027C026EA6B
:1019C0003BE944EC5BEBC701B6010E94EAB1181693
:1019D000ECF0C501B40128EE33E040E050E00E9495
:1019E000D7AFCA01B9010E94ABAE4B015C0120E048
:1019F00030E04AE754E4C701B6010E940AAFA501EE
:101A000094010E94FBB0AB01BC0103C040E050E078
:101A1000BA0122E0CE0180960E94F74BBE01605EC3
:101A20007F4FCE0101960E944E4C69ED75E0CE01CC
:101A300001960E945B4BBC0184E192E10E94DD4B68
:101A4000CE0101960E94F24BCE0180960E94F24B8D
:101A50006DED75E0CE0101960E94564C64E172E195
:101A6000CE0101960E94724BBC0180E292E10E947D
:101A7000094BCE0101960E94F24B68ED7BE0CE014E
:101A800001960E94564C64E172E1CE0101960E94DB
:101A9000724BBC018AE192E10E94094BCE01019692
:101AA0000E94F24B69E573E0CE0101960E94464C1C
:101AB0004AE050E060E070E0CE0101960E94BB8FEA
:101AC000CE0101960E94F24B6AE172E1CE010196CD
:101AD0000E944E4C45E050E06FEF7FEFCE01019643
:101AE0000E94738DCE0101960E94F24B61EE75E06B
:101AF00080E292E10E94FB4A60E0809102020E9433
:101B0000A5850C940A1D6091550270915602809132
:101B10005702909158020E94EB790C940A1D809113
:101B20005B0290915C020E94EE7B0C940A1D409136
:101B30005D0226964FAF269760E0842F0E94A58510
:101B40008091450C811109C08091151181110EC041
:101B50008FE090E0A0E0B0E00DC023E030E040E096
:101B600050E02CAF3DAF4EAF5FAF08C083E090E0D8
:101B7000A0E0B0E08CAF9DAFAEAFBFAF68E673E062
:101B800080E292E10E94834B60E272E1CE01019615
:101B90000E944E4C4AE050E06FEF7FEFCE0101967D
:101BA0000E94BB8FCE0101960E94F24B21961FAE80
:101BB000219725961FAE2597212C312CC12CD12C95
:101BC000760182E3682E712C812C912C540126968B
:101BD0008FAD26970E94E185092E000CAA0BBB0B46
:101BE000880E991EAA1EBB1E65E070E080E090E0A2
:101BF0000E942B8691E0691A710849F740902102F2
:101C0000509022026090230270902402C501B4011A
:101C10000E94ABAE20E030E040EA50E40E940AAF00
:101C200020E030E040E85AE30E940AAF20E030E0D4
:101C300048E452E40E94FBB0A30192010E9434B038
:101C400020E030E040E751E40E940AAF4B015C0124
:101C5000A30192016AE979E989E390E40E9434B032
:101C60009B01AC01C501B4010E94FBB020E030E053
:101C7000A9010E9435B020E030E040E251E40E942A
:101C80000AAF4B015C0121962FAD219725963FAD00
:101C90002597A1010E94EAB118163CF421968FAE57
:101CA000219725969FAE2597150120E030E0A901E8
:101CB000B401C5010E94A5AE87FF04C0812C912C00
:101CC000A12CB12C22E0A401B501CE0180960E9486
:101CD000F74BBE01605E7F4FCE0101960E944E4CD5
:101CE00064EF75E0CE0101960E945B4BBC018AE176
:101CF00092E10E94DD4BCE0101960E94F24BCE0193
:101D000080960E94F24B6AE172E1CE0101960E9438
:101D10004E4C4AE050E060E070E0CE0101960E9437
:101D2000738DCE0101960E94F24B0E9487878090AE
:101D30008F1390909013A0909113B0909213A4E6FB
:101D40008A0E911CA11CB11C86169706A806B9061E
:101D500010F40C942B1D0E9487870E94A9AE4B01A2
:101D60005C0160918F137091901380919113909109
:101D700092130E94ABAE20E030E048EC51E40E94A8
:101D800035B09B01AC01C501B4010E94A5AE87FF2F
:101D900002C00C942B1D6CE370E080E090E00E9488
:101DA0002B86BFEFCB1ADB0AEB0AFB0A2CAD3DAD4D
:101DB0004EAD5FAD2C153D054E055F050CF001CF16
:101DC00064E670E080E090E00E942B860E94DC3E9A
:101DD00064E670E080E090E00E942B8660E673E0AD
:101DE0008AE192E10E94834B6AE172E1CE010196A1
:101DF0000E944E4C44E150E060E070E0CE0101965C
:101E00000E94BB8FCE0101960E94F24B22E02196E8
:101E10004FAD219725965FAD2597B101CE018096F4
:101E20000E94F74BBE01605E7F4FCE0101960E947B
:101E30004E4C64EF75E0CE0101960E945B4BBC01F5
:101E40008AE192E10E94DD4BCE0101960E94F24BA5
:101E5000CE0180960E94F24B6AE172E1CE010196BA
:101E60000E944E4C42E350E06FEF7FEFCE010196AF
:101E70000E94738DCE0101960E94F24B64E170E0E6
:101E800080E090E00E942B860E94003F6EE170E0AF
:101E900080E090E00E942B866EE170E080E090E0B0
:101EA0000E942B8669EF75E0CE0101960E94564C88
:101EB0006AE172E1CE0101960E94724B6DEF75E00E
:101EC0000E945B4B60E272E10E94724BBC0180E2B7
:101ED00092E10E94DD4BCE0101960E94F24B0C94E0
:101EE0000A1D80915F029091600299270E94B37849
:101EF0002DE038E643E55BE30E940AAF6B017C010D
:101F00002091830230918402409185025091860293
:101F10000E94A5AE18164CF060916B0270916C0295
:101F200080916D0290916E021BC0209197023091BA
:101F300098024091990250919A02C701B6010E94FD
:101F4000EAB187FF05C0C701B6010E94F16C08C065
:101F500060917F0270918002809181029091820253
:101F600020E030E048EC52E40E940AAF20E030E08C
:101F700048EA51E40E940AAF2091250230912602DE
:101F800040912702509128020E94FBB06B017C0116
:101F900065E773E08AE192E10E94834B6AE172E1B6
:101FA000CE0101960E944E4C42E350E060E070E0AA
:101FB000CE0101960E94BB8FCE0101960E94F24B8A
:101FC00022E0B701A601CE0101960E94F74B67E01F
:101FD00076E0CE0180960E94564CBE016F5F7F4F27
:101FE000CE0180960E94724B61E076E00E945B4BCE
:101FF000BC0180E292E10E94DD4BCE0180960E94FE
:10200000F24BCE0101960E94F24B60E272E1CE01EA
:1020100001960E944E4C42E350E06FEF7FEFCE01FD
:1020200001960E94738DCE0101960E94F24B809121
:10203000450C882311F40C940A1D60E273E080E0E3
:1020400090E00E942B860C940A1D0E94DC3E69EAF7
:1020500073E080E292E10E94834B60E272E1CE0184
:1020600001960E944E4C4AE050E060E070E0CE01E4
:1020700001960E94BB8FCE0101960E94F24B60EA4E
:1020800073E08AE192E10E94834B6AE172E1CE0142
:1020900001960E944E4C44E150E06FEF7FEFCE017D
:1020A00001960E94738DCE0101960E94F24B8091A1
:1020B000EE0B9091EF0B8230910549F40E946386FC
:1020C00081111AC01092EF0B1092EE0B15C0892BE4
:1020D000C9F40E946386882339F082E090E09093EF
:1020E000EF0B8093EE0B08C00E9463868111F5CF41
:1020F0000E9463868111F1CF8091EE0B9091EF0BDE
:10210000029741F164E973E080E292E10E94834B1F
:1021100060E272E1CE0101960E944E4C4AE050E02E
:1021200060E070E0CE0101960E94BB8FCE01019667
:102130000E94F24B60E272E1CE0101960E944E4C89
:1021400068ED7BE0CE0101960E945B4B6AE172E193
:102150000C94321A8AE090E00E9486766B017C0132
:1021600020E030E0A9010E94A5AE181634F08AE004
:1021700090E00E9486766B017C01BBE0AB2EB12C17
:1021800020E030E042ED53E4C701B6010E94A5AE65
:1021900018168CF031E0A31AB10869F068EC70E011
:1021A00080E090E00E942B8683E090E00E9486769B
:1021B0006B017C01E5CF20E030E0A901C701B60149
:1021C0000E94A5AE18163CF066E873E080E292E14A
:1021D0000E94834B31C020E030E048EC52E4C7015C
:1021E000B6010E94A5AE87FF02C021E001C020E039
:1021F000B701A601CE0101960E94F74B66E076E09A
:10220000CE0180960E94564CBE016F5F7F4FCE017B
:1022100080960E94724B6BE076E00E945B4BBC01A3
:1022200080E292E10E94DD4BCE0180960E94F24B4B
:10223000CE0101960E94F24B60E272E1CE0101965E
:102240000E944E4C42E350E06FEF7FEFCE010196CB
:102250000E94738DCE0101960E94F24B6DE773E0F0
:102260008AE192E10E94834B6AE172E1CE0101961C
:102270000E944E4C42E350E060E070E0CE010196D7
:102280000E94BB8FD0CE0E9487872B013C0186ED38
:102290009DE00E940D8E64E670E080E090E00E9478
:1022A0002B8640E855E260E070E086ED9DE00E94FC
:1022B000D06D64E670E080E090E00E942B8662EED4
:1022C00073E08AE192E10E94834B6AE172E1CE0100
:1022D00001960E944E4C42E350E06FEF7FEFCE013B
:1022E00001960E94BB8FCE0101960E94F24B67EDD2
:1022F00073E08AE192E10E94834B6AE172E1CE01D0
:1023000001960E944E4C42E350E06FEF7FEFCE010A
:1023100001960E94738DCE0101960E94F24B80912E
:102320000F0C9091100C8D7F1CAEA12CB12CC12CE8
:10233000D12CE12CF12C019709F46FC0AE01405E65
:102340005F4F59AF48AFCE014E969BAF8AAF0E9408
:102350008787DC01CB0184199509A609B709883B59
:102360009B40A105B10508F058C086ED9DE00E9494
:10237000AC47892B09F44AC02CED35E040E050E031
:102380002093DA0D3093DB0D4093DC0D5093DD0D7F
:102390000E949C6D97FD06C082349105C9F780E0CC
:1023A00090E002C08FEF9FEF892B81F5AE014F5F68
:1023B0005F4F1A014A010E949C6D97FF06C08981F8
:1023C0008D3421F520E030E009C0D4018D934D011A
:1023D000E8ADF9ADEA17FB0771F7F1CFD1018D91A7
:1023E0001D01280F311DEAADFBADAE17BF07B1F7D8
:1023F0002E5B3F4F8E8D90E0982F88274F8D840F56
:10240000911D2817390711F40C942F1D62E370E019
:1024100080E090E00E942B869ACF0E948787DC01A3
:10242000CB0184199509A609B709883B9B40A105F2
:10243000B10518F42CAD2111BDC00E94DC3E6AE14B
:1024400072E1CE0180960E944E4C42E350E066E07D
:1024500070E0CE0180960E94BB8FCE0180960E94D4
:10246000F24B3CAD332311F40C94481D82E090E014
:102470009093100C80930F0CB501CE0180960E94B2
:102480007C50B601CE0186960E947C50B701CE01E9
:10249000C2960E947C50BE016E5C7F4FCE018C962E
:1024A0000E944E4C66E177E0CE018C960E945B4B19
:1024B000BE016A5D7F4F0E94724B66E177E00E9429
:1024C0005B4BBE01605E7F4F0E94724BBC0180E29D
:1024D00092E10E94DD4BCE018C960E94F24BCE0120
:1024E000C2960E94F24BCE0186960E94F24BCE011C
:1024F00080960E94F24B60E272E1CE0180960E94CB
:102500004E4C4AE050E06FEF7FEFCE0180960E9484
:10251000738DCE0180960E94F24B61ED73E081E2F3
:1025200093E10E94C24CB501CE0180960E947C507E
:10253000B601CE0186960E947C50B701CE018C96E2
:102540000E947C506FE076E0CE01C2960E94564C0D
:10255000BE01645D7F4FCE01C2960E94724B68ED52
:102560007BE00E945B4BBE016A5D7F4F0E94724B15
:1025700068ED7BE00E945B4BBE01605E7F4F0E9476
:10258000724B6FE176E00E945B4BBC0180E292E10E
:102590000E94DD4BCE01C2960E94F24BCE018C967A
:1025A0000E94F24BCE0186960E94F24BCE0180969D
:1025B0000E94F24B62E370E080E090E00E942B8684
:1025C00086ED9DE00E940D8E12C6E0905902F090BB
:1025D0005A0265E276E08AE192E10E94C84B0E94CD
:1025E000DC3E6AE172E1CE0101960E944E4C4AE067
:1025F00050E06FEF7FEFCE0101960E94BB8FCE01BE
:1026000001960E94F24BC7010E94C47924966CAFD8
:102610007DAF8EAF9FAF249780902F0290903002B5
:10262000A0903102B0903202A501940160912B027A
:1026300070912C0280912D0290912E020E9434B054
:102640002B013C0120E030E0A9010E94A5AE8823C7
:1026500009F453C0C0903702D0903802E09039029C
:10266000F0903A0220E030E0A901C701B6010E94D3
:10267000A5AE18160CF041C080913302909134023F
:10268000A0913502B09136028CAF9DAFAEAFBFAF17
:102690009C01AD01C701B6010E94A5AE882369F176
:1026A000A70196016CAD7DAD8EAD9FAD0E94FBB0D4
:1026B0000E9430B26CAF7DAF8EAF9FAFA501940189
:1026C00024966CAD7DAD8EAD9FAD24970E9434B045
:1026D000A30192010E94FBB02CAD3DAD4EAD5FADAC
:1026E0000E940AAF0E9468B19B01AC01C701B6010C
:1026F0000E940AAF6B017C0103C0C12CD12C760172
:102700006AE172E1CE0101960E944E4C4AE050E02F
:1027100060E070E0CE0101960E94BB8FCE01019671
:102720000E94F24B20E030E64AEE56E4C701B601C3
:102730000E94EAB118163CF46EEE73E080E292E17A
:102740000E94834B25C021E0B701A601CE018096EF
:102750000E94F74B6FE276E0CE0101960E94564C44
:10276000BE01605E7F4FCE0101960E94724B63E313
:1027700076E00E945B4BBC0180E292E10E94DD4B5F
:10278000CE0101960E94F24BCE0180960E94F24B40
:1027900060E272E1CE0101960E944E4C4AE050E0A8
:1027A0006FEF7FEFCE0101960E94738DCE010196EF
:1027B0000E94F24B64E670E080E090E00E942B867D
:1027C00036CCE090B902F090BA020E94DC3E65E09F
:1027D00070E080E090E00E942B868091B7108330FB
:1027E000E4F4C7010E94B3786B017C016091B810DA
:1027F0007091B910072E000C880B990B0E94ABAE9C
:10280000A70196010E940AAF20E030EC4FE754E4A4
:102810000E94FBB0AB01BC0103C040E050E0BA0134
:1028200023E0CE0101960E94F74B6AEF75E0CE01DE
:1028300080960E94564CBE016F5F7F4FCE018096FE
:102840000E94724B6DEC75E00E945B4BBC0180E214
:1028500092E10E94DD4BCE0180960E94F24BCE01A8
:1028600001960E94F24B67E376E00C94940B9091F2
:10287000080C81E089278093080C8091450C8823FF
:1028800031F060E272E189E39DE00E94C76968EC83
:1028900070E080E090E0D5CB1092450C0C940A1DBE
:1028A00081E08093450C8093231180911A11882335
:1028B00049F16FEE77E08CE292E10E94C84B86EE20
:1028C0009FEF90930A0C8093090C20911D11309179
:1028D0001E1180911F11909120118217930724F0EF
:1028E0001092201110921F111092111110921211BA
:1028F00010921311109214116CE271E080E090E0DC
:102900000E942B866CE272E182E392E10E94DD4B31
:102910008091090C90910A0C9093400C80933F0C8D
:102920000C940A1D0E94333F0C940A1D83E79EE01D
:102930000E940D8E40E052EC61E070E083E79EE083
:102940000E94D06D8CED95E0A0E0B0E08093770E12
:102950009093780EA093790EB0937A0E64E670E0AF
:1029600080E090E00E942B868091EE0B9091EF0B1F
:10297000019759F483E090E00E942779811140C0CB
:102980001092EF0B1092EE0B1AC081E090E00E94C3
:102990002779882339F081E090E09093EF0B8093C2
:1029A000EE0B0DC083E090E00E9427798111F3CFF8
:1029B00083E090E00E9427798111EDCF06C08091DD
:1029C000EE0B9091EF0B0197D9F06DE274E08AE184
:1029D00092E10E94834B6AE172E1CE0101960E946E
:1029E0004E4C44E150E06FEF7FEFCE0101960E9424
:1029F000738DCE0101960E94F24B61E274E0CDC06E
:102A000065E174E080E292E10E94834B60E272E152
:102A1000CE0101960E944E4CCE0101960E948F8FEE
:102A2000CE0101960E94F24B62E370E080E090E0FC
:102A30000E942B8660E272E1CE0101960E944E4C0C
:102A400042E350E06FEF7FEFCE0101960E94BB8F13
:102A5000CE0101960E94F24B69E074E08AE192E1B6
:102A60000E94834B6AE172E1CE0101960E944E4CB6
:102A700044E150E06FEF7FEFCE0101960E94738D2D
:102A8000CE0101960E94F24B8BEB88A38AEA89A3C0
:102A900081E08AA3C12CD12C412C512C3201212C54
:102AA000312CC6016AE070E00E945CB3892B49F4C6
:102AB00043E050E0BE01605E7F4F83E79EE00E94EE
:102AC000514765E070E080E090E00E942B86BFEF08
:102AD000CB1ADB0AE12CF12C812C912C540183E7D9
:102AE0009EE00E94AC47892B81F4E4E08E169104AD
:102AF000A104B10454F094E02916310464F4A0E96F
:102B0000CA16A1E0DA0669F606C0F6E0EF16F1048F
:102B10000CF4EAC7F0CFC301B2010E94ABAE20E0D3
:102B200030E040E251E40E94FBB020E030E040E8B9
:102B30005EE30E940AAF6B017C0120E030E040EAD6
:102B400051E40E94EAB1181634F521E0B701A6015C
:102B5000CE0101960E94F74B61E677E0CE018096A8
:102B60000E94564CBE016F5F7F4FCE0180960E943F
:102B7000724B6FE376E00E945B4BBC0180E292E116
:102B80000E94DD4BCE0180960E94F24BCE01019651
:102B90000E94F24B06C06DEF73E080E292E10E946A
:102BA000834B60E272E1CE0101960E944E4C4AE0F6
:102BB00050E060E070E0CE0101960E94BB8FCE0134
:102BC00001960E94F24B60E272E1CE0101960E94F2
:102BD0004E4C68ED7BE0CE0101960E945B4B6AE1B2
:102BE00072E10E94724BBC0180E292E10E94DD4BD7
:102BF000CE0101960E94F24B83E79EE00E940D8E6B
:102C000016CA68EC74E0CE0101960E94464C4AE078
:102C100050E06FEF7FEFCE0101960E94738DCE01E1
:102C200001960E94F24B6091B7027091B8028091B8
:102C3000290290912A020E94D76EE4E18E2E912CF7
:102C4000A12CB12CC12CD12CAFEFCA1ADA0AC501C4
:102C5000B4010E942B866091B7027091B8028091F6
:102C6000290290912A020E94D76E7C01B3E0CB1614
:102C7000D10434F08EE1C816D10444F4EF2851F0A9
:102C800094E1890E911CA11CB11CDECFE114F1046A
:102C900009F00CC18091290290912A028B30910594
:102CA000C9F480917E1290917F12A0918012B09110
:102CB000811280933F1390934013A0934113B093DC
:102CC000421380917A1290917B12A0917C12B09164
:102CD0007D121DC08631910521F30C9701F580917D
:102CE000321390913313A0913413B0913513809324
:102CF0003F1390934013A0934113B09342138091DC
:102D00002E1390912F13A0913013B0913113809313
:102D10003B1390933C13A0933D13B0933E1340910B
:102D20003F1350914013609141137091421321E081
:102D3000CE0101960E94F74B6DE07AE0CE018096BD
:102D40000E94564CBE016F5F7F4FCE0180960E945D
:102D5000724BBC0180E292E10E94DD4BCE01809675
:102D60000E94F24BCE0101960E94F24B40913B1320
:102D700050913C1360913D1370913E1321E0CE01C0
:102D800001960E94F74B62E476E0CE0180960E94A5
:102D9000564CBE016F5F7F4FCE0180960E94724BF2
:102DA000BC0180E292E10E94094BCE0180960E9414
:102DB000F24BCE0101960E94F24B64E076E080E295
:102DC00092E10E94FB4A6FEB79E0CE0101960E94EE
:102DD000564C44E150E060E070E0CE0101960E9464
:102DE000BB8FCE0101960E94F24BC0903F13D09052
:102DF0004013E0904113F090421320E030E0A9012D
:102E0000C701B6010E94EAB120E030E040E05FE394
:102E100087FD05C0C701B6010E9435B004C0C701D7
:102E2000B6010E9434B00E9494B1AB01BC01CE0146
:102E300001960E94816ABE016F5F7F4F8AE192E135
:102E40000E940F4BCE0101960E94F24B60E087E09A
:102E50000E94566A6AE172E181E293E10E94B44CF9
:102E60006FED81E293E10E94AD4C68E476E081E28F
:102E700093E10E948D4D60913B1370913C138091C2
:102E80003D1390913E130E9494B14AE050E081E2DC
:102E900093E10E94434D64E076E081E293E10E9479
:102EA0008D4D64E670E080E090E0CBC8EFEFEE1669
:102EB000FE06ACF06AEB74E0CE0101960E94464C2F
:102EC0004AE050E060E070E0CE0101960E94BB8FC6
:102ED000CE0101960E94F24B67E974E048C0FEEF14
:102EE000EF16FFEFFF0679F169E874E0CE01019675
:102EF0000E94464C4AE050E060E070E0CE0101964E
:102F00000E94BB8FCE0101960E94F24B6AE774E0EB
:102F100080E292E10E94834BB701CE0101960E94AC
:102F20007C50BE016F5F7F4F80E292E10E94094BAF
:102F3000CE0101960E94F24B64E674E080E292E1D9
:102F40000E94B94A67C569E574E0CE0101960E9406
:102F5000464C4AE050E060E070E0CE0101960E94ED
:102F6000BB8FCE0101960E94F24B69E374E080E2D0
:102F700092E10E94834B4EC580910402882309F49C
:102F800049C56FEB79E0CE0101960E94564C4AE0AC
:102F900050E061E070E0CE0101960E94BB8FCE014F
:102FA00001960E94F24B0E94F98B34C58091450C2A
:102FB00081110AC080911511811106C07EE1472E52
:102FC000512C612C712C05C063E0462E512C612CD4
:102FD000712C66ED74E080E292E10E94834B60E226
:102FE00072E1CE0101960E944E4C4AE050E06FEF34
:102FF0007FEFCE0101960E94738DCE0101960E9453
:10300000F24B812C912C54011CAE1DAE1EAE1FAE96
:1030100083E20E943B6A87E090E00E94366A0E9449
:10302000346A66E970E080E090E00E942B8683E2DB
:103030000E943B6A80E290E00E94366A0E94346AF5
:1030400066E970E080E090E00E942B8662E070E02C
:1030500083E290E00E94298FC12CD12C76018091CF
:103060006D1390E020916E13821B910918161906BA
:103070006CF48DEA9FE00E94FC55FE2CED2CDC2CBC
:10308000CC24C80ED11CE11CF11CE9CFC701B6014C
:103090000E94ABAE2AE939E949E95FE30E94FBB03F
:1030A0000E9494B1AB01BC0184169506A606B70632
:1030B00014F44A015B01CE0180960E94816ABE0130
:1030C000605E7F4FCE0101960E944E4C6BE476E02D
:1030D000CE0101960E945B4BBC018AE192E10E9405
:1030E000DD4BCE0101960E94F24BCE0180960E94EC
:1030F000F24B6AE172E1CE0101960E944E4C4EE124
:1031000050E060E070E0CE0101960E946090CE0138
:1031100001960E94F24B2CAD3DAD4EAD5FAD2F5FE1
:103120003F4F4F4F5F4F2CAF3DAF4EAF5FAF42169B
:103130005306640675060CF06BCFB501A401CE01F1
:1031400080960E94816ABE01605E7F4FCE0101962B
:103150000E944E4C6BE476E0CE0101960E945B4BE0
:10316000BC018AE192E10E94DD4BCE0101960E94F2
:10317000F24BCE0180960E94F24B6AE172E1CE01E1
:1031800001960E944E4C4AE050E060E070E0CE01B3
:1031900001960E94BB8FCE0101960E94F24BB501B1
:1031A000A401CE0101960E94816A65E279E0CE0118
:1031B00080960E94564CBE016F5F7F4FCE01809675
:1031C0000E94724B6FE476E00E945B4B60E272E11A
:1031D0000E94724BBC0180E292E10E94DD4BCE0165
:1031E00080960E94F24BCE0101960E94F24B62E360
:1031F00070E080E090E00C942110E090B502F09037
:10320000B60281E080932C0564E670E080E090E0F7
:103210000E942B860E94DC3EC7010E94B3780E9468
:1032200094B120E034E0A901461B570BBA01CE014E
:1032300001960E947C5064E576E0CE0180960E9463
:10324000564CBE016F5F7F4FCE0180960E94724B3D
:10325000BC0180E292E10E94DD4BCE0180960E948B
:10326000F24BCE0101960E94F24B60E087E00E9493
:10327000566A66EE74E0CE0101960E94464C42E327
:1032800050E068E070E0CE0101960E94BB8FCE0155
:1032900001960E94F24B60E272E1CE0101960E941B
:1032A0004E4C42E350E06FEF7FEFCE0101960E945B
:1032B000738DCE0101960E94F24B6BE576E0CAC099
:1032C0008091B3029091B4020E94B3780E9494B1AD
:1032D0006B017C017093F10B6093F00B62E370E083
:1032E00080E090E00E942B86B601CE0101960E94FC
:1032F0007C50BE016F5F7F4F80E292E10E940F4BD6
:10330000CE0101960E94F24B809178129091791231
:10331000892B09F45EC064E772E1CE0180960E94B9
:103320004E4CBE01605E7F4FCE0101960E944E4C16
:1033300044E150E060E070E0CE0101960E94BB8F56
:10334000CE0101960E94F24B65E676E0CE01019631
:103350000E94564C60E272E1CE0101960E94724BCF
:10336000BC018AE192E10E94DD4BCE0101960E94F0
:10337000F24B6AE172E1CE0101960E944E4C44E1AB
:1033800050E06FEF7FEFCE0101960E94738DCE016A
:1033900001960E94F24BBE01605E7F4FCE01019606
:1033A0000E944E4C68ED7BE0CE0101960E945B4B83
:1033B0006AE172E10E94724BBC0180E292E10E94DC
:1033C000DD4BCE0101960E94F24BCE0180960C940B
:1033D000151060E776E08AE192E10E94C84B6AE14D
:1033E00072E1CE0101960E944E4C44E150E060E053
:1033F00070E0CE0101960E94BB8FCE0101960E9423
:10340000F24B64E576E0CE0101960E94564C60E2F4
:1034100072E1CE0101960E94724BBC018AE192E1F9
:103420000E94DD4BCE0101960E94F24B6AE172E1EF
:10343000CE0101960E944E4C44E150E06FEF7FEFC9
:10344000CE0101960E94738DCE0101960E94F24B2F
:1034500065E676E0CE0101960E94564C60E272E18C
:10346000CE0101960E94724BBC0180E292E10E9463
:10347000DD4BCE0101960E94F24B0C941710809107
:103480000402882309F4C6C28091450C811104C04E
:1034900080911511882329F082E090E00E94B742C4
:1034A000B9C2C0905502D0905602E0905702F090F9
:1034B000580220E030E040E450E4C701B6010E9429
:1034C000EAB118166CF420E030E04AEF54E4C7018A
:1034D000B6010E940AAF0E9494B16B017C0106C044
:1034E00040E3C42E45E7D42EE12CF12C0E94DC3EB3
:1034F00060E080E00E94566A67EF74E081E293E149
:103500000E94C24C61E080E00E94566A6FEE74E057
:1035100081E293E10E94C24C64E670E080E090E0BA
:103520000E942B860E9487876093EA0B7093EB0BB7
:103530008093EC0B9093ED0B0E9487878090EA0BB1
:103540009090EB0BA090EC0BB090ED0BDC01CB015D
:1035500088199909AA09BB098C159D05AE05BF05F7
:103560000CF058C283E090E00E94B7420E94878727
:1035700064E170E080E090E00E942B86DDCF0E9445
:10358000486289E39DE00E944A4844C267E175E0D1
:103590008AE192E10E94834B6AE172E1CE010196D9
:1035A0000E944E4C4AE050E060E070E0CE0101968F
:1035B0000E94BB8FCE0101960E94F24B5091610296
:1035C0005CAF8091000C811105C00E94878781E06B
:1035D0008093000C8091F80B811105C00E948787B1
:1035E00081E08093F80B1092F70B1092F60B20906D
:1035F000F60B3090F70B88E2281631040CF07CC0F3
:103600008CAD0E94E185F101EE0FFF1FE156F34FF3
:10361000918380830E94CC6B20E030E040EA50E44C
:103620000E940AAF20E030E040E85AE30E940AAF6F
:103630002B013C0180901D0290901E02A0901F0261
:10364000B0902002A50194016091190270911A02B4
:1036500080911B0290911C020E9434B09B01AC012E
:1036600060E070E080EC90E40E9434B06B017C017B
:1036700020E030E0A9010E94A5AE20E030E040E665
:1036800050E4811105C0C301B2010E940AAF1EC0FF
:10369000C301B2010E940AAFA50194010E9435B096
:1036A00020E030E040E850E40E9434B0A7019601E9
:1036B0000E94FBB020E030E040EC50E40E940AAFF2
:1036C00020E030E040E850E40E9435B06093F20B17
:1036D0007093F30B8093F40B9093F50B64E170E01F
:1036E00080E090E00E942B869FEF291A390A3092E1
:1036F000F70B2092F60B7BCFC090F20BD090F30B20
:10370000E090F40BF090F50B20E030E0A901C70148
:10371000B6010E94EAB187FD1EC022E0B701A601F2
:10372000CE0101960E94F74B64E776E0CE018096C9
:103730000E94564CBE016F5F7F4FCE0180960E9463
:10374000724BBC0180E292E10E94DD4BCE0180967B
:103750000E94F24B49C168E075E080E292E10E946C
:10376000834B46C180910402882309F453C18091A0
:10377000450C81112BC080911511811127C0C0907B
:103780005502D0905602E0905702F090580220E087
:1037900030E04AE754E4C701B6010E940AAF0E9434
:1037A00094B14B015C0120E030E040EA50E4C701F5
:1037B000B6010E940AAF20E030E040EA50E40E94E7
:1037C00035B00E9494B1A501940108C021E030E019
:1037D00040E050E06AE070E080E090E00E949D658B
:1037E00019C1C7010E94E99115C1C7010E945A5D24
:1037F00011C180919713882309F40CC165E675E027
:10380000CE0101960E94464CCE0101960E940A719B
:10381000FDC080919D0C90919E0C892BA1F481E0BC
:1038200090E090939E0C80939D0C8EED93E090938E
:103830003A0C8093390C0E94336E68EC70E080E0A3
:1038400090E00E942B8668E575E0CE0101960E940B
:10385000464C44E650E06FEF7FEFCE0101960E94A8
:10386000738DCE0101960E94F24BE0E0F0E01995D5
:10387000D1C00E941F870E94DC3E0E944A76CAC0C7
:1038800090911A1181E0892780931A11882369F198
:1038900061E575E080E292E10E94834B0E94878798
:1038A000609311117093121180931311909314115E
:1038B00080911D1190911E11181619065CF420912B
:1038C0001F11309120112817390724F01092201170
:1038D00010921F119091211180911C1198175CF08A
:1038E000109221111092221106C069E475E080E265
:1038F00092E10E94834B80911A118093151160E22E
:1039000072E1CE0101960E944E4C4AE050E068E020
:1039100070E0CE0101960E94BB8FCE0101960E94FD
:10392000F24B6CE375E0CE0101960E94464C4AE0F2
:1039300050E06FEF7FEFCE0101960E94738DCE01B4
:1039400001960E94F24B6EE275E080E292E10E94E5
:10395000B94A61E179E0CE0101960E94564C60E2DD
:1039600072E1CE0101960E94724BBC0180E292E1AD
:103970000E94DD4BCE0101960E94F24B8091450CD6
:10398000809323118CE291E00E94596E8091450C46
:10399000882309F43FC06FEE77E08CE292E10E9449
:1039A000C84B86EE9FEF90930A0C8093090C32C0AF
:1039B000F0920A0CE092090C89E39DE00E944A48CB
:1039C00060E275E080E292E10E94834B6FEB79E068
:1039D000CE0101960E94564C4AE050E060E070E053
:1039E000CE0101960E94BB8FCE0101960E94F24B40
:1039F00060E272E1CE0101960E944E4C4AE050E036
:103A00006FEF7FEFCE0101960E94738DCE0101967C
:103A10000E94F24B80912412909125120097A1F000
:103A2000419720F4023011050CF0A3C060E272E16E
:103A3000CE0101960E944E4CCE0101960E940A7161
:103A4000CE0101960E94F24B64E670E080E090E0C7
:103A50000E942B86A1C00E94003F0C94CB0EEC80EC
:103A6000F12CFE2CEE248D81E80EF11CCE80D12CA1
:103A7000DC2CCC248F81C80ED11CA884B12CBA2C8C
:103A8000AA248985A80EB11C21E02CAF0C94061243
:103A900066EC73E080E292E10E94834B60E272E1A7
:103AA000CE0180960E944E4C4AE050E060E070E00B
:103AB000CE0180960E94738DCE0180960E94F24BBB
:103AC00063EB73E080E292E10E94834B80910F0CE4
:103AD0009091100C029711F00C94DA121092100CC5
:103AE00010920F0C0C94DA1283E79EE00E94AC4710
:103AF000892B71F083E79EE00E948A47E1E0F0E0C5
:103B0000EC0FFD1FEE0DFF1D80832FEFE21AF20A6E
:103B100065E070E080E090E00E942B8636E0E316DE
:103B2000F10401F5998188A198131CC09A8189A19B
:103B3000981318C09B818AA1981314C08D8190E0BE
:103B4000A0E0B0E0BA2FA92F982F88272C81820FF0
:103B5000911DA11DB11D480E591E6A1E7B1E4FEFFF
:103B6000241A340A5FEF851A950AA50AB50A0C943F
:103B70006F1560E272E1CE0101960E944E4C4AE060
:103B800050E06FEF7FEFCE0101960E94738DCE0162
:103B900001960E94F24B4ACFCB5BDF4F0FB6F894F1
:103BA000DEBF0FBECDBFDF91CF911F910F91FF9070
:103BB000EF90DF90CF90BF90AF909F908F907F90CD
:103BC0006F905F904F903F902F9008952F923F926B
:103BD0004F925F926F927F928F929F92AF92BF921D
:103BE000CF92DF92EF92FF920F931F93CF93DF93C9
:103BF000CDB7DEB728970FB6F894DEBF0FBECDBFA6
:103C0000FC018FEB9FE0938782878091BC0F90E04F
:103C1000958784878091891090E097878687809127
:103C2000B90F853009F063C68091C10F9091C20F22
:103C3000885891098D35910588F48091BC0F8430A6
:103C400041F48091C30F9091C40F8097479708F477
:103C50007DC08091BC0F843408F05EC08091BC0FA1
:103C60008A3108F4D5C08091BF0F9091C00F843F76
:103C7000914050F4118610868FEF9FEFDC01848312
:103C80009583A683B7833CC08091C10F9091C20FEA
:103C900085974B9708F0BCC005ECE02E0FE0F02EA6
:103CA00082E090E040E050E0BA018C010F5F1F4FCE
:103CB0002091BC0F30E0021713076CF497012250DB
:103CC0003109D9012D913C91275031092730310517
:103CD00008F47FC0C80101979595879591878087E3
:103CE0000C971CF41186108693C044835583668319
:103CF000778384E090E00DC04483558366837783A7
:103D00008BE090E006C044835583668377838CE024
:103D100090E0918380831EC58091C30F9091C40F62
:103D2000825491098E9708F099CF20E030E0C12CA1
:103D3000D12C7601A9014B53504FDA014D915C9182
:103D4000495051094930510598F088CF8091C50FED
:103D50009091C60F0997099708F07BCF11861086BE
:103D60008FEF9FEFDC0184839583A683B783C2C561
:103D7000B9016953704FDB014D915C914751510975
:103D800042315105C0F4D701C601880F991FAA1FFF
:103D9000BB1F6C017D016894C0F82C5F3F4F203839
:103DA000310541F620E230E031872087C482D58298
:103DB000E682F7829FC5DB014D915C914650510927
:103DC0004730510508F04ACFCC0CDD1CEE1CFF1C1F
:103DD000E4CFD7012D913C91235131092F3031058A
:103DE00050F4440F551F661F771F41600296B4E0E0
:103DF000EB0EF11C5ACFD7012D913C912A5031097D
:103E00002930310528F4440F551F661F771FEECF68
:103E10008091BC0F8A3108F460C08091BF0F9091EF
:103E2000C00F8032934008F425CF8091C10F90914C
:103E3000C20FC697869708F050C08091C30F90912B
:103E4000C40FC697869708F048C0B7ECEB2EBFE0CA
:103E5000FB2E83E090E040E050E0BA018C010F5F60
:103E60001F4F2091BC0F30E00217130764F4970135
:103E700022503109D9012D913C912C5031092B3020
:103E8000310560F0C80101979595879591878087E6
:103E90000C970CF031CF118610861FC0D7012D91E1
:103EA0003C91255231092B31310550F4440F551FF7
:103EB000661F771F41600296B4E0EB0EF11CCECF77
:103EC000D7012D913C912C5031092A30310528F42D
:103ED000440F551F661F771FEECF8091BC0F8232B3
:103EE00008F452C08091C10F9091C20F06970797B6
:103EF00008F04AC045ECC42E4FE0D42E82E090E09A
:103F000040E050E0BA018C010F5F1F4F2091BC0FC1
:103F100030E002171307F4F4D6011297ED90FC90ED
:103F200011979D01BEE1EB1AF108A7E1EA16F10431
:103F3000E0F4440F551F661F771F4160D6012D9195
:103F40003C91B4E0CB0ED11C235031092530310512
:103F5000C8F0C8010197959587959187808740970C
:103F60000CF0D1CE118610860FC0D9012D913C9155
:103F70002C5031092B30310538F4440F551F661F82
:103F8000771FDCCF0296BFCF7F011C821B8281E0AE
:103F900090E09A8389838091BC0F8D3070F41C82ED
:103FA0001B8281E090E09A838983F701848595855F
:103FB000181619060CF474C0D1C029E733E0AE011D
:103FC0004D5F5F4FBE016F5F7F4FC7010E944599F4
:103FD000892B29F729E733E0AE014D5F5F4FBE0122
:103FE0006F5F7F4FC7010E9445990197C1F629E78E
:103FF00033E0AE014D5F5F4FBE016F5F7F4FC70182
:104000000E944599892B59F6812C912C540100E08E
:1040100010E08091BC0F90E029813A812817390780
:1040200094F529E733E0AE014D5F5F4FBE016F5F4E
:104030007F4FC7010E9445996C0129E733E0AE012B
:104040004D5F5F4FBE016F5F7F4FC7010E94459973
:10405000F1E0CF16D10451F4892B09F0A0CF880CE0
:10406000991CAA1CBB1C689480F80AC0CD2809F0D2
:1040700096CF019709F093CF880C991CAA1CBB1C02
:104080000F5F1F4FC6CFD70119961C930E93189739
:10409000F70184829582A682B78281E090E039CED2
:1040A0000284F385E02D82E090E09A838983828107
:1040B000938189974E9708F051C083E090E09A83EE
:1040C0008983848195810B970A9708F047C02CEB70
:1040D00031E0AE014D5F5F4FBE016F5F7F4FC701A3
:1040E0000E944599892BD1F52CEB31E0AE014D5F53
:1040F0005F4FBE016F5F7F4FC7010E9445990197D7
:1041000069F5412C512C320100E010E0F7012485C3
:10411000358589819A81821793070CF02FC12CEB8A
:1041200031E0AE014D5F5F4FBE016F5F7F4FC70152
:104130000E9445995C010330110509F0E5C02CEBA4
:1041400031E0AE014D5F5F4FBE016F5F7F4FC70132
:104150000E944599A816B90609F4D6C0D7011A9647
:10416000ED91FC911B9782819381C6978697E0F42D
:10417000848195814B974597B8F4DF0116966F01BE
:1041800026ECC20ED11C20E030E040E050E060E0C0
:1041900070E080E090E00D911C9111970950110999
:1041A0000830110508F4F4C08091BC0F893370F118
:1041B00082819381895791098335910508F41BC148
:1041C00025C0D90112966D917C91139766517109A2
:1041D0006131710508F037C1D501C401880F991FFD
:1041E000AA1FBB1F4C015D01689480F84E5F5F4FB2
:1041F0002C5F3F4F4B33510509F40CC1D9016D9130
:104200007C916A50710969307105D8F28091BC0FB8
:10421000823231F4828193810A97099708F423C18D
:10422000828193818957910983359105D0F48091DA
:10423000BC0F8132B0F084819581CA97899788F448
:104240009F012A5F3F4F812C912C540143E050E0A5
:10425000D9016D917C916A5071096930710508F43A
:104260001EC1828193818C549109C59778F4809105
:10427000BC0F843031F4848195818097479708F48E
:104280006CC18091BC0F843408F04EC18091BC0F8A
:10429000863460F1828193810C970B9708F4A9C151
:1042A00025C0D90112966D917C9113976E517109B9
:1042B0006731710508F0D1C1D501C401880F991F7C
:1042C000AA1FBB1F4C015D01689480F84E5F5F4FD1
:1042D0002C5F3F4F4534510509F4A6C1D9016D91BA
:1042E0007C916C5071096B307105D8F28091BC0FD4
:1042F000883508F4E4C182819381855891098B3512
:10430000910508F4BAC1DBC12CEB31E0AE014D5F81
:104310005F4FBE016F5F7F4FC7010E9445996C01DF
:104320000330110579F42CEB31E0AE014D5F5F4FA6
:10433000BE016F5F7F4FC7010E944599C816D9061D
:1043400009F00CCFA114B10459F4CA94CD2809F096
:1043500005CF440C551C661C771C689440F80BC0B4
:10436000AA94AB2809F0FACECD2809F0F7CE440C78
:10437000551C661C771C0F5F1F4FC8CE1187008726
:10438000F701448255826682778282E090E0C1CC58
:1043900012960D911C911397015111090D301105C1
:1043A000E0F401E00E9477B321601496AC15BD05DE
:1043B00009F0F1CEF701248335834683578300E269
:1043C0000E9492B32283338385E090E091838083BF
:1043D00080E390E091878087BDC112960D911C917A
:1043E0001397045011090530110508F0DDCE01E0E6
:1043F0000E9477B3DACF84819581CA97899708F0B4
:1044000005CF9F012A5F3F4F812C912C540143E03F
:1044100050E0F4CE9F012A583F4FD9012D913C9195
:104420002A5031092930310508F0F0CE2CE130E076
:10443000F70131872087D70184829582A682B782CF
:104440008AE090E085C1D90112966D917C91139715
:10445000665071096730710508F0D8CE880C991C38
:10446000AA1CBB1CC3CE2091BC0FCF01820F911D93
:10447000820F911DDC0112978D919C910A970997EB
:1044800008F0CECEF701118610868FEF9FEFDC018A
:1044900084839583A683B78386E090E03ACCD901E4
:1044A00012966D917C911397665171096131710576
:1044B00058F5D501C401880F991FAA1FBB1F4C01D5
:1044C0005D01689480F84E5F5F4F2C5F3F4F433231
:1044D000510509F0BDCE9F012A5B3F4FD9012D91B7
:1044E0003C912A5031092930310508F0BACE20E13B
:1044F00030E0F70131872087D70184829582A68238
:10450000B78286E090E024C1D90112966D917C912A
:104510001397665071096730710508F0A2CE880CB8
:10452000991CAA1CBB1CCFCF848195818954910909
:10453000C39708F0ABCE9F012A5F3F4FAF014A57A8
:104540005F4F812C912C5401D9016D917C91695060
:10455000710969307105B8F099CE86819781099704
:10456000099708F08ECED70119961C921E921897C3
:104570008FEF9FEFDC01F70184839583A683B783D8
:1045800087E090E0C6CBD90112966D917C9113978C
:104590006651710961317105E0F4D501C401880FDC
:1045A000991FAA1FBB1F4C015D01689480F82C5F06
:1045B0003F4F2417350741F620E230E0F7013187FD
:1045C0002087D70184829582A682B78287E090E017
:1045D000BFC0D90112966D917C91139766507109F5
:1045E0006730710508F052CE880C991CAA1CBB1CC0
:1045F000DECF848195810997099708F077CE86816F
:1046000097818C974F9708F071CE80859185899717
:104610004D9708F06BCE9F01265F3F4F812C912C68
:10462000540145E050E05ACE9F0126573F4FD90133
:104630002D913C912C5031092B30310508F056CE8C
:1046400020E230E0F70131872087D701848295820C
:10465000A682B78288E090E07BC0D90112966D9166
:104660007C911397695071096930710508F03ECE4D
:10467000880C991CAA1CBB1C29CE8481958182546C
:1046800091098E97E0F48F01045C1F4F8DE190E05B
:1046900040E050E02091BC0F30E0245031098217F7
:1046A00093070CF063C0980122503109D9012D9174
:1046B0003C91295031092830310508F46EC08091B1
:1046C000BC0F803209F07EC08281938106970697E5
:1046D00008F078C0848195810997099708F072C025
:1046E0009F012A5F3F4FAF01425C5F4F812C912CAD
:1046F0005401D9016D917C91665071096630710544
:1047000008F060C0D90112966D917C9113976951A0
:1047100071096331710508F0D5C0D501C401880F56
:10472000991FAA1FBB1F4C015D01689480F82C5F84
:104730003F4F24173507E9F62EE030E0F7013187C7
:104740002087D70184829582A682B7828FE090E08D
:104750008D939C9381E090E0D0C0D8012D913C9145
:10476000285131092231310550F1CB01019795953E
:104770008795D70119969C938E9318978A970CF476
:104780009ECF052E000C660B770BF70144835583F3
:104790006683778389E090E0BCCABC016F5F7F4F7E
:1047A000D8012D913C912750310927303105A8F6C9
:1047B000440F551F416002960C5F1F4F6BCF440F93
:1047C000551FF9CFD7011C962D903C901D97B6E050
:1047D0002B1631040CF486C08F010E5F1F4F75EC51
:1047E000872E7DE9972E7CE1A72E71E8B72EE3E0B6
:1047F000CE2ED12CF801648175816080718080E0BB
:1048000090E00E94A9AE6D837E838F839887B30169
:1048100080E090E00E94A9AE2B013C012DEC3CEC25
:104820004CE45FE30E940AAF9B01AC016D817E8185
:104830008F8198850E94A5AE87FD19C02DEC3CECB8
:104840004CE45FE36D817E818F8198850E940AAF81
:104850009B01AC01C301B2010E94A5AEE82F880FF5
:10486000FF0BEE27FF0FEE1FFF27319602C0E0E09F
:10487000F0E0A501940163E971E080E091E00E941D
:104880004DB34F01FF0FAA08BB0886269726A8261E
:10489000B926FFEFCF1ADF0A0E5F1F4F2C143D041D
:1048A00009F0A8CFD70114968D929D92AD92BC923B
:1048B000179780E290E019969C938E9318978FEF4C
:1048C0009FEF46CFD90112966D917C911397695055
:1048D00071096930710508F075CF880C991CAA1C04
:1048E000BB1C25CF82E08093B90F1092BC0F80E0F3
:1048F00090E003C083E090E00CCA28960FB6F894CD
:10490000DEBF0FBECDBFDF91CF911F910F91FF9002
:10491000EF90DF90CF90BF90AF909F908F907F905F
:104920006F905F904F903F902F9008955F926F929D
:104930007F928F929F92AF92BF92CF92DF92EF922F
:10494000FF920F931F93CF93DF93CDB7DEB7E4971A
:104950000FB6F894DEBF0FBECDBF6EE372E188E301
:1049600092E10E94DD4B0E94218563E277E0CE0157
:1049700001960E94564CBE016F5F7F4F88E392E123
:104980000E940685182FCE0101960E94F24B11233A
:1049900009F476C026E030E045E050E06EE372E1D5
:1049A000CE0101960E946A4CBE016F5F7F4F8AE183
:1049B00092E10E940F4BCE0101960E94F24B8AE1D8
:1049C00092E10E943D4A6B017C0164ED7AE0CE01E8
:1049D00001960E94564CBE016F5F7F4F8EE392E1BD
:1049E0000E94B684AC014F5F5F4F6EE372E1CE016F
:1049F0000B960E94273FBE01655F7F4F8AE192E1DF
:104A00000E940F4BCE010B960E94F24BCE010196F5
:104A10000E94F24B8AE192E10E943D4A9B01E7E04D
:104A2000F2E041E050E0A0910702B0910802A41723
:104A3000B5075CF0A281B3812A173B0711F41382FA
:104A400012824F5F5F4F3296EECF9601220F331FD7
:104A5000F901E95FFD4F7183608382E090E00E947D
:104A6000A4776EE372E1CE0101960E944E4CCE0116
:104A700001960E948F8FCE0101960E94F24B31C0A9
:104A800069E277E0CE0101960E94564CBE016F5F4D
:104A90007F4F88E392E10E940685182FCE01019690
:104AA0000E94F24B112349F1E7E0F2E081E090E04F
:104AB00020910702309108022817390774F08630D8
:104AC00091051CF49383828305C09C012E5F3F4FA8
:104AD0003383228301963296EBCF82E090E00E94EE
:104AE000A47710923A0C1092390C80E090E00E946A
:104AF000836E109254020C944E2F6FE277E0CE0139
:104B000001960E94564CBE016F5F7F4F88E392E191
:104B10000E940685182FCE0101960E94F24B1123A8
:104B2000F9F080919D0C90919E0C892BA1F481E06D
:104B300090E090939E0C80939D0C8EED93E090936B
:104B40003A0C8093390C0E94336E68EC70E080E080
:104B500090E00E942B86E0E0F0E019950C944E2F37
:104B600066E377E0CE0101960E94564CBE016F5F6E
:104B70007F4F88E392E10E940685182FCE010196AF
:104B80000E94F24B1123B1F06EE377E0CE01019663
:104B90000E94564C6FE073E1CE0101960E94724B69
:104BA000BC0180E292E10E94DD4BCE0101960E94A1
:104BB000F24B20C068E477E0CE0101960E94564C8B
:104BC000BE016F5F7F4F88E392E10E940685182F38
:104BD000CE0101960E94F24B112351F16CE577E072
:104BE00080E292E10E94834B65E173E180E292E111
:104BF0000E94094B61E179E0CE0101960E94564C7A
:104C000060E272E1CE0101960E94724BBC01CE01BE
:104C10000B960E944E4CCE010B960E940A71CE015B
:104C20000B960E94F24BCE0101960E94F24B61CF8F
:104C30006FE477E0CE0101960E94564CBE016F5F93
:104C40007F4F88E392E10E940685182FCE010196DE
:104C50000E94F24B112311F169E377E080E292E1C7
:104C60000E94834B60E272E1CE0101960E944E4C9D
:104C7000CE0101960E940A71CE0101960E94F24B6C
:104C80000E94E3591092540265E577E08EE392E1C9
:104C90000E94C84B0E94837E0C944E2F69E577E0FA
:104CA000CE0101960E94564CBE016F5F7F4F88E394
:104CB00092E10E940685182FCE0101960E94F24BC8
:104CC000112309F48CC064ED7AE0CE0101960E94B4
:104CD000564CBE016F5F7F4F8EE392E10E94B68417
:104CE000AC014F5F5F4F6EE372E1CE010B960E9405
:104CF000273FBE01655F7F4F8AE192E10E940F4B23
:104D0000CE010B960E94F24BCE0101960E94F24B0F
:104D10008AE192E10E943D4A8B016CE277E080E2F9
:104D200092E10E94834B80911A11882331F060E256
:104D300077E080E292E10E94834B0115110511F4A6
:104D40000C943A2FCE0101960E94365ACE0101965C
:104D50000E940A71CE0101960E94F24B02301105A9
:104D60000CF4C7CE67E775E0CE010B960E94464C67
:104D7000BE01655F7F4FCE0101960E944E4CCE0171
:104D800001960E940A71CE0101960E94F24BE12C1D
:104D9000F12C80911C11082E000C990BE816F906D5
:104DA0008CF4B701CE0101960E943F5CCE010196C2
:104DB0000E940A71CE0101960E94F24BFFEFEF1A9A
:104DC000FF0AE7CFCE010B960E94F24B023011058D
:104DD00009F48FCE8CE291E00E94AD6E8ACE60E63F
:104DE00077E0CE0101960E94564CBE016F5F7F4F67
:104DF00088E392E10E940685182FCE0101960E9459
:104E0000F24B112309F488C36EE372E1CE018F9651
:104E10000E944E4C64ED7AE0CE0101960E94564C01
:104E2000BE016F5F7F4FCE018F960E94B684AC01AA
:104E30004F5F5F4FBE01615D7F4FCE0189960E943B
:104E4000273FCE0101960E94F24BBE01615D7F4F6C
:104E5000CE0101960E944E4CCE0101960E948F8F8A
:104E6000CE0101960E94F24B64E677E0CE010196F6
:104E70000E94564CBE016F5F7F4FCE0189960E9403
:104E80007A848C01CE0101960E94F24B6FEB79E09F
:104E9000CE0183960E94564C6FEB79E0CE014D9681
:104EA0000E94564C1016110684F5A8014F5F5F4F03
:104EB0008DA59EA54817590790F4BE01675D7F4FE9
:104EC000CE0101960E94273FBE016F5F7F4FCE014A
:104ED00083960E940F4BCE0101960E94F24B9801DF
:104EE00040E050E0BE01675D7F4FCE0101960E9419
:104EF0006A4CBE016F5F7F4FCE014D960E940F4BF3
:104F0000CE0101960E94F24B0DC06FEB79E0CE010D
:104F100083960E94C84BBE01675D7F4FCE014D96C0
:104F20000E94DD4B89A19AA1892B09F4E6C2CE012A
:104F30004D960E943D4A8B0101501109083111051F
:104F400014F007E110E017FF02C00FEF1FEFB801E8
:104F5000CE010B960E947C5066E677E0CE0101966A
:104F60000E94564CBE01655F7F4FCE0101960E94A4
:104F7000724BBC01CE0141960E944E4CCE0141962F
:104F80000E948F8FCE0141960E94F24BCE01019676
:104F90000E94F24BCE010B960E94F24BBE016D5D5A
:104FA0007F4FCE0189960E94DD4B64E677E0CE010B
:104FB00001960E94564CBE016F5F7F4FCE018996CD
:104FC0000E947A847C01CE0101960E94F24B6FEB25
:104FD00079E0CE0183960E94C84B6FEB79E0CE0159
:104FE0004D960E94C84B1E141F040CF04EC0A70122
:104FF0004F5F5F4F8DA59EA54817590790F4BE01DE
:10500000675D7F4FCE0101960E94273FBE016F5F13
:105010007F4FCE0183960E940F4BCE0101960E94D6
:10502000F24B970140E050E0BE01675D7F4FCE013B
:1050300001960E946A4CBE016F5F7F4FCE014D9674
:105040000E940F4BCE0101960E94F24BAE014F5FC2
:105050005F4F5A01E12CF12CA8014F5F5F4F8AE0AE
:10506000849F9001859F300D1124F901E65EFE4E6C
:105070006F01809F9001819F300D1124A901485D2F
:105080005E4E3A018AE2582EC1C06FEB79E0CE0144
:1050900083960E94C84BBE01675D7F4FCE014D963F
:1050A0000E94DD4BD3CFE114F10409F0BCC00F3FE7
:1050B0008FEF180709F4B7C0CE014D960E94484AF9
:1050C000C114D10439F044E050E0B601CE014D9650
:1050D0000E949484B601CE0141960E94564C6BE624
:1050E00077E0CE010B960E94564CBE016F5E7F4F5B
:1050F000CE010B960E94724BBC01CE0147960E94D6
:105100004E4CCE0147960E948F8FCE0147960E944B
:10511000F24BCE010B960E94F24BCE0141960E94BB
:10512000F24B89A19AA1029708F476C061E070E081
:10513000CE014D960E94A84A082E000C990B803390
:1051400091050CF44C96E52DE81B8E2FF30180831E
:10515000FFEFEF1AFF0ABE016D5D7F4FCE0189960A
:105160000E94DD4B64E677E0CE010B960E94564C20
:10517000BE01655F7F4FCE0189960E947A844C0103
:10518000CE010B960E94F24B6FEB79E0CE01839635
:105190000E94C84B6FEB79E0CE014D960E94C84B40
:1051A000181419040CF047C0A4014F5F5F4F8DA580
:1051B0009EA54817590790F4BE01675D7F4FCE0149
:1051C0000B960E94273FBE01655F7F4FCE018396FD
:1051D0000E940F4BCE010B960E94F24B940140E0CF
:1051E00050E0BE01675D7F4FCE010B960E946A4C76
:1051F000BE01655F7F4FCE014D960E940F4BCE01E1
:105200000B960E94F24B52E0A50EB11C89A19AA107
:10521000892B09F048CF1DC0CE014D960E943D4A12
:10522000F301608395CFCE014D960E943D4AF50172
:10523000718360838DCF6FEB79E0CE0183960E94FE
:10524000C84BBE01675D7F4FCE014D960E94DD4B7E
:10525000DACF0F3F2FEF120709F07DC064E677E049
:10526000CE010B960E94564CBE01655F7F4FCE016A
:1052700083960E947A848C01CE010B960E94F24B99
:1052800017FF3BC109811A811016110634F4093148
:1052900011052CF008E110E002C001E010E00093DD
:1052A0001C11B801CE0141960E947C5069E777E05D
:1052B000CE010B960E94564CBE016F5E7F4FCE0111
:1052C0000B960E94724BBC01CE0147960E944E4C39
:1052D000CE0147960E948F8FCE0147960E94F24BD7
:1052E000CE010B960E94F24BCE0141960E94F24BEA
:1052F000E114F10459F18B819C8197FF02C080E099
:1053000090E090931E1180931D1141E0E416F1048A
:10531000E9F08D819E81181619062CF480179107EB
:1053200024F48C0102C001E010E00150009321112F
:1053300052E0E516F10451F08F8198851816190690
:1053400014F081E090E08150809322118CE291E092
:105350000E94596ED2C080911B11082E000C990B2F
:10536000081719070CF083C0B701CE0141960E94BF
:105370007C5063E877E0CE010B960E94564CBE014C
:105380006F5E7F4FCE010B960E94724BBC01CE0127
:1053900047960E944E4CCE0147960E948F8FCE01B9
:1053A00047960E94F24BCE010B960E94F24BCE0123
:1053B00041960E94F24B8AE0809FF001819FF00DA0
:1053C0001124E65EFE4E81E0878783E090E0918BBA
:1053D000808B938B828BE114F10409F48EC08B8156
:1053E0009C818038910514F08FE790E080382FEF92
:1053F000920714F480E89FEF878741E0E416F104F8
:1054000009F47BC08AE0809FF001819FF00D112498
:10541000E65EFE4E8D819E8197FF02C080E090E0A7
:10542000918B808B52E0E516F10409F466C08AE0A6
:10543000809FF001819FF00D1124E65EFE4E8F816A
:10544000988597FF02C080E090E0938B828B8091DB
:105450001C11082E000C990B081719071CF00F5F80
:1054600000931C118CE291E00E94AD6E46C0BE011B
:105470006D5D7F4FCE0147960E944E4C60911B118F
:10548000062E000C770BCE0141960E947C506BE8F3
:1054900077E0CE010B960E94564CBE01695E7F4FAD
:1054A000CE010B960E94724B6CE977E00E945B4B39
:1054B000BE016F5E7F4F0E94724BBC01CE014796CA
:1054C0000E94DD4BCE010B960E94F24BCE0141961D
:1054D0000E94F24BBE01695E7F4FCE010B960E9487
:1054E0004E4CCE010B960E940A71CE010B960E9483
:1054F000F24BCE0147960E94F24BCE014D960E9490
:10550000F24BCE0183960E94F24BCE0189960E9407
:10551000F24BCE018F9650C260EA77E0CE01019641
:105520000E94564CBE016F5F7F4F88E392E10E945C
:105530000685182FCE0101960E94F24B1123C9F166
:1055400064ED7AE0CE0101960E94564CBE016F5F79
:105550007F4F8EE392E10E94B684AC014F5F5F4FB4
:105560006EE372E1CE010B960E94273FBE01655F9C
:105570007F4F8AE192E10E940F4BCE010B960E9471
:10558000F24BCE0101960E94F24B8AE192E10E9419
:105590003D4A6115710521F481E080932E0506C016
:1055A0006130710509F0A5CA10922E050E945A7645
:1055B000A0CA65EA77E0CE0101960E94564CBE0172
:1055C0006F5F7F4F88E392E10E940685182FCE011E
:1055D00001960E94F24B112309F452C143E050E0BE
:1055E0006EE372E1CE0101960E94273FBE016F5F1C
:1055F0007F4F8AE192E10E940F4BCE0101960E94FB
:10560000F24B6AE172E1CE0101960E944E4CCE014E
:1056100001960E948F8FCE0101960E94F24B10924C
:105620003A0C1092390C6AE172E1CE0101960E94A7
:105630004E4C60E0CE0101960E94E84A811104C000
:10564000CE0101960E94494BBE016F5F7F4F8BE1F7
:1056500093E10E94DD4BCE0101960E94F24B6AE17C
:1056600072E1CE0101960E944E4C60E0CE0101969F
:105670000E94E84A811104C0CE0101960E94494B64
:10568000BE016F5F7F4F85E193E10E94DD4BCE014C
:1056900001960E94F24B40911F1350912013411527
:1056A000510549F087EA90E1009729F0BC018BE1B0
:1056B00093E10E9494844091191350911A1341155B
:1056C000510549F085E091E1009729F0BC0185E1A1
:1056D00093E10E9494848091390C90913A0C0E943D
:1056E000836E6AEF76E0CE0101960E94564C6AE125
:1056F00072E1CE0101960E94724BBC01CE0141962F
:105700000E944E4CCE0101960E94F24B80910111F5
:1057100090910211892B39F4BE016F5E7F4F89E3AE
:105720009DE00E94B44C68EB7BE080E090E00E943A
:105730002B868091011190910211029709F087C088
:105740006AE172E1CE0147960E944E4C69EA77E029
:10575000CE0101960E94564CCE0101960E9492A95C
:10576000CE0101960E94F24B64EF71E080E090E080
:105770000E942B866CEA77E0CE0101960E94564C7F
:10578000CE0101960E9492A9CE0101960E94F24B91
:105790006CED75E080E090E00E942B8665EB77E091
:1057A000CE0101960E94564CCE0101960E9492A90C
:1057B000CE0101960E94F24B64EF71E080E090E030
:1057C0000E942B8663EC77E0CE0101960E94564C36
:1057D000CE0101960E9492A9CE0101960E94F24B41
:1057E00064EF71E080E090E00E942B866AEF76E043
:1057F000CE0101960E94564CBE01695E7F4FCE01DC
:1058000001960E94724BBC01CE010B960E944E4C39
:10581000CE0101960E94F24BCE010B960E94484A9F
:10582000BE01655F7F4FCE0101960E944E4CCE01B6
:1058300001960E9492A9CE0101960E94F24BCE01E0
:105840000B960E94F24BCE0147960E94F24B68EBFA
:105850007BE080E090E00E942B8667EA70E1CE0159
:1058600001960E94564CCE0101960E948F8FCE0168
:1058700001960E94F24B10925402CE0141969CC0B8
:1058800061ED77E0CE0101960E94564CBE016F5F3C
:105890007F4F88E392E10E940685182FCE01019682
:1058A0000E94F24B112309F48AC044E050E06EE3F9
:1058B00072E1CE0101960E94273FBE016F5F7F4FCC
:1058C0008AE192E10E940F4BCE0101960E94F24BB9
:1058D00062E077E0CE0101960E94564C6AE172E1E7
:1058E000CE0101960E94724BBC01CE010B960E9424
:1058F0004E4CCE0101960E94F24B80910111909185
:105900000211892B69F4BE01655F7F4F89E39DE039
:105910000E94B44C68E873E180E090E00E942B861E
:105920008091011190910211029709F041C066ED3A
:1059300077E0CE0101960E94564C80911E12909104
:105940001F12892B39F46FED77E0CE0101960E948A
:10595000C84B15C0BE016F5F7F4FCE0141960E94BC
:105960004E4CCE0141960E9492A9CE0141960E94D2
:10597000F24B60ED77E080E090E00E942B86BE0164
:10598000655F7F4FCE0141960E944E4CCE014196FD
:105990000E9492A9CE0141960E94F24B60ED77E001
:1059A00080E090E00E942B86CE0101960E94F24B8F
:1059B00010925402CE010B960E94F24B6FC268EE19
:1059C00077E0CE0101960E94564CBE016F5F7F4F7B
:1059D00088E392E10E940685182FCE0101960E946D
:1059E000F24B112309F462C06EE372E18AE192E1A5
:1059F0000E94DD4B81E0809354026EE372E1CE01A0
:105A000001960E944E4CCE0101960E948F8FCE01CE
:105A100001960E94F24B8091011190910211029720
:105A200009F16AE172E189E39DE00E94B44C68EB00
:105A30007BE080E090E00E942B86CE0101960E94E0
:105A4000BA75BE016F5F7F4F8EE392E10E940F4BEC
:105A5000CE0101960E94F24B60ED77E080E090E08D
:105A60000E942B868091011190910211029771F48E
:105A70006AE172E1CE0101960E944E4CCE01019680
:105A80000E9492A9CE0101960E94F24B809142128F
:105A900090914312892B09F42CC861E179E0CE0181
:105AA00001960E94564C6EE372E1ACC86CEE77E052
:105AB000CE0101960E94564CBE016F5F7F4F88E376
:105AC00092E10E940685182FCE0101960E94F24BAA
:105AD000112309F45CC0809101119091021101978A
:105AE00009F007C8CE0101960E94C9608D819E8190
:105AF000009709F4C9C1E981FA812081222309F4C0
:105B0000C3C1079708F4C0C167E177E0CE010B96E7
:105B10000E94464C48EC50E06FEF7FEFCE010B96B1
:105B20000E946090CE010B960E94F24BBE016F5F07
:105B30007F4FCE010B960E944E4C40ED57E06FEF29
:105B40007FEFCE010B960E94738DCE010B960E94C3
:105B5000F24B62EF77E0CE010B960E94564C6EE35B
:105B600072E1CE010B960E94724BBC01CE014196B0
:105B70000E944E4CCE0141960E940A71CE01419680
:105B80000E94F24BCE010B960E94F24B7DC160E069
:105B900078E0CE0101960E94564CBE016F5F7F4FA8
:105BA00088E392E10E940685182FCE0101960E949B
:105BB000F24B112361F125E030E044E050E06EE368
:105BC00072E1CE0101960E946A4CBE016F5F7F4F69
:105BD0008AE192E10E940F4BCE0101960E94F24BA6
:105BE0006EE372E1CE0101960E944E4CCE01019609
:105BF0000E948F8FCE0101960E94F24B8AE192E1C2
:105C00000E943D4ACB010E9419910C94792565E0D0
:105C100078E0CE0101960E94564CBE016F5F7F4F27
:105C200088E392E10E940685182FCE0101960E941A
:105C3000F24B112361F127E030E046E050E06EE3E3
:105C400072E1CE0101960E946A4CBE016F5F7F4FE8
:105C50008AE192E10E940F4BCE0101960E94F24B25
:105C60008AE192E10E943D4A672B19F41092971342
:105C700003C081E0809397136EE372E1CE01019639
:105C80000E944E4CCE0101960E948F8FFDC06CE0A9
:105C900078E0CE0101960E94564CBE016F5F7F4FA7
:105CA00088E392E10E940685182FCE0101960E949A
:105CB000F24B112309F476C0809142129091431265
:105CC000079708F4EBC046E050E06EE372E1CE01C6
:105CD00001960E94273FBE016F5F7F4F8AE192E1EC
:105CE0000E940F4BCE0101960E94F24B8AE192E195
:105CF0000E94324A60935002709351028093520284
:105D00009093530267E077E080E292E10E94834B38
:105D10004091500250915102609152027091530291
:105D200021E0CE0101960E94F74BBE016F5F7F4FCD
:105D3000CE010B960E944E4C6BED75E0CE010B969A
:105D40000E945B4BBC0180E292E10E94094BCE01B4
:105D50000B960E94F24BCE0101960E94F24B60E23C
:105D600072E1CE0101960E944E4CCE0101960E9436
:105D70000A71CE0101960E94F24B0E94878728EE9D
:105D800033E040E050E00E9403B0CA01B9010E9434
:105D9000A9AE6093410C7093420C8093430C909396
:105DA000440C7CC063E178E0CE0101960E94564C21
:105DB000BE016F5F7F4F88E392E10E940685182F36
:105DC000CE0101960E94F24B112309F463C0809129
:105DD000421290914312079708F460C046E050E0E9
:105DE0006EE372E1CE0101960E94273FBE016F5F14
:105DF0007F4F8AE192E10E940F4BCE0101960E94F3
:105E0000F24B8AE192E10E94324A6093550270930C
:105E10005602809357029093580267EF76E080E233
:105E200092E10E94834B409155025091560260913D
:105E300057027091580221E0CE0101960E94F74B63
:105E4000BE016F5F7F4FCE010B960E944E4C6BEDF3
:105E500075E0CE010B960E945B4BBC0180E292E1A3
:105E60000E94094BCE010B960E94F24BCE01019687
:105E70000E94F24B60E272E1CE0101960E944E4C0C
:105E8000CE0101960E940A71CE0101960E94F24B4A
:105E90000C947925E9D5182F8823A1F0109154028C
:105EA000112379F06EE372E1CE0101960E944E4C0F
:105EB000CE0101960E948F8FCE0101960E94F24B77
:105EC00001C011E0812FE4960FB6F894DEBF0FBE3B
:105ED000CDBFDF91CF911F910F91FF90EF90DF9099
:105EE000CF90BF90AF909F908F907F906F905F907A
:105EF00008954F925F926F927F929F92AF92BF925E
:105F0000CF92DF92EF92FF920F931F93CF93DF9385
:105F1000CDB7DEB7A9970FB6F894DEBF0FBECDBFE1
:105F2000982E882351F080919713882331F06FEBDE
:105F300079E080E19FE00E94AE6A0E944A5060E0F2
:105F40008DE20E94A55160E18DE20E94A55168E0BA
:105F50008DE20E94A55140908A1250908B12609061
:105F60008C1270908D12498E5A8E6B8E7C8EC090E2
:105F70008E12D0908F12E0909012F0909112CD8EF0
:105F8000DE8EEF8EF8A28091921290919312A091E2
:105F90009412B09195128EA39FA3A8A7B9A789A325
:105FA0009AA3ABA3BCA39920C9F18091971388232E
:105FB000A9F164E47BE0CE0101960E94464CCE013B
:105FC00001960E948F8FCE0101960E94F24B8E01A6
:105FD000075E1F4F5E0195E2A90EB11CD8016D91BD
:105FE0007D918D919D918D0146E00E94F26A68ED50
:105FF0007BE080E19FE00E948D4DA016B10671F715
:106000006FEB79E0CE0101960E94564CCE010196CD
:106010000E948F8FCE0101960E94F24B23E938E156
:1060200044E85FE3C301B2010E940AAF2B013C01C7
:106030006D877E878F87988B22E430E645E85FE3A3
:10604000C701B6010E940AAF6B017C01698B7A8B94
:106050008B8B9C8B25E83BEE41E95FE36EA17FA132
:1060600088A599A50E940AAF6D8B7E8B8F8B988F28
:1060700040928A1250928B1260928C1270928D1202
:10608000C0928E12D0928F12E0929012F0929112E2
:10609000609392127093931280939412909395123E
:1060A000992009F4A0C080919713882309F49BC01C
:1060B00067E37BE0CE0101960E94464CCE0101963B
:1060C0000E948F8FCE0101960E94F24B8E01035FDA
:1060D0001F4F6E01B9E1CB0ED11C7801F80161911F
:1060E0007191819191918F0142E00E94F26A68ED75
:1060F0007BE080E19FE00E948D4DC016D10671F7D4
:106100006FEB79E0CE0101960E94564CCE010196CC
:106110000E948F8FCE0101960E94F24B46E952E118
:1061200066E070E082E30E944051A0909612B09029
:106130009712C0909812D090991200919A121091D3
:106140009B126AE27BE080E19FE00E94C24C4AE041
:1061500050E0B50180E19FE00E94434D68ED7BE097
:1061600080E19FE00E948D4D4AE050E0B60180E161
:106170009FE00E94434D68ED7BE080E19FE00E943C
:106180008D4D4AE050E0B80180E19FE00E94434D10
:106190006FEB79E080E19FE00E94AE6ACE0101964C
:1061A0000E94125261E27BE080E19FE00E94C24CBB
:1061B0008E010F5F1F4FD8016D917D918D919D9143
:1061C0008D014AE00E94F26A68ED7BE080E19FE089
:1061D0000E948D4D0E151F0571F76FEB79E080E180
:1061E0009FE00E94AE6A61E08DE10E94A551992076
:1061F000B1F080919713882391F06DE07BE080E10E
:106200009FE00E94C24CAE014B5D5F4F61E070E0C9
:106210008DE10E9440518DA190E00E94795162E091
:106220008EE10E94A55163E08FE10E94A55164E0D8
:1062300080E20E94A551992009F450C080919713E3
:10624000882309F44BC061EF7AE080E19FE00E946F
:10625000C24CAE014B5D5F4F61E070E08EE10E9489
:106260004051CDA0D12CAE014B5D5F4F61E070E09D
:106270008FE10E944051EDA0F12CAE014B5D5F4FCC
:1062800061E070E080E20E9440510DA110E04AE020
:1062900050E0B60180E19FE00E94434D68ED7BE055
:1062A00080E19FE00E948D4D4AE050E0B70180E11F
:1062B0009FE00E94434D68ED7BE080E19FE00E94FB
:1062C0008D4D4AE050E0B80180E19FE00E94434DCF
:1062D0006FEB79E080E19FE00E94AE6A65E081E2C9
:1062E0000E94A5519920B1F080919713882391F0D5
:1062F0006EED7AE080E19FE00E94C24CAE014B5D02
:106300005F4F61E070E081E20E9440518DA190E01A
:106310000E94795166E082E20E94A5519920B1F075
:1063200080919713882391F066EC7AE080E19FE0FA
:106330000E94C24CAE014B5D5F4F61E070E082E2B3
:106340000E9440518DA190E00E94795167E083E264
:106350000E94A5519920B1F080919713882391F064
:1063600060EB7AE080E19FE00E94C24CAE014B5DA1
:106370005F4F61E070E083E20E9440518DA190E0A8
:106380000E94795168E084E20E94A5519920B1F001
:1063900080919713882391F068E97AE080E19FE08B
:1063A0000E94C24CAE014B5D5F4F61E070E084E241
:1063B0000E9440518DA190E00E94795169E085E2F0
:1063C0000E94A5519920B1F080919713882391F0F4
:1063D0006EE77AE080E19FE00E94C24CAE014B5D27
:1063E0005F4F61E070E085E20E9440518DA190E036
:1063F0000E9479516AE086E20E94A5519920B1F08D
:1064000080919713882391F068E67AE080E19FE01D
:106410000E94C24CAE014B5D5F4F61E070E086E2CE
:106420000E9440518DA190E00E9479516BE088E27A
:106430000E94A5519920B1F080919713882391F083
:106440006FE47AE080E19FE00E94C24CAE014B5DB8
:106450005F4F61E070E088E20E9440518DA190E0C2
:106460000E9479516CE089E20E94A551992009F4BB
:1064700079C080919713882309F474C067E37AE0A8
:1064800080E19FE00E94C24CAE014B5D5F4F61E036
:1064900070E089E20E9440518DA190E00E94795104
:1064A00060E27AE080E19FE00E94C24C66E070E02A
:1064B00087E20E948B5190E00E94795169E07AE076
:1064C00080E19FE00E94C24C65E070E087E20E949C
:1064D0008B5190E00E94795162EF79E080E19FE07A
:1064E0000E94C24C64E070E087E20E948B5190E011
:1064F0000E94795169ED79E080E19FE00E94C24CF1
:1065000062E070E087E20E948B5190E00E94795136
:1065100060EC79E080E19FE00E94C24C61E070E0B5
:1065200087E20E948B5190E00E94795167EA79E0FE
:1065300080E19FE00E94C24C60E070E087E20E9430
:106540008B5190E00E94795166E979E080E19FE00B
:106550000E94C24C63E070E087E20E948B5190E0A1
:106560000E94795141E067E070E087E20E94B851F3
:1065700041E063E070E087E20E94B85141E063E0EF
:1065800070E08AE20E94B851992091F080919713AF
:10659000882371F06DE779E080E19FE00E94C24CB2
:1065A00063E070E08AE20E948B5190E00E94795192
:1065B00040E063E070E08AE20E94B851992091F0D7
:1065C00080919713882371F063E679E080E19FE082
:1065D0000E94C24C63E070E08AE20E948B5190E01E
:1065E0000E94795141E062E070E08AE20E94B85175
:1065F000992091F080919713882371F067E479E0F6
:1066000080E19FE00E94C24C62E070E08AE20E945A
:106610008B5190E00E94795140E062E070E08AE2A4
:106620000E94B851992091F080919713882371F0BE
:106630006AE279E080E19FE00E94C24C62E070E093
:106640008AE20E948B5190E00E94795141E061E022
:1066500070E08AE20E94B851992091F080919713DE
:10666000882371F06EE079E080E19FE00E94C24CE7
:1066700061E070E08AE20E948B5190E00E947951C3
:1066800040E061E070E08AE20E94B851992091F008
:1066900080919713882371F061EF78E080E19FE0AB
:1066A0000E94C24C61E070E08AE20E948B5190E04F
:1066B0000E94795141E060E070E08AE20E94B851A6
:1066C000992091F080919713882371F065ED78E01F
:1066D00080E19FE00E94C24C60E070E08AE20E948C
:1066E0008B5190E00E94795140E060E070E08AE2D6
:1066F0000E94B851992091F080919713882371F0EE
:1067000068EB78E080E19FE00E94C24C60E070E0BE
:106710008AE20E948B5190E00E94795141E066E04C
:1067200070E087E20E94B85141E065E070E087E2E6
:106730000E94B85141E064E070E087E20E94B851E5
:1067400040E062E070E087E20E94B85140E061E022
:1067500070E087E20E94B85140E060E070E087E2BC
:106760000E94B851992009F475C08091971388232D
:1067700009F470C060EA78E080E19FE00E94C24CBA
:1067800066E070E08BE20E948B5190E00E947951AC
:1067900062E878E080E19FE00E94C24C65E070E032
:1067A0008BE20E948B5190E00E94795164E678E080
:1067B00080E19FE00E94C24C64E070E08BE20E94A6
:1067C0008B5190E00E9479516BE478E080E19FE08A
:1067D0000E94C24C62E070E08BE20E948B5190E01C
:1067E0000E94795162E378E080E19FE00E94C24C10
:1067F00061E070E08BE20E948B5190E00E94795141
:1068000069E178E080E19FE00E94C24C60E070E0C6
:106810008BE20E948B5190E00E94795166E078E013
:1068200080E19FE00E94C24C63E070E08BE20E9436
:106830008B5190E00E94795161EF77E080E19FE019
:106840000E94C24C64E070E08CE20E948B5190E0A8
:106850000E94795140E064E070E08CE20E94B851FF
:10686000AE014B5D5F4F61E070E08CE20E944051F1
:106870006DA1607F66608CE20E94A551992009F4A9
:106880005FC080919713882309F45AC06DED77E0BB
:1068900080E19FE00E94C24CAE014B5D5F4F61E022
:1068A00070E08CE20E9440516DA16F7070E0665004
:1068B0007109072E000C880B990B0E94ABAE9B014F
:1068C000AC0160E070E080E090E40E94A3B220E0C0
:1068D00030E048EC50E40E940AAF0E94035266EC9C
:1068E00077E080E19FE00E94C24CAE014B5D5F4FBC
:1068F00061E070E080E30E9440516DA14AE050E009
:1069000080E19FE00E94E8516EEA77E080E19FE03D
:106910000E94C24C61E070E080E30E948B5190E0E5
:106920000E94795165E977E080E19FE00E94C24CC6
:1069300061E070E08FE20E948B5190E00E947951FB
:1069400041E061E070E08FE20E94B851992091F03F
:1069500080919713882371F06DE777E080E19FE0E5
:106960000E94C24C61E070E08EE20E948B5190E088
:106970000E94795141E061E070E08EE20E94B851DE
:1069800040E067E070E081E30E94B851992009F48B
:1069900055C080919713882309F450C06AE677E0C8
:1069A00080E19FE00E94C24C67E070E081E30E94BA
:1069B0008B5190E00E9479516AE178E080E19FE09C
:1069C0000E948D4DAE014B5D5F4F61E070E080E055
:1069D0000E9440518DA10E948D586FEB79E080E1BB
:1069E0009FE00E94AE6A0DE110E06DE976E080E183
:1069F0009FE00E948D4D40E150E0B80180E19FE0B2
:106A00000E94434D6EE178E080E19FE00E948D4D51
:106A1000AE014B5D5F4F61E070E0802F0E944051FE
:106A20008DA10E948D586FEB79E080E19FE00E947C
:106A3000AE6A0F5F1F4F0A331105B9F6A9960FB65C
:106A4000F894DEBF0FBECDBFDF91CF911F910F91A4
:106A5000FF90EF90DF90CF90BF90AF909F907F908E
:106A60006F905F904F9008954F925F926F927F92D8
:106A70009F92AF92BF92CF92DF92EF92FF920F93CD
:106A80001F93CF93DF93CDB7DEB7A8970FB6F894D7
:106A9000DEBF0FBECDBF6EE372E188E392E10E94DC
:106AA000DD4B0E9421856EE478E0CE0101960E94C4
:106AB000564CBE016F5F7F4F88E392E10E940685CE
:106AC000182FCE0101960E94F24B112309F4E6C063
:106AD0008091421290914312409718F080E00C94FC
:106AE000C53E42E050E06EE372E1CE0101960E94A5
:106AF000273FBE016F5F7F4F8AE192E10E940F4BFB
:106B0000CE0101960E94F24B6AE172E1CE0101963C
:106B10000E944E4CCE0101960E948F8FCE010196AD
:106B20000E94F24B8AE192E10E94324A20E030E07A
:106B300048EC52E40E940AAF0E9494B1AB01BC0140
:106B4000409343025093440260934502709346027F
:106B5000CE0101960E94816ACE0101960E948F8F1C
:106B6000CE0101960E94F24B609143027091440263
:106B700080914502909146028B019C0100591F456E
:106B80002140310901341C4921053105D0F061E271
:106B900078E0CE0101960E94564C6AE172E1CE0186
:106BA00001960E94724B64E378E00E945B4BBC014B
:106BB00080E292E10E94DD4BCE0101960E94F24BF1
:106BC0004EC01A821982FE01339626E0DF011D9223
:106BD0002A95E9F70E94ABAE20E030E048EC52E4A1
:106BE0000E94FBB08E010F5F1F4F22E047E00E9422
:106BF00015AABC0180E292E10E94C84B64E478E0EF
:106C0000CE0145960E94564C60E272E1CE01459657
:106C10000E94724B61E578E00E945B4BBC0180E210
:106C200092E10E94DD4BCE0145960E94F24B1092FC
:106C30003A0C1092390C8091430290914402A09139
:106C40004502B091460280938B1090938C10A093D4
:106C50008D10B0938E1080E090E00E94836E61E111
:106C600079E0CE0101960E94564C60E272E1CE01BD
:106C700001960E94724BBC01CE0145960E944E4C7B
:106C8000CE0145960E940A71CE0145960E94F24BB4
:106C9000CE0101960E94F24B0C94C23E66E578E06C
:106CA000CE0101960E94564CBE016F5F7F4F88E374
:106CB00092E10E940685182FCE0101960E94F24BA8
:106CC0001123C9F126E030E044E050E06EE372E1C8
:106CD000CE0101960E946A4CBE016F5F7F4F8AE130
:106CE00092E10E940F4BCE0101960E94F24B8AE185
:106CF00092E10E943D4A70930411609303117093D6
:106D00002A02609329026EE372E1CE0101960E948D
:106D10004E4CCE0101960E948F8FCE0101960E94AB
:106D2000F24B10923A0C1092390C80E090E00E94E5
:106D3000836E0C94C23E6BE578E0CE0101960E9412
:106D4000564CBE016F5F7F4F88E392E10E9406853B
:106D5000182FCE0101960E94F24B112309F411C1A4
:106D60000AE010E0C12CD12C7601AA24AA9443E0B9
:106D7000B42E6EE170E080E090E00E942B8680915E
:106D800061020E94E185B5010E945CB3072E000CF0
:106D9000880B990B0E94ABAE20E030E040EA50E453
:106DA0000E940AAF9B01AC01C701B6010E9435B039
:106DB0006B017C0101501109E1F620E030E040E276
:106DC00051E40E94FBB06B017C016EE578E0CE01DE
:106DD00001960E94564CBE016F5F7F4F88E392E19F
:106DE0000E940685182FCE0101960E94F24B1123B6
:106DF00009F446C020E030E040E650E4C701B601A7
:106E00000E940AAF9B01AC0160E070E080E890E472
:106E10000E9434B060931D0270931E0280931F0283
:106E20009093200260EC7CE080E292E10E94834B30
:106E300040911D0250911E0260911F02709120022C
:106E400022E0CE0101960E94F74BBE016F5F7F4F9B
:106E500080E292E10E94094BCE0101960E94F24B22
:106E600080911D0290911E02A0911F02B0912002FC
:106E70008093AF109093B010A093B110B093B21064
:106E800062E678E0CE0101960E94564CBE016F5F2B
:106E90007F4F88E392E10E940685182FCE0101966C
:106EA0000E94F24B112309F44EC020E030E040E68E
:106EB00050E4C701B6010E940AAF9B01AC0160E03B
:106EC00070E080E291E40E9434B060931902709304
:106ED0001A0280931B0290931C026FEA7CE080E20E
:106EE00092E10E94834B4091190250911A026091E5
:106EF0001B0270911C0222E0CE0101960E94F74B0A
:106F0000BE016F5F7F4F80E292E10E94094BCE018C
:106F100001960E94F24B8091190290911A02A09161
:106F20001B02B0911C028093B3109093B410A093F5
:106F3000B510B093B61010923A0C1092390C80E054
:106F400090E00E94836E61E179E0CE0101960E949B
:106F5000564C60E272E1CE0101960E94724BBC0178
:106F6000CE0145960E944E4CCE0145960E940A7174
:106F7000CE0145960E94F24BCE0101960E94F24B43
:106F800003C767E678E0CE0101960E94564CBE0129
:106F90006F5F7F4F88E392E10E940685182FCE0134
:106FA00001960E94F24B112309F4B8C0809142125D
:106FB000909143120797F0F046E050E06EE372E1E3
:106FC000CE01019644D7BE016F5F7F4F8AE192E107
:106FD0000E940F4BCE0101960E94F24B8AE192E192
:106FE0000E94324A60932502709326028093270202
:106FF0009093280280915F029091600299270E94ED
:10700000B3782DE038E643E55BE30E940AAF6B01FD
:107010007C0120918302309184024091850250913D
:1070200086020E94A5AE18164CF060916B0270911A
:107030006C0280916D0290916E021BC020919702AC
:10704000309198024091990250919A02C701B6017D
:107050000E94EAB187FF05C0C701B6010E94F16C2A
:1070600008C060917F0270918002809181029091AE
:10707000820220E030E048EC52E40E940AAF6B014B
:107080007C0120E030E0A9010E94A5AE181634F082
:10709000C12CD12C38EAE32E31E4F32EC092250224
:1070A000D0922602E0922702F0922802C092BF10EE
:1070B000D092C010E092C110F092C210809197134C
:1070C000882381F06DE97CE080E19FE00E94C24C62
:1070D00060912502709126028091270290912802EA
:1070E0000E94035210923A0C1092390C80E090E00A
:1070F0000E94836E63E97CE080E292E10E94834B10
:107100004091250250912602609127027091280239
:1071100022E0CE0101960E94F74B44C26DE678E072
:10712000CE0101960E94564CBE016F5F7F4F88E3EF
:1071300092E10E940685182FCE0101960E94F24B23
:10714000112309F46EC0B0905D0260E08B2D0E94A7
:10715000A58509E110E0C12CD12C76018B2D0E9470
:10716000E185BC01990F880B990B0E94ABAE9B0186
:10717000AC01C701B6010E9435B06B017C016AE029
:1071800070E080E090E00E942B860150110931F7F9
:1071900020E030E040EA50E4C701B6010E940AAFA7
:1071A00020E030EC4FE754E40E94FBB020E030E0F8
:1071B00048EC51E40E94FBB06093210270932202DC
:1071C00080932302909324026093D5107093D6107D
:1071D0008093D7109093D81010923A0C1092390CDB
:1071E00080E090E00E94836E60E87CE080E292E1C3
:1071F0000E94834B40912102509122026091230210
:107200007091240222E0CE0101960E94F74BBE014C
:107210006F5F7F4FCE0145960E944E4C6DEC75E03E
:1072200054C061E778E0CE0101960E94564CBE0141
:107230006F5F7F4F88E392E10E940685182FCE0191
:1072400001960E94F24B112309F454C08091BA10A8
:10725000082E000C990B0197039708F044C089E3AE
:1072600090E00E94B3782AE137E64CE950E40E94AE
:107270000AAF6093BB107093BC108093BD109093C5
:10728000BE1010923A0C1092390C80E090E00E94EF
:10729000836E6FE57CE080E292E10E94834B409137
:1072A000BB105091BC106091BD107091BE1022E0D7
:1072B000CE0101960E94F74BBE016F5F7F4FCE015A
:1072C00045960E944E4C67E778E0CE0145960E94B5
:1072D0005B4BBC0180E292E10E94094BCE014596D6
:1072E0000E94F24B66C169E37CE080E292E10E9479
:1072F000834B3AC56AE778E0CE0101960E94564C6E
:10730000BE016F5F7F4F88E392E10E940685182FD0
:10731000CE0101960E94F24B112309F44DC126E0E3
:1073200030E044E050E06EE372E1CE0101960E944D
:107330006A4CBE016F5F7F4F8AE192E10E940F4B62
:10734000CE0101960E94F24B8AE192E10E943D4AF1
:107350006B017C015B0164ED7AE0CE0101960E9435
:10736000564CBE016F5F7F4F8EE392E10E94B68460
:107370008E010B5E1F4FAC014F5F5F4F6EE372E1FA
:10738000C80165D5B8018AE192E10E940F4BC8019E
:107390000E94F24BCE0101960E94F24B90905B024C
:1073A0008AE192E10E94324A2B013C0180919713BD
:1073B0008823B9F062E57BE080E19FE00E94C24C47
:1073C0004AE050E0B60180E19FE00E94434D68ED45
:1073D0007BE080E19FE00E948D4DC301B2010E94DD
:1073E0000352692DC8010E94345718870F831D82EC
:1073F0001E82198289E08A8381E08B838C831C8AB8
:107400001B8ACE0101960E944154CE0101960E9432
:10741000D553CE0101960E9406530E8110E00B3029
:10742000110514F00AE010E0BBE5CB16D10408F416
:107430004CC021E1C22E2CE0D22E5601412C512C01
:107440003201E12CF12CE016F106BCF46E2DCE01D8
:1074500001960E9497529B01AC01F50161937193D3
:10746000819391935F01C301B2010E9435B02B015A
:107470003C01FFEFEF1AFF0AE6CFB801012E000C26
:10748000880B990B0E94ABAE9B01AC01C301B2010A
:107490000E94FBB02B013C01E12CF12CE016F1061F
:1074A0000CF05AC0D6012D913D914D915C91C301D4
:1074B000B2010E9434B0F60161937193819391936C
:1074C0006F01FFEFEF1AFF0AE9CF1A141B0424F52E
:1074D0000A151B0524F041E0C41AD10804C0680154
:1074E00081E0C81AD1086C2DCE0101960E949752F6
:1074F0009B01AC018601000F111F000F111F0F5ED1
:10750000134FC301B2010E9434B0D8016D937D9333
:107510008D939C93139720C0AB28F1F481E1C82E82
:107520008CE0D82EE12CF12CE016F106ACF46E2D97
:10753000CE0101960E9497529B01AC01C301B2019A
:107540000E9434B0F60161937193819391936F011E
:10755000FFEFEF1AFF0AE8CFE1E1FCE0A9EDB0E1AF
:1075600089E39CE041915191619171914D935D93BB
:107570006D937D938E179F07A9F710923A0C109286
:10758000390C80E090E00E94836E68E17CE080E24C
:1075900092E10E94834B44E050E06EE372E1CE0141
:1075A000019655D4BE016F5F7F4F80E292E10E9449
:1075B000094BCE010196D6C36EE778E0CE01019665
:1075C0000E94564CBE016F5F7F4F88E392E10E949C
:1075D0000685182FCE0101960E94F24B112309F463
:1075E00024C127E030E046E050E06EE372E1CE01D6
:1075F00001960E946A4CBE016F5F7F4F8AE192E163
:107600000E940F4BCE0101960E94F24B8AE192E15B
:107610000E943D4A8B016093BA108EE392E10E9472
:10762000484A68ED7BE0CE0101960E94564CBE01AF
:107630006F5F7F4F8EE392E10E94B684AC014F5F93
:107640005F4F6EE372E1CE01459601D4CE014596BF
:107650000E94324A6093BB107093BC108093BD109F
:107660009093BE10CE0145960E94F24BCE0101963A
:107670000E94F24B67E07CE080E292E10E94834B43
:107680000430110594F4023011050CF05BC00115B3
:107690001105B1F00130110509F09BC069EF7BE0E5
:1076A00080E292E10E94B94A77C00430110509F0E6
:1076B00090C066EE7BE080E292E10E94B94AACC0E5
:1076C00020E030E0A9016091BB107091BC10809166
:1076D000BD109091BE100E94A5AE181664F080E017
:1076E00090E0A0E8BFE38093BB109093BC10A09300
:1076F000BD10B093BE102091BB103091BC104091D2
:10770000BD105091BE1060E070E080EA90E40E94ED
:10771000FBB0AB01BC0122E0CE0145960E94F74BC5
:1077200065E878E0CE0101960E94564CBE016B5E82
:107730007F4FCE0101960E94724B64ED78E00E946B
:107740005B4B5DC06DEE7BE080E292E10E94B94A46
:107750008AE0809FB001819F700D1124CE010196B7
:107760000E947C50BE016F5F7F4FCE0145960E9404
:107770004E4C6DEC78E0CE0145960E945B4BBC010F
:1077800080E292E10E94094BCE0145960E94F24BA5
:10779000CE0101960E94F24B20E030E048E453E431
:1077A0006091BB107091BC108091BD109091BE1083
:1077B0000E94A5AE181684F180E090E4ACE1B5E437
:1077C0008093BB109093BC10A093BD10B093BE10DB
:1077D00023C06091BA10062E000C770BCE0145969F
:1077E0000E947C5060E978E0CE0101960E94564CE0
:1077F000BE016B5E7F4FCE0101960E94724BBC01B1
:1078000080E292E10E94094BCE0101960E94F24B68
:10781000CE0145960E94F24B10923A0C1092390C10
:1078200080E090E00E94836E9FC267E978E0CE011D
:1078300001960E94564CBE016F5F7F4F88E392E134
:107840000E940685182FCE0101960E94F24B11234B
:1078500009F4CEC027E030E046E050E06EE372E18C
:10786000CE0101960E946A4CBE016F5F7F4F8AE194
:1078700092E10E940F4BCE0101960E94F24B8AE1E9
:1078800092E10E943D4A6093B7108EE392E10E941C
:10789000484A8AE192E10E943D4A611571058105DD
:1078A000910519F485E090E007C06130710581050C
:1078B000910539F489E190E09093B9108093B81064
:1078C00025C068ED7BE0CE0101960E94564CBE01BA
:1078D0006F5F7F4F8EE392E10E94B684AC014F5FF1
:1078E0005F4F6EE372E1CE014596B1D2CE0145966F
:1078F0000E943D4A7093B9106093B810CE0145962E
:107900000E94F24BCE0101960E94F24B10923A0C6B
:107910001092390C80E090E00E94836E65ED7BE070
:1079200080E292E10E94834B8091B710833044F54E
:107930006AEC7BE080E292E10E94B94A6091B81063
:107940007091B910CE0101960E947C50BE016F5F0C
:107950007F4FCE0145960E944E4C62EB7BE0CE01FC
:1079600045960E945B4BBC0180E292E10E94094B6C
:10797000CE0145960E94F24BCE0101960E94F24B39
:107980008091B71083300CF4EFC16091B810709102
:10799000B910CE0183960E947C506091B710062EDC
:1079A000000C770BCE0145960E947C5060E978E090
:1079B000CE0101960E94564CBE016B5E7F4FCE01F8
:1079C00001960E94724BBE016D5D7F4F0E94724B0B
:1079D000BC0180E292E10E94094BCE0101960E9417
:1079E000F24BCE0145960E94F24BCE018396BAC16E
:1079F0006EE978E0CE0101960E94564CBE016F5FA1
:107A00007F4F88E392E10E940685182FCE010196F0
:107A10000E94F24B112309F456C0809159029091B3
:107A20005A020E94C47960932B0270932C028093B7
:107A30002D0290932E026093A3107093A410809354
:107A4000A5109093A61080E090E5A3ECB7E4809396
:107A5000330290933402A0933502B09336028093A0
:107A60009B1090939C10A0939D10B0939E108091BA
:107A70009713882381F06CEA7BE080E19FE00E940D
:107A8000C24C60912B0270912C0280912D0290913A
:107A90002E020E94035210923A0C1092390C80E090
:107AA00090E00E94836E40912B0250912C026091D5
:107AB0002D0270912E0222E0CE0145960E94F74BD6
:107AC00062EA78E039C16DEA78E0CE0101960E9461
:107AD000564CBE016F5F7F4F88E392E10E9406859E
:107AE000182FCE0101960E94F24B112309F484C095
:107AF00080914212909143120497F0F044E050E0DC
:107B00006EE372E1CE010196A2D1BE016F5F7F4F9D
:107B10008AE192E10E940F4BCE0101960E94F24B46
:107B20008AE192E10E94324A6093370270933802F0
:107B30008093390290933A028091370290913802F3
:107B4000A0913902B0913A028093971090939810C7
:107B5000A0939910B0939A1080919713882389F07D
:107B600063E97BE080E19FE00E94C24C60913702B4
:107B7000709138028091390290913A0242E00E945D
:107B8000F26A8091590290915A020E94C4796093DE
:107B90002F027093300280933102909332026093EF
:107BA0009F107093A0108093A1109093A2108091C9
:107BB0009713882381F069E87BE080E19FE00E94D1
:107BC000C24C60912F0270913002809131029091ED
:107BD00032020E94035210923A0C1092390C80E04B
:107BE00090E00E94836E40912F025091300260918C
:107BF00031027091320299C069EB78E0CE010196B2
:107C00000E94564CBE016F5F7F4F88E392E10E9455
:107C10000685182FCE0101960E94F24B112311F414
:107C20000C946E3580914212909143120497F0F0BB
:107C300044E050E06EE372E1CE01019608D1BE014E
:107C40006F5F7F4F8AE192E10E940F4BCE01019658
:107C50000E94F24B8AE192E10E94324A6093330221
:107C600070933402809335029093360280913302F0
:107C700090913402A0913502B091360280939B100E
:107C800090939C10A0939D10B0939E108091971399
:107C9000882389F060E77BE080E19FE00E94C24C8E
:107CA00060913302709134028091350290913602D6
:107CB00042E00E94F26A8091590290915A020E9419
:107CC000C47960932B0270932C0280932D029093C1
:107CD0002E026093A3107093A4108093A51090932C
:107CE000A61080919713882381F066E67BE080E1FF
:107CF0009FE00E94C24C60912B0270912C028091F7
:107D00002D0290912E020E94035210923A0C109272
:107D1000390C80E090E00E94836E40912B025091DC
:107D20002C0260912D0270912E0222E0CE01459628
:107D30000E94F74B61EB78E0CE0101960E94564C11
:107D4000BE016B5E7F4FCE0101960E94724BBC015B
:107D500080E292E10E94DD4BCE0101960E94F24B3F
:107D6000CE0145960E94F24B60E272E1CE0101968F
:107D70000E944E4CCE0101960E940A71CE010196DE
:107D80000E94F24B1092540281E0A8960FB6F8942C
:107D9000DEBF0FBECDBFDF91CF911F910F91FF903E
:107DA000EF90DF90CF90BF90AF909F907F906F90BB
:107DB0005F904F900895089580912E058823F9F0E3
:107DC00080912D058823D9F081E00E94456A8BE3DC
:107DD0009FE10197F1F760E080E00E94566A6CE94C
:107DE0007DE081E293E10E94C24C61E080E00E946C
:107DF000566A6CE87DE081E293E10C94C24C0895F0
:107E000080912E05882349F080912D05882329F043
:107E100060E081E293E10C9488570895FF920F93FC
:107E20001F93CF93DF93EC01F62E08811981C801CF
:107E30000E94C1AFF81621F06F2DC8010E94C9AF92
:107E4000CE01DF91CF911F910F91FF900895CF93B5
:107E5000DF93EC01FB01248135810E946A4CCE0145
:107E6000DF91CF9108953F924F925F926F927F92F0
:107E70008F929F92AF92BF92CF92DF92EF92FF923A
:107E80000F931F93CF93DF93CDB7DEB7E4970FB671
:107E9000F894DEBF0FBECDBF80914413882319F044
:107EA000109244134CC381E0809344136FEB79E04C
:107EB000CE0185960E94564C6FEB79E0CE018B96F1
:107EC0000E94564C00E010E082E0382E98EEC92E59
:107ED00093E0D92EE12CF12CF8013197E031F10536
:107EE00030F48827E856FF4F8F4F0C946FB36FEB39
:107EF00079E0CE0185960E94C84B80910111909146
:107F00000211892B31F469E077E0CE0185960E9459
:107F1000C84B8091011190910211019731F46DE0ED
:107F200077E0CE0185960E94C84B80910111909117
:107F30000211029731F463E177E0CE0185960E9449
:107F4000C84B89A59AA5892B31F065E173E1CE0173
:107F500085960E94094B6DEB78E0CE0101960E9458
:107F6000564C6FE073E1CE0101960E94724BBC014A
:107F7000CE018B960E94DD4BCE0101960E94F24B02
:107F80008091011190910211019709F03BC2BE014D
:107F90006B5D7F4FCE0101960E944E4C48EC50E045
:107FA0006FEF7FEFCE0101960E94BB8FCE0101964D
:107FB0000E94F24BBE01655D7F4FCE0101960E948B
:107FC0004E4C40ED57E06FEF7FEFCE0101960E94DF
:107FD000738DCE0101960E94F24BCE0101960E9454
:107FE000C9608D819E810097A1F0E981FA8120818D
:107FF000222379F0079768F065E77FE0CE01859648
:108000000E94834BBE016F5F7F4FCE018B960E9413
:10801000DD4BCE01019696C069E67FE0CE018596E4
:108020000E94834B0E9487874B015C010E948787D7
:10803000A70196010E9403B0CA01B90120E831E509
:1080400041E050E00E9403B020E13EE040E050E01B
:108050000E94D7AF29AB3AAB4BAB5CAB2CE330E023
:1080600040E050E00E94D7AF29013A01AB01BC01CA
:10807000CE0101960E94816AB301A201CE0107964A
:108080000E94816A49A95AA96BA97CA9CE010D96C3
:108090000E94816AC501B40120E03CE546E255E05A
:1080A0000E9403B0BA01A901CE0149960E94816ADB
:1080B000BE01675E7F4FCE0143960E944E4C62EC3C
:1080C00078E0CE0143960E945B4BBE01635F7F4F19
:1080D0000E94724B65EC78E00E945B4BBE01695FC9
:1080E0007F4F0E94724B68EC78E00E945B4BBE01B0
:1080F0006F5F7F4F0E94724B6BED75E00E945B4B90
:10810000BC01CE014F960E944E4CCE0143960E9478
:10811000F24BCE0149960E94F24BCE010D960E9481
:10812000F24BCE0107960E94F24BCE0101960E94BF
:10813000F24BBE01615E7F4FCE018B960E940F4BCA
:10814000CE014F960E94F24B5DC180910F0C909131
:10815000100C019719F46AE57FE002C06CE47FE03F
:10816000CE0185960E94834B6CE37FE047C16CE2B1
:108170007FE0CE0185960E94834B6FE17FE03EC198
:1081800062E17FE0CE0185960E94834B67E07FE04D
:1081900035C16BEF7EE0CE0185960E94834B6AEE7F
:1081A0007EE02CC180910F0C9091100C039719F474
:1081B0006FED7EE002C065ED7EE0CE0185960E9407
:1081C000834B6AEC7EE01AC16DEB7EE0CE018596B2
:1081D0000E94834B6EEA7EE011C163EA7EE0CE012D
:1081E00085960E94834B6091B8107091B910CE01B2
:1081F00007960E947C5061EE7BE0CE0101960E94C2
:10820000564CBE01695F7F4FCE0101960E94724BB2
:1082100062EB7BE00E945B4BBC01CE0185960E9425
:10822000094BCE0101960E94F24BCE0107960E94A7
:10823000F24B66E97EE0E2C080910F0C9091100C49
:10824000029719F465E87EE002C065E77EE0CE01A2
:1082500085960E94834B68E67EE0D0C06CE57EE0A8
:10826000CE0185960E94834B6CE47EE0C7C061E43A
:108270007EE0CE0185960E94834B67E37EE0BEC020
:108280006BE27EE0CE0185960E94834B6BE17EE03F
:10829000B5C0B090BA1060E17EE0CE0185960E9434
:1082A000834B83E08B1574F092E0B9160CF045C057
:1082B000BB2081F081E0B81261C06BEC78E0CE01A8
:1082C000859659C094E0B91259C06FEC78E080E20D
:1082D00092E151C08090BB109090BC10A090BD1056
:1082E000B090BE1020E030E048E452E4C501B40193
:1082F0000E94A5AE87FF02C033243394A5019401E8
:1083000060E070E080EA90E40E94FBB0AB01BC0149
:10831000232DCE0107960E94F74B69EF78E0CE013E
:1083200001960E94564CBE01695F7F4FCE010196B7
:108330000E94724B64ED78E018C08B2D9AE08902A0
:10834000B0011124CE0107960E947C5061EE7BE0C3
:10835000CE0101960E94564CBE01695F7F4FCE014F
:1083600001960E94724B6DEC78E00E945B4BBC0161
:10837000CE0185961CC00E94FB4A23C06091BA10B2
:10838000062E000C770BCE0107960E947C5067E901
:108390007AE0CE0101960E94564CBE01695F7F4F84
:1083A000CE0101960E94724BBC0180E292E10E94D4
:1083B000094BCE0101960E94F24BCE0107960E9416
:1083C000F24B60E07EE01AC063EF7DE0CE0185965F
:1083D0000E94834B63EE7DE011C067ED7DE0CE012E
:1083E00085960E94834B68EC7DE008C06CEB7DE0D5
:1083F000CE0185960E94834B6CEA7DE0CE018B9680
:108400000E94834BBE016B5D7F4FCE0101960E949F
:108410004E4C48EC50E06FEF7FEFCE0101960E948A
:108420006090CE0101960E94F24BBE01655D7F4FC8
:10843000CE0101960E944E4C48EC50E06FEF7FEF6A
:10844000CE0101960E94738DCE0101960E94F24BDF
:108450000E94FA97982EA12CB12C91106DC08FEF2D
:10846000A81AB80A95E6A916B10451F00E94FA9725
:10847000982E64E170E080E090E00E942B86EDCFC2
:108480006FEB79E08EE392E10E94C84BCE0101963A
:108490000E947174BE016F5F7F4F8EE392E10E9474
:1084A0000F4BCE0101960E94F24B809142129091A7
:1084B0004312892B89F461E070E0CE0101960E949D
:1084C0002F8BBE016F5F7F4F8EE392E10E940F4BB7
:1084D000CE0101960E94F24B80914212909143127C
:1084E000892B89F461E070E0CE0101960E94CD896C
:1084F000BE016F5F7F4F8EE392E10E940F4BCE0172
:1085000001960E94F24B8091421290914312892B66
:1085100051F480914413882331F00F5F1F4F0131D4
:10852000110509F0D9CCCE018B960E94F24BCE01F9
:1085300085960E94F24B03C010924413F4CFE49648
:108540000FB6F894DEBF0FBECDBFDF91CF911F9164
:108550000F91FF90EF90DF90CF90BF90AF909F90E2
:108560008F907F906F905F904F903F9008954F92C3
:108570005F926F927F928F929F92AF92BF92CF92B3
:10858000DF92EF92FF920F931F93CF93DF93CDB7BC
:10859000DEB7C654D1090FB6F894DEBF0FBECDBF0B
:1085A0008C016FEB79E0CE01C7960E94564C6FEBC1
:1085B00079E0CE01CD960E94564CBE016F5F7F4F91
:1085C0008BE592E154D68D889E88AF88B88C498C13
:1085D0005A8C6B8C7C8C8D8D9E8DAF8DB8A127961F
:1085E0008CAF9DAFAEAFBFAF2797C8010197039780
:1085F00008F0ADC1A3019201C501B40190580E94D9
:10860000A8B02BED3FE049EC5FE30E9435B020912C
:108610003F023091400240914102509142020E943B
:1086200035B06B017C0120E030E0A9010E94A5AECD
:1086300087FD09C0C0924E0CD0924F0CE092500CB6
:10864000F092510C10C02BED3FE049EC50E4C70113
:10865000B6010E9435B060934E0C70934F0C80931E
:10866000500C9093510CC0904E0CD0904F0CE09059
:10867000500CF090510C2BED3FE049EC50E4C70159
:10868000B6010E94EAB1181684F42BED3FE049ECE4
:1086900050E4C701B6010E9434B060934E0C709351
:1086A0004F0C8093500C9093510C20E030E044E349
:1086B00053E460914E0C70914F0C8091500C90914E
:1086C000510C0E940AAF2BED3FE049E450E40E94B8
:1086D000FBB060934A0C70934B0C80934C0C9093BE
:1086E0004D0C0E9494B1CE018B960E947C5067ED98
:1086F00078E0CE0185960E94564CBE01655D7F4FA5
:10870000CE018596EFD761EE78E0D5D7BC0186E241
:1087100092E10E94DD4BCE0185960E94F24BCE0184
:108720008B960E94F24BC0904A0CD0904B0CE0907C
:108730004C0CF0904D0C20E030E044EB52E4C701CB
:10874000B6010E94A5AE18168CF020E030E040E0A3
:108750005FE3C701B6010E9435B00E9494B1CE011B
:108760008B960E947C5068EE78E022C020E030E0DA
:1087700044E353E4C701B6010E94A5AE18168CF17C
:10878000A701960160E070E884E393E40E9434B0AE
:1087900060934A0C70934B0C80934C0C90934D0C4F
:1087A0000E9494B1CE018B960E947C506BEE78E0D3
:1087B000CE0185960E94564CBE01655D7F4FCE016D
:1087C000859690D7BC01CE01C796F7D7CE01859686
:1087D0000E94F24BCE018B960E94F24B6AE27BE044
:1087E0005DC020E030E047E853E4C701B6010E94D5
:1087F000A5AE1816FCF020E030E044E353E4C701D6
:10880000B6010E9434B020E030E040E05FE30E9417
:1088100035B060934A0C70934B0C80934C0C909342
:108820004D0C0E9494B1CE018B960E947C506BEE51
:1088300078E01EC0A701960160E070E084EB93E44D
:108840000E9434B020E030E040E05FE30E9435B0A9
:1088500060934A0C70934B0C80934C0C90934D0C8E
:108860000E9494B1CE018B960E947C5068EE78E015
:10887000CE0185960E94564CBE01655D7F4FCE01AC
:10888000859630D7BC01CE01C79697D7CE01859685
:10889000A9D7CE018B96A6D76EEE78E0CE01CD9605
:1088A00077D7BE01695C7F4FCE018596F7D74AE046
:1088B00050E060E070E0CE0185960E94BB8FCE0153
:1088C000859690D70E948787C0909313D090941379
:1088D000E0909513F0909613A4E6CA0ED11CE11C0B
:1088E000F11CC616D706E806F90608F4E7C10E948F
:1088F00087870E94A9AE6B017C01609193137091F0
:10890000941380919513909196130E94ABAE20E042
:1089100030E048EC51E40E9435B09B01AC01C70146
:10892000B6010E94A5AE87FDC9C168ED7BE0CE010E
:108930008596BCD7BE01635C7F4FCE018596D2D6AB
:10894000BC01CE01C79665D6CE0185964BD7C8012E
:108950000297029708F08EC120E030E040E251E437
:10896000C501B4010E940AAF6B017C0120E030E038
:1089700040E251E4C301B2010E940AAF4B015C0125
:1089800020E030E040E251E427966CAD7DAD8EAD45
:108990009FAD27970E940AAF2B013C010E94878759
:1089A0002091EA0B3091EB0B4091EC0B5091ED0BC9
:1089B000621B730B840B950B0E94A9AE20E030E084
:1089C0004AE754E40E94FBB0AB01BC0123E0CE01B6
:1089D0008B960DD769EF78E0CE01859667D7BE01FB
:1089E000655D7F4FCE0185967DD66EEF7AE063D6CA
:1089F000BC0184E192E1E1D6CE018596F3D6CE01A9
:108A00008B96F0D664E172E1CE01859647D766E297
:108A100072E1CE01859666D6BE01695C7F4F62D653
:108A2000BC01CE01C796C9D6CE018596DBD661E8DA
:108A30007DE080E292E167D621E0B701A601CE0198
:108A40008596D5D6BE016B5D7F4F80E292E1E1D580
:108A5000CE018596C7D621E0B301A201CE01C19611
:108A6000C6D621E0B501A401CE018B96C0D668ED33
:108A70007BE0CE0185961AD7BE01655D7F4FCE01A2
:108A8000859630D668ED7BE016D6BE016F5C7F4FD1
:108A900029D660EF78E00FD6BC0180E292E1B9D52B
:108AA000CE0185969FD6CE018B969CD6CE01C196DF
:108AB00099D6A7019601C701B6010E940AAF6B01C2
:108AC0007C01A5019401C501B4010E940AAF9B017C
:108AD000AC01C701B6010E9435B06B017C01A30156
:108AE0009201C301B2010E940AAF9B01AC01C70110
:108AF000B6010E9435B00E94F3B26B017C01609315
:108B0000460C7093470C8093480C9093490C64EF8B
:108B100078E080E292E16FD521E0B701A601CE01B5
:108B2000859665D6BE016B5D7F4FCE018B96B6D61E
:108B300065E079E0CE018B96BED5BC0186E292E17C
:108B40003CD6CE018B964ED6CE0185964BD666E2AC
:108B500072E180E292E15DD5C090460CD090470C66
:108B6000E090480CF090490C20E030E04AE754E4F3
:108B7000C701B6010E94EAB187FD23C020E030E0C2
:108B80004AE754E4C701B6010E94FBB0AB01BC0147
:108B900023E0CE0185962BD6BE016B5D7F4FCE01C3
:108BA0008B967CD666E079E0CE018B9684D5BC01AD
:108BB00086E292E102D6CE018B9614D6CE0185963E
:108BC00011D620E030E64AE656E46091460C7091FA
:108BD000470C8091480C9091490C0E94A5AEBE01B3
:108BE000695C7F4F87FF43C0CE01859657D668EFFB
:108BF00078E0CE0185965FD560E272E173D5BC0165
:108C000080E292E1DAD5CE018596ECD503301105EC
:108C100089F460E272E1CE01859640D6CE01859658
:108C20000E940A71CE018596DDD56FEB79E080E276
:108C300092E1AED56BEF78E0CE01859637D666E24D
:108C400072E1CE0185964ED5BC01CE018B9626D61B
:108C50004AE050E06FEF7FEFCE018B960E94738D5C
:108C6000CE018B96BFD5CE018596BCD503C080E2E0
:108C700092E1A3D56AE070E080E090E00E942B864C
:108C8000CE01CD96AFD5CE01C796ACD5CA5BDF4F2E
:108C90000FB6F894DEBF0FBECDBFDF91CF911F910D
:108CA0000F91FF90EF90DF90CF90BF90AF909F908B
:108CB0008F907F906F905F904F9008956FEB79E069
:108CC000CE018596F3D5CE0185960E94EF8DCE011B
:108CD000859688D5BE01635C7F4F81E293E144D6DF
:108CE00024CE1F93CF93DF93CDB7DEB7A8970FB6EF
:108CF000F894DEBF0FBECDBF182F0E944A508EE100
:108D00000E943B6A62E08DEA9FE00E94445660E068
:108D10008DEA9FE00E9444560E94346A8EE10E94D0
:108D20003B6A61E08DEA9FE00E94445660E28DEA72
:108D30009FE00E9444560E94346A80E290E0909343
:108D40005F1280935E1280E090E8A9E8B4E480931B
:108D5000670290936802A0936902B0936A0280E070
:108D600090E0A5E7B4E48093630290936402A0933B
:108D70006502B0936602BE016F5F7F4F8BE592E1A3
:108D800029D2112309F47CC066E57DE080E19FE0F3
:108D9000F9D580E19FE00E94C36966E47DE080E14F
:108DA0009FE0F0D5BE016F5F7F4F80E19FE00E94A2
:108DB000AE6A66E37DE080E19FE0E4D56D857E8567
:108DC0008F8598890E94BF6A66E27DE080E19FE01E
:108DD000D9D569897A898B899C890E94BF6A66E1A5
:108DE0007DE080E19FE0CED520E030E040E251E43C
:108DF000698D7A8D8B8D9C8D0E940AAF42E00E9416
:108E0000F26A64E079E080E19FE00E94AE6A66E089
:108E10007DE080E19FE0B6D520E030E040E251E423
:108E20006D8D7E8D8F8D98A10E940AAF42E00E94C9
:108E3000F26A64E079E080E19FE00E94AE6A66EF4A
:108E40007CE080E19FE09ED520E030E040E251E40C
:108E500069A17AA18BA19CA10E940AAF42E00E9465
:108E6000F26A64E079E080E19FE00E94AE6A60ED22
:108E70007CE080E19FE086D580E19FE00E94C369AD
:108E800064EF71E080E090E00E942B86A8960FB618
:108E9000F894DEBF0FBECDBFDF91CF911F91089533
:108EA0000895CF92DF92EF92FF920F931F93CF938B
:108EB000DF936C017A018B01C0E0D0E0CE15DF05B5
:108EC00081F0D8016D918D01D601ED91FC91019059
:108ED000F081E02DC6011995892B11F02196EECF76
:108EE0007E01C701DF91CF911F910F91FF90EF900D
:108EF000DF90CF900895FC01538D448D252F30E0F5
:108F0000842F90E0821B930B541710F0CF96089596
:108F100001970895FC01918D828D981761F0828DE3
:108F2000DF01A80FB11D5D968C91928D9F5F9F739D
:108F3000928F90E008958FEF9FEF0895FC01918D3F
:108F4000828D981731F0828DE80FF11D858D90E0AC
:108F500008958FEF9FEF0895FC01918D228D892F49
:108F600090E0805C9F4F821B91098F739927089531
:108F700089E39DE0F1DF21E0892B09F420E0822FD5
:108F8000089586ED9DE0E8DF21E0892B09F420E0DB
:108F9000822F089583E79EE0DFDF21E0892B09F42B
:108FA00020E0822F089580E19FE0D6DF21E0892B29
:108FB00009F420E0822F0895FC01848DDF01A80FC1
:108FC000B11DA35ABF4F2C91848D90E001968F73F1
:108FD0009927848FA689B7892C93A089B1898C9110
:108FE000837080648C93938D848D981306C002885F
:108FF000F389E02D80818F7D80830895EF92FF9229
:109000000F931F93CF93DF93EC0181E0888F9B8DAB
:109010008C8D981305C0E889F989808185FD25C06C
:10902000F62E0B8D10E00F5F1F4F0F731127E02EF0
:109030008C8DE8120BC00FB607FCFACFE889F989CE
:10904000808185FFF5CFCE01B7DFF2CF8B8DFE019A
:10905000E80FF11DE35AFF4FF0829FB7F8940B8F92
:10906000EA89FB89808180620AC09FB7F894EE8903
:10907000FF896083E889F9898081837080648083B7
:109080009FBF81E090E0DF91CF911F910F91FF9002
:10909000EF900895CF93DF93EC01888D8823C1F082
:1090A000EA89FB89808185FD05C0A889B9898C91F1
:1090B00086FD0EC00FB607FCF5CF808185FFF2CF8D
:1090C000A889B9898C9185FFEDCFCE0175DFE8CFF6
:1090D000DF91CF91089580E090E0892B19F063DF54
:1090E000811116C080E090E0892B19F053DF8111C7
:1090F00012C080E090E0892B19F043DF81110EC08F
:1091000080E090E0892B79F033DF81110AC0089567
:109110000E940000E7CF0E940000EBCF0E940000F9
:10912000EFCF0C94000008950E94C3B50F931F93D6
:10913000CF93DF93EC0188819981009729F02A81F0
:109140003B812617370788F48B016F5F7F4F0E94A2
:10915000E3B4009761F0998388831B830A832C8191
:109160003D81232B11F4FC01108281E001C080E0DD
:10917000DF91CF911F910F910895EF92FF920F937E
:109180001F93CF93DF936115710511F480E01BC02D
:1091900041155105B9F07B01EC018C819D818A015B
:1091A000080F191FB801CE01C1DF882379F3288188
:1091B00039818C819D81B701820F931F0E94FAB57E
:1091C0001D830C8381E0DF91CF911F910F91FF9060
:1091D000EF9008950F931F93CF93DF938C01EB01D2
:1091E00088E2FB0111928A95E9F74BE050E068E0D4
:1091F00079E0CE010E940FB61B8681E090E0A0E0EE
:10920000B0E08C879D87AE87BF87F80185899689F6
:10921000A789B08D888B998BAA8BBB8B82E090E05D
:10922000A0E0B0E08C8B9D8BAE8BBF8B1CA21DA2EF
:109230001EA21FA280E090E0A8E4B4E4888F998F7A
:10924000AA8FBB8F80E090E0A8E4B4EC8C8F9D8F58
:10925000AE8FBF8F8DEC9CECACE4BEE388A399A3EA
:10926000AAA3BBA3DF91CF911F910F9108954F92B5
:109270005F926F927F928F929F92AF92BF92CF92A6
:10928000DF92EF92FF920F931F93CF93DF938C01A6
:10929000EB0184E2FB0111928A95E9F78EE10E94CD
:1092A0003B6A83E090E00E94366A0E94346A66E07E
:1092B0008EE14DD780916D1390E020916E13821B4B
:1092C000910986309105ECF38DEA9FE00E94FC55F0
:1092D000882E8DEA9FE00E94FC55982E8DEA9FE033
:1092E0000E94FC55682E8DEA9FE00E94FC55782E66
:1092F0008DEA9FE00E94FC55482E8DEA9FE00E9477
:10930000FC55582EB82CA12CB5016929072E000C4C
:10931000880B990B0E94ABAE4B015C01F801658391
:10932000768387839087D42CC12CB6016529072EBC
:10933000000C880B990B0E94ABAEF8016187728715
:1093400083879487F62CE12CB7016729072E000C40
:10935000880B990B0E94ABAEF801658776878787EB
:10936000908B118A128A138A148A84E290E0A0E01A
:10937000B0E088839983AA83BB8385899689A7896E
:10938000B08D8C839D83AE83BF8382E090E0A0E0AC
:10939000B0E088879987AA87BB87188A198A1A8AB2
:1093A0001B8AC0906702D0906802E0906902F0903A
:1093B0006A02A7019601C501B4010E94FBB020E03A
:1093C00030E048EC52E40E940AAF6C8B7D8B8E8BB0
:1093D0009F8BA7019601F80161857285838594852D
:1093E0000E94FBB020E030E048EC52E40E940AAF5B
:1093F000688F798F8A8F9B8F2091630230916402EE
:109400004091650250916602F801658576858785F1
:1094100090890E94FBB020E030E048EC52E40E94CA
:109420000AAF6C8F7D8F8E8F9F8F81E0DF91CF9100
:109430001F910F91FF90EF90DF90CF90BF90AF9072
:109440009F908F907F906F905F904F900895862FA0
:109450000C944F85862F642F0C947785862F642F6C
:109460000C94A585FC0180819181009711F00C94EA
:1094700034AA60E070E0CB010895FC018081918105
:10948000009711F00C9437AA60E070E0CB010895CA
:10949000AF92BF92CF92DF92EF92FF920F931F9302
:1094A000CF93DF93DC01CD90DC901197C114D104F0
:1094B00009F443C01496CD91DC9115972097E9F1FA
:1094C0008C0176015701BFEFAB1ABB0AF70180810F
:1094D000082E000C990B0E9475AE892B11F07501B6
:1094E000F1CF2197CC0DDD1D8881082E000C990B42
:1094F0000E9475AE892B29F0CE15DF0510F021975B
:10950000F3CFAE014F5F5F4F4E195F09D80115963B
:109510005C934E931497CE14DF0420F4B701C60178
:109520000E94E8B5D801ED91FC91119714968D91A8
:109530009C911597E80FF91F1082DF91CF911F9131
:109540000F91FF90EF90DF90CF90BF90AF90089574
:10955000FC01248135816217730748F48081918171
:10956000009729F0FC01E60FF71F8081089580E045
:109570000895EF92FF920F931F93CF93DF9361159E
:10958000710511F480E01DC08B01EC01CB010E943C
:1095900064AA0097A9F02C813D817C01E20EF31EA4
:1095A000B701CE01C3DD882369F3288139818C811D
:1095B0009D81B801820F931F0E945DAAFD82EC82FB
:1095C00081E0DF91CF911F910F91FF90EF9008956F
:1095D000CF93DF931F921F92CDB7DEB769831A82B4
:1095E00041E050E0BE016F5F7F4FC7DD0F900F90ED
:1095F000DF91CF9108956115710549F0FB0101904C
:109600000020E9F73197AF01461B570BB6CD80E03C
:109610000895FB014481558160817181AECD0F9326
:109620001F93CF93DF938C01EB01FC01808191812B
:10963000009739F06881798161157105A1F40E9464
:109640005AB488819981F801918380838A819B81B2
:10965000938382838C819D81958384831982188270
:109660001B821A820FC0F801428153812C813D81F7
:109670004217530720F30E94FAB58C819D81F801AF
:10968000958384831D821C82DF91CF911F910F915E
:109690000895CF93DF93EC0188819981009711F0B1
:1096A0000E945AB4198218821D821C821B821A825F
:1096B000DF91CF910895CF93DF93EC016115710590
:1096C00059F0FB0101900020E9F73197AF01461BEB
:1096D000570B53DD811102C0CE01DBDFCE01DF91DC
:1096E000CF910895CF93DF93EC01FB014481558125
:1096F0006081718142DD811102C0CE01CADFCE01DD
:10970000DF91CF910895EF92FF920F931F93CF9324
:10971000DF93EC018B016115710549F0CB010E94CB
:1097200064AA7C01BC01CE0101DD811103C0CE0120
:10973000B0DF07C0FD82EC82B801888199810E9468
:109740005DAACE01DF91CF911F910F91FF90EF9015
:109750000895EF92FF920F931F93CF93DF93EC0145
:109760007B018A01BA01E2DC811103C0CE0191DFE5
:1097700007C01D830C83B701888199810E94FAB5C7
:10978000CE01DF91CF911F910F91FF90EF9008953F
:10979000CF93DF93EC016115710551F0FB0101904E
:1097A0000020E9F73197AF01461B570BD2DF01C00C
:1097B00070DFCE01DF91CF910895CF93DF93EC015D
:1097C000FB018617970751F0608171816115710562
:1097D00021F044815581BDDF01C05BDFCE01DF9107
:1097E000CF910895FC01808191810C945AB4EF923D
:1097F000FF920F931F93CF93DF93CDB7DEB7A1975F
:109800000FB6F894DEBF0FBECDBF7C01CB01BA010D
:10981000F70111821082138212821582148242E0B3
:10982000420F8E010F5F1F4F0E9415AABC01C70196
:10983000AFDFA1960FB6F894DEBF0FBECDBFDF91AC
:10984000CF911F910F91FF90EF900895CF93DF93E9
:109850001F921F92CDB7DEB7FC01118210821382D6
:1098600012821582148269831A82BE016F5F7F4F54
:109870008FDF0F900F90DF91CF910895FC0111823F
:1098800010821382128215821482C9CEFC011182C9
:109890001082138212821582148235CFFC0111824C
:1098A0001082138212821582148287CFFC011182EA
:1098B000108213821282158214826115710549F09B
:1098C000FB0101900020E9F73197AF01461B570BD0
:1098D00040CF0895BF92CF92DF92EF92FF920F9305
:1098E0001F93CF93DF937C016B018A01E901241759
:1098F000350720F4812F8901C42FD82F6FEB79E031
:10990000C701D4DFD60114968D919C911597081745
:109910001907C0F48C179D0708F4EC01D601ED91EE
:10992000FC911197EC0FFD1FB08010826D917C911E
:10993000600F711FC7012CDFD601ED91FC91EC0F78
:10994000FD1FB082C701DF91CF911F910F91FF9052
:10995000EF90DF90CF90BF900895DC01ED91FC91E6
:109960000190F081E02D1994DB0114964D915C91EA
:1099700015976D917C91DC01ED91FC910280F38152
:10998000E02D1994EF92FF920F931F93CF93DF93E3
:109990008C017B01C0E0D0E0F701EC0FFD1F64916A
:1099A000662361F0D801ED91FC910190F081E02DEA
:1099B000C8011995892B11F02196EECFCE01DF91C8
:1099C000CF911F910F91FF90EF9008956115710550
:1099D00079F0FB0101900020E9F73197AF01461BB8
:1099E000570BDC01ED91FC910280F381E02D19947D
:1099F00080E090E008958F929F92AF92BF92EF9295
:109A0000FF920F931F93CF93DF93CDB7DEB7A1974C
:109A10000FB6F894DEBF0FBECDBF7C01FA01CB01BB
:109A200019A2223008F42AE08E010F5D1F4F822E0A
:109A3000912CA12CB12CBF01A50194010E9403B06F
:109A4000F901CA01015011096A3014F4605D01C0C6
:109A5000695CD8016C93232B242B252B61F7B8016B
:109A6000C701B4DFA1960FB6F894DEBF0FBECDBF1D
:109A7000DF91CF911F910F91FF90EF90BF90AF902A
:109A80009F908F900895CF92DF92EF92FF920F9365
:109A90001F93CF93DF934115510579F4DC01ED91CC
:109AA000FC910190F081E02DDF91CF911F910F91FA
:109AB000FF90EF90DF90CF9019946B01770FEE0835
:109AC000FF084A305105E9F4F7FE19C0EC016DE2D8
:109AD00044DF8C0144275527BA014C195D096E09F2
:109AE0007F092AE0CE0187DF800F911FDF91CF91A0
:109AF0001F910F91FF90EF90DF90CF9008952AE093
:109B000001C0242FB701A601DF91CF911F910F91C2
:109B1000FF90EF90DF90CF906ECF58CF1F920F92B3
:109B20000FB60F9211240BB60F922F933F934F93C2
:109B30005F936F937F938F939F93AF93BF93EF93B5
:109B4000FF9389E39DE038DAFF91EF91BF91AF91E8
:109B50009F918F917F916F915F914F913F912F9145
:109B60000F900BBE0F900FBE0F901F9018951F9275
:109B70000F920FB60F9211240BB60F922F933F93B3
:109B80004F935F936F937F938F939F93AF93BF9305
:109B9000EF93FF9389E39DE00E943685FF91EF915B
:109BA000BF91AF919F918F917F916F915F914F91F5
:109BB0003F912F910F900BBE0F900FBE0F901F90F3
:109BC00018951F920F920FB60F9211240BB60F9299
:109BD0002F933F934F935F936F937F938F939F93B5
:109BE000AF93BF93EF93FF9386ED9DE0E5D9FF918F
:109BF000EF91BF91AF919F918F917F916F915F9105
:109C00004F913F912F910F900BBE0F900FBE0F9071
:109C10001F9018951F920F920FB60F9211240BB63A
:109C20000F922F933F934F935F936F937F938F93F5
:109C30009F93AF93BF93EF93FF9386ED9DE00E94B8
:109C40003685FF91EF91BF91AF919F918F917F9159
:109C50006F915F914F913F912F910F900BBE0F909D
:109C60000FBE0F901F9018951F920F920FB60F9274
:109C700011240BB60F922F933F934F935F936F93E3
:109C80007F938F939F93AF93BF93EF93FF9383E75C
:109C90009EE092D9FF91EF91BF91AF919F918F91EB
:109CA0007F916F915F914F913F912F910F900BBEDC
:109CB0000F900FBE0F901F9018951F920F920FB626
:109CC0000F9211240BB60F922F933F934F935F93F4
:109CD0006F937F938F939F93AF93BF93EF93FF9374
:109CE00083E79EE00E943685FF91EF91BF91AF918F
:109CF0009F918F917F916F915F914F913F912F91A4
:109D00000F900BBE0F900FBE0F901F9018951F92D3
:109D10000F920FB60F9211240BB60F922F933F9311
:109D20004F935F936F937F938F939F93AF93BF9363
:109D3000EF93FF9380E19FE03FD9FF91EF91BF91B7
:109D4000AF919F918F917F916F915F914F913F91D3
:109D50002F910F900BBE0F900FBE0F901F90189574
:109D60001F920F920FB60F9211240BB60F922F93E2
:109D70003F934F935F936F937F938F939F93AF9393
:109D8000BF93EF93FF9380E19FE00E943685FF91A0
:109D9000EF91BF91AF919F918F917F916F915F9163
:109DA0004F913F912F910F900BBE0F900FBE0F90D0
:109DB0001F901895DC0180E0615098F02D91982F4C
:109DC0009227E92FEF70F0E0E258F04F249192953E
:109DD0009F70E92FF0E0E257F04FE491822F8E2739
:109DE000EBCF0895EF92FF920F931F93CF93DF93E2
:109DF0008C017B0140E065E5CDD7E70188E0E80E06
:109E0000F11C699140E0C801C5D7CE15DF05C9F73F
:109E1000DF91CF911F910F91FF90EF9008956F9276
:109E20007F928F929F92AF92BF92CF92DF92EF92EA
:109E3000FF920F931F93CF93DF93EC017B018A0175
:109E40008E819F81DAD7882389F1B7018E819F8126
:109E5000C9DF40E06EEB8E819F819CD7780168015D
:109E600089E0C80ED11CAE80BF8088E0882E912C7E
:109E7000712C66246394C5013AD781117628660C4B
:109E8000E1E08E1A9108B9F7F70171927F01EC15A4
:109E9000FD0549F78E819F81B0D7813039F468E0A4
:109EA000C80188DF91E0F8012085281390E0892F10
:109EB000DF91CF911F910F91FF90EF90DF90CF90A6
:109EC000BF90AF909F908F907F906F900895CF93A9
:109ED000DF93CDB7DEB729970FB6F894DEBF0FBE7C
:109EE000CDBFAE014F5F5F4F9ADF882389F08D8130
:109EF0008F3361F020F48F3159F489E00CC08F3535
:109F000019F08F3739F004C08BE005C08AE003C038
:109F100080E001C08CE029960FB6F894DEBF0FBE3A
:109F2000CDBFDF91CF910895BF92CF92DF92EF9294
:109F3000FF920F931F93CF93DF93EC016B018D85FD
:109F4000811104C0CE0159D7811105C01B861D8621
:109F50001C8680E05CC040E060EFCE011BD701E0D2
:109F6000E12CB12C11E0CE01C2D6F82ECE01BFD625
:109F700091E0F91203C08130B1F433C02E2D30E0EE
:109F8000F8121BC08B85181738F4FE01E20FF31F7F
:109F90008381802341F402C0811729F0F12C19300C
:109FA00058F41C8709C0FE01EE0DF11D8381802B42
:109FB0008383FF24F39409C0B12EFE01E20FF31F47
:109FC0009381802F8095892383836F2DCE01B3D613
:109FD0001F5F000F11F4E39401E087E08E1508F095
:109FE000C2CF113408F4B2CFBB86B11002C081E0F9
:109FF0008D878B81882309F4A9CFDE011396F601A2
:10A000002B968D918193CA17DB07D9F781E0DF91F9
:10A01000CF911F910F91FF90EF90DF90CF90BF9065
:10A020000895DF92EF92FF920F931F93CF93DF93E8
:10A030007C018B01D42EDC011696ED91FC911797D3
:10A04000138615861486DF011B9633961E92EA1737
:10A05000FB07E1F7C0E0B801F7018681978164DF73
:10A06000D82F882369F0DC1208C067E0C801A2DE9F
:10A07000D80117969C91891721F0CF5FDC1658F70D
:10A08000D0E08D2FDF91CF911F910F91FF90EF9036
:10A09000DF90089510926E1310926D131092170DA9
:10A0A0001092380D1092150D81E08093140D1092CE
:10A0B000EF0C61E084E10E94778561E085E10E9418
:10A0C0007785E9EBF0E080818E7F808380818D7FD2
:10A0D000808388E48093B80085E48093BC008AEE96
:10A0E00095E59093550C8093540C8BEE95E59093E9
:10A0F000530C8093520C08950F931F93CF93DF93CB
:10A10000CDB7DEB762970FB6F894DEBF0FBECDBFF6
:10A110008C01CB01F8011182108213821282158208
:10A1200014824AE0BE016F5F7F4F0E946DAABE019C
:10A130006F5F7F4FC8012CDB62960FB6F894DEBFCD
:10A140000FBECDBFDF91CF911F910F910895613266
:10A1500008F060E20E94E78E10926E1380936D13F8
:10A160000895AF92BF92CF92DF92EF92FF920F933A
:10A170001F93CF93DF93C82FD62F10928212109285
:10A18000831210928412109285121092861261E04E
:10A190000E94A58560E08C2F0E9477856D2F70E06E
:10A1A00080E090E00E942B8660E08C2F0E94A585C5
:10A1B0008BE990E00197F1F700E911E08C2F0E9404
:10A1C0004F85892B31F401501109C1F78EEF9FEFB4
:10A1D0004CC000E911E08C2F0E944F85019709F4D3
:10A1E0003FC018E2D0E800E090E9E92EFF24F394A4
:10A1F0008C2F0E944F85892B29F481E0E81AF10801
:10A20000B9F7E4CF0E9406866B017C0180E9A82E95
:10A21000BB24B3948C2F0E944F85019729F481E0D1
:10A22000A81AB108B9F7D2CF0E940686DC01CB018B
:10A230008C199D09AE09BF098997A105B10538F0B0
:10A24000E02FF0E0E658FD4E80858D2B8087D69577
:10A2500011F40F5FD0E8115039F680E090E005C0AE
:10A260000150110909F0B7CFB1CFDF91CF911F9104
:10A270000F91FF90EF90DF90CF90BF90AF90089537
:10A28000EF92FF920F931F93CF93DF93C82F8B0111
:10A290007A0183E50E943B6A6C2F8DEA9FE0F4D43B
:10A2A0000E94346A83E50E943B6AB80183E590E02E
:10A2B0000E94298FE701CE018E199F0930916D13FD
:10A2C00020916E13321729F08DEA9FE095D489937F
:10A2D000F2CF0817190729F01092881281E08093B5
:10A2E0008912DF91CF911F910F91FF90EF900C9405
:10A2F000346ACF93DF934AE050E0BC0180E19FE0F5
:10A30000C2DBEC0180E19FE00E94C3698C0F9D1FBE
:10A31000DF91CF9108951F93CF93DF931F92CDB715
:10A32000DEB7162FAE014F5F5F4F61E070E0A8DF30
:10A33000898190E002C0959587951A95E2F7817022
:10A340000F90DF91CF911F910895CF93DF93D82F76
:10A35000C62F83E50E943B6A6D2F8DEA9FE094D45F
:10A360006C2F8DEA9FE090D4DF91CF910C94346AEA
:10A37000FF920F931F93CF93DF931F92CDB7DEB75A
:10A38000182F062FF42EAE014F5F5F4F61E070E093
:10A3900077DF4981FF2049F021E030E001C0220F42
:10A3A0000A95EAF7242B298309C081E090E001C0D7
:10A3B000880F0A95EAF78095842389836981812F24
:10A3C000C4DF0F90DF91CF911F910F91FF900895FF
:10A3D0000F931F93CF93DF93EC019A01452B19F450
:10A3E0000E94FE4705C0462F50E060E070E003DBAE
:10A3F0008C01CE010E94C369800F911FDF91CF9124
:10A400001F910F910895CF93DF9342E00E94F26A6B
:10A41000EC0180E19FE00E94C3698C0F9D1FDF91DA
:10A42000CF9108958F929F92AF92BF92CF92DF9279
:10A43000EF92FF920F931F93CF93DF9300D000D042
:10A44000CDB7DEB75C0146E952E166E070E082E339
:10A4500017DF80919612909197129A838983809149
:10A460009812909199129C838B8380919A1290916B
:10A470009B129E838D83CE0101966C018AE8E82EA3
:10A4800082E1F82E8501F601619171916F01F7016A
:10A4900081909190A190B1907F01072E000C880BC4
:10A4A000990B0E94ABAEA50194010E940AAFF8017E
:10A4B00061937193819391938F01F6E9EF16F2E125
:10A4C000FF0609F726960FB6F894DEBF0FBECDBF84
:10A4D000DF91CF911F910F91FF90EF90DF90CF9080
:10A4E000BF90AF909F908F900895CF93DF93C82F28
:10A4F00080910E130E943B6A6C2F8DEA9FE0C4D3BB
:10A5000080E00E94D86963E080910E1320DE8DEA1E
:10A510009FE072D3EC018DEA9FE06ED320E030E043
:10A52000382FC9018C2B9D2BDF91CF9108950F936C
:10A530001F93CF93DF93CDB7DEB761970FB6F89433
:10A54000DEBF0FBECDBF8C01462FBE01665F7F4FC1
:10A5500068DD811105C060E070E08EEF92EC4BC0C9
:10A56000AE014F5F5F4FBE01665F7F4FC80157DC92
:10A57000882361F12A8130E0C901982F8827990F3B
:10A58000990F990F698128E0629FB00111249C0105
:10A59000262B372B8A858031E1F4688570E08F8126
:10A5A000AB01481B5109CA019695982F88279795AA
:10A5B00087950E945CB360517109207F53E0220FA0
:10A5C000331F5A95E1F7620F731F04C060E874EE01
:10A5D00001C0B901613854EE75070CF4BCCF072EE9
:10A5E000000C880B990B0E94ABAE20E030E040E0FD
:10A5F0005CE30E940AAF61960FB6F894DEBF0FBE0F
:10A60000CDBFDF91CF911F910F9108959F92AF928F
:10A61000BF92CF92DF92EF92FF920F931F93CF934F
:10A62000DF93CDB7DEB761970FB6F894DEBF0FBEEC
:10A63000CDBF8C018CE0F8018183C12CD12C2FE59A
:10A64000E22E3FE7B32E4FE1A42E5FE3952EF801F3
:10A65000848190E0C816D9060CF095C04C2DBE013F
:10A66000665F7F4FC801DDDCF8018181893038F0F9
:10A67000F82EFCE0F81728F49CE0F92E02C089E0DF
:10A68000F82E8A85803131F0BE01665F7F4FC801A8
:10A690001EDC01C08CE0F81609F471C0AE014F5FFA
:10A6A0005F4FBE01665F7F4FC801B9DB882309F4A5
:10A6B00066C08A85803109F462C08BE0F81651F0DB
:10A6C000ECE0FE1629F0FAE0FF1206C09D8205C0FC
:10A6D000BD8203C0ED8201C0AD82F8018681978101
:10A6E0008CD3BE01665F7F4FF801868197817ADB4C
:10A6F00040E06EE4F801868197814CD340E06B81A5
:10A70000F8018681978146D340E06C81F80186810B
:10A71000978140D38A85803131F040E06D81F80126
:10A720008681978137D3F8018681978166D3BE01F0
:10A73000665F7F4FF8018681978154DBF801408185
:10A7400068E48681978126D364E170E080E090E040
:10A750000E942B86F8018081882331F06AE070E046
:10A7600080E090E00E942B86F8018681978145D396
:10A77000F80181818F1508F48F2DF8018183FFEF97
:10A78000CF1ADF0A64CF61960FB6F894DEBF0FBE12
:10A79000CDBFDF91CF911F910F91FF90EF90DF9090
:10A7A000CF90BF90AF909F9008958F929F92AF925D
:10A7B000BF92CF92DF92EF92FF920F931F93CF93AE
:10A7C000DF93EC018E819F8118D340E06CEC8E8189
:10A7D0009F81E0D2488164E48E819F81DBD28A81AF
:10A7E000882309F441C0E981E950E33040F4F0E006
:10A7F000EE0FFF1FEB5CFA4F0081118102C00EEEDD
:10A8000012E08B818823F1F0888181111BC00E94A6
:10A8100087874B015C016801110FEE08FF088E81EC
:10A820009F8165D2813001F10E948787DC01CB01D5
:10A830008C199D09AE09BF0988159905AA05BB05A4
:10A8400070F312C0B801110F880B990BDF91CF91F3
:10A850001F910F91FF90EF90DF90CF90BF90AF903E
:10A860009F908F900C942B86DF91CF911F910F9129
:10A87000FF90EF90DF90CF90BF90AF909F908F9020
:10A880000895EF92FF920F931F93CF93DF93CDB76D
:10A89000DEB728970FB6F894DEBF0FBECDBF8C0190
:10A8A000DC011696ED91FC91179713861586148698
:10A8B000DF011B9633961E92EA17FB07E1F7F801BA
:10A8C00014821582EE24E394BE016F5F7F4FD8019E
:10A8D00016968D919C91179727DB882309F46DC0FC
:10A8E00067E0CE01019666DA98858913EDCFF8010D
:10A8F000808181111FC0868197817FD2BE016F5FE9
:10A900007F4FD80116968D919C9117976BDA40E096
:10A9100064EBF801868197813DD2D80116968D911E
:10A920009C911797E4D1F82EF8018681978165D222
:10A93000FF20A1F1D8011196FC9089818031C9F1E5
:10A94000BE016F5F7F4FC801C2DA8F1518F4F8019E
:10A9500081810AC08981803111F48CE005C0BE017B
:10A960006F5F7F4FC801B3DAD80111968C931197AE
:10A9700014968C9114978F5F14968C9389818832EA
:10A9800081F030F4803169F0823209F09DCF09C046
:10A990008B3339F0823409F097CF03C0F801E0829D
:10A9A000C9CFD80115968C9115978F5F15968C930A
:10A9B0008BCFBCE0BF1558F2D0CF28960FB6F894D5
:10A9C000DEBF0FBECDBFDF91CF911F910F91FF90E2
:10A9D000EF9008956F927F928F929F92AF92BF9265
:10A9E000CF92DF92EF92FF920F931F93CF93DF935B
:10A9F000CDB7DEB72C970FB6F894DEBF0FBECDBF34
:10AA00007C015B014A016FEB79E00E94564C6FEBD1
:10AA100079E0CE0107960E94564CC12CD12C35010D
:10AA20008FEF681A780A8E010F5F1F4FC814D90480
:10AA30000CF084C0F701848195818615970508F094
:10AA40007DC0B501C8010E942F8BB801CE010796C9
:10AA50000E940F4BC8010E94F24B64E170E080E05D
:10AA600090E00E942B868B859C85892B61F4B50133
:10AA7000C8010E94CD89B801CE0107960E940F4BF4
:10AA8000C8010E94F24B8B859C85892B79F060EF81
:10AA900077E08F8198850E94F1B5892BD9F4F70171
:10AAA000248135812115310569F514C064E170E018
:10AAB00080E090E00E942B86F701848195818A15C1
:10AAC0009B0520F4EFEFCE1ADE0AB0CFF5E1CF0EF2
:10AAD000D11CACCFBE01695F7F4FC7010E94094BFB
:10AAE000F2E3CF1AD108B701C8010E944E4C42E3ED
:10AAF00050E06FEF7FEFC8010E94738DC8010E9484
:10AB0000F24BDACF2230310530F46FEB79E0C70138
:10AB10000E94C84BE5CF2150310940E050E0B70119
:10AB2000C8010E946A4C0E151F0521F0B801C7012B
:10AB30000E940F4BC8010E94F24BD2CFCE01079664
:10AB40000E94F24BC7012C960FB6F894DEBF0FBEE1
:10AB5000CDBFDF91CF911F910F91FF90EF90DF90CC
:10AB6000CF90BF90AF909F908F907F906F900895FF
:10AB700085ED8093BC008091BC0084FDFCCF1092D9
:10AB8000150D08954091760C262F30E0240F311DCD
:10AB900021323105DCF42091150D2430C9F4FC017B
:10ABA00080E090E0861758F43091760C2191DC011A
:10ABB000AA5AB34FA30FB11D2C930196F3CF8091E6
:10ABC000760C680F6093760C80E0089581E008951C
:10ABD00082E00895089508950895E0916E1380919C
:10ABE0006D13E81730F4F0E0E159FC4E808190E0FD
:10ABF00008958FEF9FEF089590916E1380916D13DC
:10AC0000981750F4E92FF0E0E159FC4E208130E034
:10AC10009F5F90936E1302C02FEF3FEFC90108951D
:10AC200080916D1390E020916E13821B910908951D
:10AC3000CF92DF92EF92FF920F931F93CF93DF9308
:10AC40007C01CB018A012091160D222389F0EB01B2
:10AC50006B01C40ED51ECC15DD0561F06991D701DD
:10AC6000ED91FC910190F081E02DC7011995F3CF92
:10AC7000642F88DFC801DF91CF911F910F91FF9062
:10AC8000EF90DF90CF900895CF93DF931F92CDB7D1
:10AC9000DEB769832091160D2223D1F02091380D63
:10ACA000203240F021E030E0FC013383228380E059
:10ACB00090E014C08091170DE82FF0E0E85EF24FAD
:10ACC000998190838F5F8093170D8093380D04C016
:10ACD00061E0CE01019656DF81E090E00F90DF91B8
:10ACE000CF91089580E090E008950C945AB4FC014F
:10ACF00090810180F281E02DF8948181892B8183FC
:10AD00002281892F809528232283A7E0B0E0119724
:10AD1000F1F7218182238183A3E2B0E01197F1F75B
:10AD200080817894EFECF0E03197F1F7982381E09F
:10AD300009F480E00895FC0190810180F281E02D0A
:10AD4000892F809560FF12C0F8942281822382832C
:10AD50008181892B8183A3E2B0E01197F1F7828191
:10AD6000982B9283789487ED90E011C0F89422811B
:10AD7000822382838181892B8183AFEFB0E0119799
:10AD8000F1F78281982B928378948FE090E001977D
:10AD9000F1F70895DF92EF92FF920F931F93CF93F5
:10ADA000DF93EC01D62EE42E08E010E0FF24F394AC
:10ADB00061E08D2D8F2109F460E0CE01BCDFFF0C36
:10ADC00001501109A9F7E11010C0F894E981FA8146
:10ADD00091818881809589238183E981FA8192819B
:10ADE00088818095892382837894DF91CF911F9108
:10ADF0000F91FF90EF90DF900895DC012C91119658
:10AE0000ED91FC911297F8948181922F909589236E
:10AE1000818378948DE743E050E0815021F1DA019D
:10AE20001197F1F730813223C1F3F894828189239D
:10AE300082838181822B81837894ABE7B7E011977D
:10AE4000F1F7F89481819823918383E191E0019750
:10AE5000F1F78081282381E009F080E07894E3E62F
:10AE6000F6E03197F1F708951F93CF93DF93EC014C
:10AE7000162F60E0812F0E94A585612F70E0FB01F5
:10AE8000E05BFC4EE491E883FB01E65FFC4EE4915D
:10AE9000F0E0EE0FFF1FE051FD4E859194919A83F3
:10AEA00089831B861D861C86FE013B962396129283
:10AEB000EC17FD07E1F7DF91CF911F9108951F93E4
:10AEC000CF93DF93EC01162F8C810E943B6A6B8538
:10AED000812F862B90E00E94366ADF91CF911F91DF
:10AEE0000C94346A0F931F93CF938C01C62FE7DF26
:10AEF0006C2F6460C801E3DF6C2F6B7FC801DFDF5C
:10AF000083EC90E00197F1F7CF911F910F91089595
:10AF10000F931F93CF938C01C62F607F6160E2DF98
:10AF200080E1C89FB00111246160C801DBDF81E0CE
:10AF300090E0CF911F910F9108951F920F920FB63D
:10AF40000F9211240BB60F922F933F934F935F9361
:10AF50006F937F938F939F93AF93BF93EF93FF93E1
:10AF60008091BA0F0E944F852091BD0F3091BE0F86
:10AF70002F5F3F4F3093BE0F2093BD0F9091BC0FBA
:10AF8000953618F096E09093B90F9091B90F9430E0
:10AF9000C9F128F4923069F09330D1F05EC0953059
:10AFA00009F451C0963009F058C091E0909389108F
:10AFB00051C0811152C02091BD0F3091BE0F243677
:10AFC000310508F442C0109289101092BC0F1CC0C9
:10AFD000813009F042C0E091BC0F91E09E0F909348
:10AFE000BC0FF0E02091BD0F3091BE0FEE0FFF1FA0
:10AFF000E154F04F318320831092BE0F1092BD0FA9
:10B0000094E029C0811117C0E091BC0F91E09E0F20
:10B010009093BC0FF0E02091BD0F3091BE0FEE0F6A
:10B02000FF1FE154F04F318320831092BE0F109226
:10B03000BD0F93E010C02091BD0F3091BE0F25369B
:10B04000310558F007C0811108C01092BE0F109250
:10B05000BD0F03C095E09093B90F9091BB0F99235A
:10B0600029F0811102C02F9A01C02F98FF91EF9112
:10B07000BF91AF919F918F917F916F915F914F9110
:10B080003F912F910F900BBE0F900FBE0F901F900E
:10B090001895CF92DF92EF92FF92CF93DF93EC015E
:10B0A000072E000C880B990B0E94ABAE6B017C0144
:10B0B00020E030E040E45FE30E940AAF20E030E0AF
:10B0C00048E452E40E94FBB00E9494B1C617D7072F
:10B0D000D4F020E030E040EA5FE3C701B6010E940F
:10B0E0000AAF20E030E048E452E40E94FBB020E0E8
:10B0F00030E040E85FE30E9435B00E9494B121E067
:10B100006C177D070CF420E0822F90E0DF91CF9147
:10B11000FF90EF90DF90CF9008950F931F93CF9300
:10B12000DF93082F60E476E080E19FE00E948D4D80
:10B13000C7E0D0E010E0B8010C2E02C0759567950D
:10B140000A94E2F76170772742E050E080E19FE0E7
:10B150000E94434D219778F7DF91CF911F910F9176
:10B1600008951F920F920FB60F9211240BB60F92F3
:10B170002F933F934F935F936F937F938F939F93FF
:10B18000AF93BF93EF93FF938091B900887F803690
:10B1900009F49CC068F5883209F45BC090F48031F2
:10B1A00009F454C038F4882309F4F6C0883009F44F
:10B1B0004DC0F5C0883109F44CC0803209F45DC03F
:10B1C000EEC0803409F468C048F4803309F455C0F7
:10B1D000883309F0E4C08093130DD8C0803509F49A
:10B1E0004FC0883509F45DC0883409F0D8C0D6C096
:10B1F000883909F4C7C0A8F4883709F467C038F45F
:10B20000883609F463C0803709F460C0C8C0883844
:10B2100009F4B8C0803909F45FC0803809F0BFC0B4
:10B220005BC0803B09F486C038F4803A09F466C0FC
:10B23000883A09F47FC0B3C0803C09F4A7C0883CB9
:10B2400009F4A4C0883B09F48AC0A9C08091F00C1D
:10B2500010C09091120D8091110D981770F5E0912A
:10B26000120D81E08E0F8093120DF0E0EF50F34F3E
:10B2700080818093BB0085EC86C08093130D8EC0C7
:10B28000E091120D81E08E0F8093120D8091BB0032
:10B29000F0E0EF50F34F80839091120D8091110DEB
:10B2A0006EC0E091120D81E08E0F8093120D80919F
:10B2B000BB00F0E0EF50F34F80838091140D8111BB
:10B2C0006DC081E08093EF0C84EA61C083E08093DD
:10B2D000150D1092980CCFCF8091980C803208F009
:10B2E00051C0E091980C81E08E0F8093980C809172
:10B2F000BB00F0E0E858F34F8083BDCF85EC80932E
:10B30000BC001092150D8091980C803230F4E091C1
:10B31000980CF0E0E858F34F10826091980C70E0C0
:10B32000E091520CF091530C88E79CE01995109233
:10B33000980C35C084E08093150D1092770C109214
:10B34000760CE091540CF091550C19958091760C87
:10B35000811105C081E08093760C1092560CE0912B
:10B36000770C81E08E0F8093770CF0E0EA5AF34F70
:10B3700080818093BB009091770C8091760C981718
:10B3800008F479CF85E88093BC0009C085EC8093F0
:10B39000BC001092150D03C01092130DE9DBFF9154
:10B3A000EF91BF91AF919F918F917F916F915F913D
:10B3B0004F913F912F910F900BBE0F900FBE0F90AA
:10B3C0001F9018950895EBE8F0E114A215A216A2BB
:10B3D00017A210A611A612A613A681E084A729E140
:10B3E00030E036A725A787A780E090E0A0EAB0E488
:10B3F00080AB91ABA2ABB3AB80E090E0A8EAB1E444
:10B4000084AB95ABA6ABB7AB809325029093260295
:10B41000A0932702B093280280E090E0A0E8BFE369
:10B420008093D5109093D610A093D710B093D810D6
:10B430008093210290932202A0932302B0932402CE
:10B4400010920211109201118BE090E09093041180
:10B450008093031190932A028093290210923A0C50
:10B460001092390C80E090E00C94836EEF92FF9282
:10B470000F931F93CF93DF93CDB7DEB768970FB6C7
:10B48000F894DEBF0FBECDBF8C0168ED7BE0CE012E
:10B490000D960E94564C60E179E0CE0143960E94E1
:10B4A000564C61EF7FE0C8010E94464CBE016D5EC4
:10B4B0007F4FC8010E94094B68EE7FE0C8010E94DF
:10B4C000B94A8AE1E82E81E1F82EF701608170E047
:10B4D000CE0101960E947C50BE016F5F7F4FCE016E
:10B4E00007960E944E4CBE01635F7F4FCE010796C8
:10B4F0000E94724BBC01C8010E94094BCE01079605
:10B500000E94F24BCE0101960E94F24B6BED7FE060
:10B51000C8010E94B94AF7016181062E000C770B21
:10B52000CE0101960E947C50BE016F5F7F4FCE011D
:10B5300007960E944E4CBE01635F7F4FCE01079677
:10B540000E94724BBC01C8010E94094BCE010796B4
:10B550000E94F24BCE0101960E94F24B61ED7FE01A
:10B56000C8010E94B94AF7016281062E000C770BD0
:10B57000CE0101960E947C50BE016F5F7F4FCE01CD
:10B5800007960E944E4CBE01635F7F4FCE01079627
:10B590000E94724BBC01C8010E94094BCE01079664
:10B5A0000E94F24BCE0101960E94F24B69EC7FE0C3
:10B5B000C8010E94B94AF70163817481CE010196E6
:10B5C0000E947C50BE016F5F7F4FCE0107960E94A4
:10B5D0004E4CBE016D5E7F4FCE0107960E94724BAE
:10B5E000BC01C8010E94094BCE0107960E94F24B94
:10B5F000CE0101960E94F24B62EB7FE0C8010E94EF
:10B60000B94AF70165817681CE0101960E947C508E
:10B61000BE016F5F7F4FCE0107960E944E4CBE0168
:10B62000635F7F4FCE0107960E94724BBC01C80139
:10B630000E94094BCE0107960E94F24BCE01019663
:10B640000E94F24B69EA7FE0C8010E94B94AF70103
:10B650006781062E000C770B6F5F7F4FCE0101963E
:10B660000E947C50BE016F5F7F4FCE0107960E9403
:10B670004E4CBE01635F7F4FCE0107960E94724B16
:10B68000BC01C8010E94094BCE0107960E94F24BF3
:10B69000CE0101960E94F24B6EE97FE0C8010E9444
:10B6A000B94AF7016085062E000C770BCE01019692
:10B6B0000E947C50BE016F5F7F4FC8010E94094B02
:10B6C000CE0101960E94F24BCE0143960E94F24BAE
:10B6D000CE010D960E94F24BC80168960FB6F89401
:10B6E000DEBF0FBECDBFDF91CF911F910F91FF90B5
:10B6F000EF9008950F931F9360E0809102020E94E3
:10B70000778583E090E00197F1F761E08091020294
:10B710000E94778583E290E00197F1F760E08091E5
:10B7200002020E9477858091000290910102992780
:10B73000FC01E05BFC4E6491FC01E65FFC4EE49191
:10B74000F0E0EE0FFF1FE051FD4E8591949100E473
:10B7500012E42FE030E0462F0E94079A6115710530
:10B760008105910549F0DC01CB010196A11DB11DB8
:10B77000BC01CD019F7003C060E070E0CB010E946E
:10B78000A9AE20E030E048EC52E40E94FBB02091EA
:10B79000990C30919A0C40919B0C50919C0C0E94FA
:10B7A0000AAF20E030E44CE156E40E94FBB020E018
:10B7B00030E040E05FE30E940AAF1F910F910895CF
:10B7C00023E333E948E853E40E94FBB020E030E093
:10B7D00040E85FE30E9435B00E94F3B226E636EA05
:10B7E00045EA53E40E940AAF6093990C70939A0C57
:10B7F00080939B0C90939C0C0895CF92DF92EF92D4
:10B80000FF9278DF6B017C0120E030E040E050E403
:10B810000E94EAB118161CF46DDF6B017C0120E078
:10B8200030E040E050E4C701B6010E94EAB11816CA
:10B830001CF460DF6B017C0120E030E040E050E46C
:10B84000C701B6010E94EAB118161CF453DF6B0160
:10B850007C0120E030E040E050E4C701B6010E94E6
:10B86000EAB118162CF4FF90EF90DF90CF9042CF02
:10B87000C701B601FF90EF90DF90CF900895BF927F
:10B88000CF92DF92EF92FF920F931F93CF93DF93AC
:10B89000CDB7DEB762970FB6F894DEBF0FBECDBF4F
:10B8A0008C016B0168ED7BE0CE010D960E94564C39
:10B8B00067E370E1C8010E94464C76012FEFE21A5F
:10B8C000F20AB701CE0101960E947C50BE016F5F63
:10B8D0007F4FCE0107960E944E4C66E177E0CE0185
:10B8E00007960E945B4BBC01C8010E94094BCE0128
:10B8F00007960E94F24BCE0101960E94F24B8AE01D
:10B90000B82EBE9CC001BF9C900D1124FC01E65EC8
:10B91000FE4E7F018081082E000C990B0E94DAB543
:10B92000892B09F4B2C0B701CE0101960E94564C92
:10B93000BE016F5F7F4FCE0107960E944E4C69EFAC
:10B940007AE0CE0107960E945B4BBC01C8010E94C1
:10B95000094BCE0107960E94F24BCE0101960E9440
:10B96000F24BBC9CC001BD9C900D11249C01265E35
:10B970003E4E7901F9016685062E000C770BCE014B
:10B9800001960E947C50BE016F5F7F4FCE010796EB
:10B990000E944E4C63E179E0CE0107960E945B4B1A
:10B9A000BE01635F7F4F0E94724BBC01C8010E94C1
:10B9B000094BCE0107960E94F24BCE0101960E94E0
:10B9C000F24B60E370E1C8010E94B94AF701678554
:10B9D000062E000C770BCE0101960E947C50BE0112
:10B9E0006F5F7F4FCE0107960E944E4CBE01635F92
:10B9F0007F4FCE0107960E94724BBC01C8010E9486
:10BA0000094BCE0107960E94F24BCE0101960E948F
:10BA1000F24B6AE270E1C8010E94B94AF7016089FD
:10BA20007189CE0101960E947C50BE016F5F7F4FED
:10BA3000CE0107960E944E4CBE01635F7F4FCE0140
:10BA400007960E94724BBC01C8010E94094BCE01AF
:10BA500007960E94F24BCE0101960E94F24B65E2DE
:10BA600070E1C8010E94B94AF70162897389CE0169
:10BA700001960E947C50BE016F5F7F4FC8010E94FB
:10BA8000094BCE0101960E94F24BCE010D960E9409
:10BA9000F24BC80162960FB6F894DEBF0FBECDBF61
:10BAA000DF91CF911F910F91FF90EF90DF90CF909A
:10BAB000BF9008950F931F93CF93DF93CDB7DEB759
:10BAC0002C970FB6F894DEBF0FBECDBF8C016FEB85
:10BAD00079E08EE392E10E94C84B0830110509F02D
:10BAE000DFC066E271E1CE0101960E94464C44E659
:10BAF00050E06FEF7FEFCE0101960E94BB8FCE0129
:10BB000001960E94F24B6AE171E1CE0101960E941A
:10BB1000464C44E650E060E070E0CE0101960E94A1
:10BB2000738DCE0101960E94F24B89E39DE00E9445
:10BB30004A484CE251E061E070E0CE0101960E947B
:10BB4000EA54809197138823D1F065E179E0CE0122
:10BB500007960E94564CBE016F5F7F4FCE0107963D
:10BB60000E94724B61E277E00E945B4BBC0180E176
:10BB70009FE00E94C769CE0107960E94F24B6DECD0
:10BB800078E0CE0107960E94564CBE01695F7F4F58
:10BB9000CE0101960E940685182FCE0107960E94BD
:10BBA000F24B112309F4A5C268E179E08EE392E13A
:10BBB0000E94C84B88E090E090930A0C8093090C97
:10BBC0000E943435182F6DE071E1CE0107960E9476
:10BBD000464C44E650E060E070E0CE0107960E94DB
:10BBE000738DCE0107960E94F24B89E39DE00E947F
:10BBF0004A4848E552E061E070E0CE0107960E94B5
:10BC0000EA54BE01695F7F4FCE0101960E940F4B3F
:10BC1000CE0107960E94F24B809197138823D1F0B2
:10BC200065E179E0CE0107960E94564CBE016F5F38
:10BC30007F4FCE0107960E94724B61E277E00E942F
:10BC40005B4BBC0180E19FE00E94C769CE01079673
:10BC50000E94F24B60E476E0CE0107960E94564CBB
:10BC6000BE01695F7F4FCE0101960E940685082FB5
:10BC7000CE0107960E94F24B002309F43AC26DE10F
:10BC800079E08EE392E10E94C84B0E94343588230C
:10BC900009F42FC2112309F42CC260E071E1F9C04C
:10BCA000093F2FEF120709F00BC16FEE70E1CE01D3
:10BCB00001960E94464C44E650E06FEF7FEFCE01C4
:10BCC00001960E94BB8FCE0101960E94F24B61EE5D
:10BCD00070E1CE0101960E94464C44E650E060E0DF
:10BCE00070E0CE0101960E94738DCE0101960E94F4
:10BCF000F24B89E39DE00E944A484CE251E064E047
:10BD000070E0CE0101960E94EA5480919713882337
:10BD1000D1F065E179E0CE0107960E94564CBE0154
:10BD20006F5F7F4FCE0107960E94724B61E277E012
:10BD30000E945B4BBC0180E19FE00E94C769CE017D
:10BD400007960E94F24B60E070E0CE0101960E94DF
:10BD5000A84A082E000C990BC0970A9708F0CCC18E
:10BD600063E279E0CE0107960E94564CBE016F5FF8
:10BD70007F4FCE0107960E94724BBC018EE392E189
:10BD80000E94DD4BCE0107960E94F24B89EF9FEF98
:10BD900090930A0C8093090C0E943435182F63EDA0
:10BDA00070E1CE0107960E94464C44E650E060E008
:10BDB00070E0CE0107960E94738DCE0107960E9417
:10BDC000F24B89E39DE00E944A4848E552E065E075
:10BDD00070E0CE0107960E94EA54BE01695F7F4F72
:10BDE000CE0101960E940F4BCE0107960E94F24BA6
:10BDF000809197138823D1F065E179E0CE01079611
:10BE00000E94564CBE016F5F7F4FCE0107960E9485
:10BE1000724B61E277E00E945B4BBC0180E19FE0E6
:10BE20000E94C769CE0107960E94F24B60E070E065
:10BE3000CE0101960E94A84A082E000C990BC097CB
:10BE40000A9708F059C168E279E0CE0107960E948E
:10BE5000564CBE016F5F7F4FCE0107960E94724B1A
:10BE6000BC018EE392E10E94DD4BCE0107960E9459
:10BE7000F24B89EF9FEF90930A0C8093090C0E947C
:10BE80003435882309F438C1112309F435C166EC2F
:10BE900070E1CE0107960E94464C44E650E060E017
:10BEA00070E0CE0107960E94738DCE0107960E9426
:10BEB000F24B6FEB79E08EE392E10E94C84B14C124
:10BEC00065EB70E1CE0101960E94464C44E650E0DD
:10BED0006FEF7FEFCE0101960E94BB8FCE010196DE
:10BEE0000E94F24B6FEB79E08EE392E10E94C84B27
:10BEF000053F8FEF180749F46DE678E08EE392E195
:10BF00000E94C84B6BEA70E126C0063F2FEF120774
:10BF100049F467E678E08EE392E10E94C84B61EA5B
:10BF200070E119C0013F8FEF180749F461E778E02D
:10BF30008EE392E10E94C84B62E970E10CC0023FBF
:10BF40002FEF1207B9F46DE279E08EE392E10E94DF
:10BF5000C84B62E870E1CE0101960E94464C44E66F
:10BF600050E06FEF7FEFCE0101960E94738DCE01FE
:10BF70000196C5C00230110509F07EC066E770E188
:10BF8000CE0101960E94464C44E650E06FEF7FEFF1
:10BF9000CE0101960E94BB8FCE0101960E94F24B0A
:10BFA00066E670E1CE0101960E94464C44E650E000
:10BFB0006FEF7FEFCE0101960E94738DCE01019647
:10BFC0000E94F24B44EF51E066E070E0CE01019632
:10BFD0000E94EA54BE016F5F7F4F8EE392E10E94A0
:10BFE0000F4BCE0101960E94F24B8091421290912C
:10BFF0004312059708F486C060E070E08EE392E19A
:10C000000E94A84A082E000C990BC0970A9708F0C6
:10C0100079C08EE392E10E943D4A613523EC7207BC
:10C02000810591050CF46EC00E94ABAE20E030E0BB
:10C0300048EC52E40E94FBB0AB01BC0122E0CE010F
:10C0400007960E94F74B6EE478E0CE0101960E94BD
:10C05000564CBE01695F7F4FCE0101960E94724B24
:10C06000BC018EE392E10E94DD4BCE0101960E945D
:10C07000F24BCE01079643C06FE470E1CE0101960A
:10C080000E94464C44E650E06FEF7FEFCE010196F0
:10C090000E94738DCE0101960E94F24B6FEB79E006
:10C0A0008EE392E10E94C84B0B3E8FEF180709F414
:10C0B00065C08091421290914312892BE1F55EC0D8
:10C0C00068EC70E080E090E00E942B8669E370E10C
:10C0D000CE0101960E94464C44EF51E06FEF7FEF96
:10C0E000CE0101960E94738DCE0101960E94F24B03
:10C0F00045C069EF70E1CDCE6FEB70E1CACE0E9412
:10C10000F24BD7CF68E570E1CE0101960E94464C14
:10C1100048EE53E06FEF7FEFCE0101960E94738DE2
:10C12000CE0101960E94F24B6FEB79E08EE392E133
:10C130000E94C84BBECF0E943435882309F268ECB8
:10C1400070E080E090E00E942B8665E470E1CE0113
:10C1500001960E94464C44EF51E06FEF7FEFCE0115
:10C1600001960E94738DCE0101960E94F24B1093AE
:10C170000A0C0093090CC8010E94D70A2C960FB62E
:10C18000F894DEBF0FBECDBFDF91CF911F910F910D
:10C1900008956F927F928F929F92AF92BF92CF92AB
:10C1A000DF92EF92FF920F931F93CF93DF93CDB760
:10C1B000DEB768970FB6F894DEBF0FBECDBF6C0137
:10C1C0008091011190910211019731F06FEB79E0AC
:10C1D000C6010E94564C46C169E379E0CE010D9636
:10C1E0000E94564CBE01635F7F4F89E39DE00E9431
:10C1F000B44C6CE271E080E090E00E942B86CE01AE
:10C2000043960E94BA7564E670E080E090E00E9478
:10C210002B86E12CF12C85E0A82EB12C9AE0892EFA
:10C22000912C64E479E0CE0101960E94564C8F89EE
:10C23000988D892B69F06B887C8869817A81C3012C
:10C240000E941EB6009721F08C010619170902C042
:10C250000FEF1FEFCE0101960E94F24BA8014F5F36
:10C260005F4FBE016D5E7F4FCE0101960E94273F5A
:10C27000BE016F5F7F4FCE010D960E940F4BCE0126
:10C2800001960E94F24B89899A89892B69F060E0B6
:10C2900070E0CE010D960E94A84A082E000C990B62
:10C2A000C0970A9708F4C7C010E065E170E1CE01BD
:10C2B00001960E94464C44E150E06FEF7FEFCE01C3
:10C2C00001960E946090CE0101960E94F24B8FEF82
:10C2D000E81AF80A62E370E080E090E00E942B86A2
:10C2E000C701B5010E945CB3019771F5CE010196BB
:10C2F0000E9471748D819E81892B59F0BE016F5F00
:10C300007F4F8EE392E10E94DD4B0E94837E11E01D
:10C3100017C084E1E816F1049CF0C701B4010E9443
:10C320005CB3892B69F4BE01635F7F4F89E39DE0B5
:10C330000E94B44C68EC70E080E090E00E942B8694
:10C34000CE0101960E94F24BCE0101960E94BA7571
:10C35000BE016F5F7F4FCE0143960E940F4BCE010F
:10C3600001960E94F24B62E370E080E090E00E9450
:10C370002B8684E6E816F10419F0112309F451CF55
:10C38000809197138823F1F061E179E0CE01019665
:10C390000E94564CBE01635F7F4FCE0101960E9402
:10C3A000724BBC01CE0107960E944E4CCE010796FF
:10C3B0000E940A71CE0107960E94F24BCE010196AF
:10C3C0000E94F24B89899A89892B61F060E070E0C4
:10C3D000CE010D960E94A84A082E000C990BC0971A
:10C3E0000A9730F066E479E0C6010E94564C1AC004
:10C3F00062E579E0CE0101960E94564CBE016F5F66
:10C400007F4FCE010D960E940685182FCE01019612
:10C410000E94F24B1111E6CFBE01635F7F4FC60150
:10C420000E943E4CCE0143960E94F24BCE010D96E7
:10C430000E94F24B17C062E579E0CE0101960E949E
:10C44000564CBE016F5F7F4FCE010D960E94068550
:10C45000082FCE0101960E94F24B11E0002309F44F
:10C4600024CF22CFC60168960FB6F894DEBF0FBE68
:10C47000CDBFDF91CF911F910F91FF90EF90DF9093
:10C48000CF90BF90AF909F908F907F906F900895C6
:10C49000AF92BF92CF92DF92EF92FF920F931F93D2
:10C4A000CF93DF93CDB7DEB72C970FB6F894DEBFEE
:10C4B0000FBECDBF8091450C811102C00E94DC3EB1
:10C4C0008091050290910602029751F080910F0C25
:10C4D0009091100C009709F48DC1039709F48AC15B
:10C4E0006FE571E18AE192E10E94834B6AE172E1BA
:10C4F000CE0101960E944E4C44E150E060E070E0B5
:10C50000CE0101960E94BB8FCE0101960E94F24B94
:10C5100060E571E18AE192E10E94834B6AE172E198
:10C52000CE0101960E944E4C44E150E06FEF7FEF48
:10C53000CE0101960E94738DCE0101960E94F24BAE
:10C5400087E00E9475528C0186E00E947552BC0102
:10C5500080E090E00E94A9AE2AE037ED43EA5CE378
:10C560000E940AAF23E333E948E853E40E9434B061
:10C570006B017C0184E0A82EB12C20E030E048EC77
:10C5800052E4C701B6010E94EAB1181614F581E021
:10C59000A81AB10809F4F4C064E670E080E090E005
:10C5A0000E942B8686E00E947552BC0180E090E0DC
:10C5B0000E94A9AE2AE037ED43EA5CE30E940AAF8D
:10C5C00023E333E948E853E40E9434B06B017C0173
:10C5D000D4CFB80180E090E00E94A9AE2AE037ED08
:10C5E00043EA5CE30E940AAF23E333E948E853E4FB
:10C5F0000E9434B0AB01BC0121E0CE0101960E9443
:10C60000F74B6CE679E0CE0107960E94564CBE01CE
:10C610006F5F7F4FCE0107960E94724BBC0180E294
:10C6200092E10E94DD4BCE0107960E94F24BCE01B3
:10C6300001960E94F24B60E272E1CE0101960E94E7
:10C640004E4C42E350E06FEF7FEFCE0101960E9427
:10C65000738DCE0101960E94F24B66E779E0CE0120
:10C6600001960E94564CCE0101960E94EF8DCE019C
:10C6700001960E94F24B65E779E080E292E10E9428
:10C68000FB4A21E0B701A601CE0101960E94F74BBB
:10C690006DE07AE0CE0107960E94564CBE016F5FB6
:10C6A0007F4FCE0107960E94724BBC0186E292E159
:10C6B0000E94DD4BCE0107960E94F24BCE010196FF
:10C6C0000E94F24B68ED7BE0CE0101960E94564C31
:10C6D00066E272E1CE0101960E94724BBC018AE1D2
:10C6E00092E10E94DD4BCE0101960E94F24B6AE17D
:10C6F00072E1CE0101960E944E4C4AE050E060E0AB
:10C7000070E0CE0101960E946090CE0101960E94D9
:10C71000F24B66E779E0CE0101960E94564CCE01BD
:10C7200001960E94EF8DCE0101960E94F24B65E7C3
:10C7300079E086E292E10E94FB4A66E272E1CE0174
:10C7400001960E944E4C68ED7BE0CE0101960E945E
:10C750005B4B60E272E10E94724BBC0180E292E1AD
:10C760000E94DD4BCE0101960E94F24B80910F0C8E
:10C770009091100C039709F006C184E090E0FFC08F
:10C7800065E471E18AE192E10E94834B6AE172E122
:10C79000CE0101960E944E4C4AE050E060E070E00D
:10C7A000CE0101960E94BB8FCE0101960E94F24BF2
:10C7B0006AE579E0CE0101960E94564C6AE172E189
:10C7C000CE0101960E94724BBC0180E292E10E9470
:10C7D000DD4BCE0101960E94F24B80910F0C90919F
:10C7E000100C049721F41092100C10920F0C81E0A1
:10C7F00090E018C186ED9DE00E940D8E64E670E029
:10C8000080E090E00E942B8665E871E18AE192E188
:10C810000E94834B6AE172E1CE0101960E944E4C68
:10C8200044E150E060E070E0CE0101960E94BB8FD1
:10C83000CE0101960E94F24B66E771E18AE192E136
:10C840000E94834B6AE172E1CE0101960E944E4C38
:10C8500044E150E06FEF7FEFCE0101960E94738DAF
:10C86000CE0101960E94F24B8CE40E942B8E6B014C
:10C870007C0104E010E0A7019601C701B6010E9407
:10C8800034B3811192C021E0B701A601CE01079611
:10C890000E94F74B6CE679E0CE0101960E94564C5F
:10C8A000BE01695F7F4FCE0101960E94724BBC01B1
:10C8B00080E292E10E94DD4BCE0101960E94F24B94
:10C8C000CE0107960E94F24B60E272E1CE01019622
:10C8D0000E944E4C42E350E06FEF7FEFCE01019695
:10C8E0000E94738DCE0101960E94F24B66E779E0BB
:10C8F000CE0101960E94564CCE0101960E94EF8D0A
:10C90000CE0101960E94F24B65E779E080E292E168
:10C910000E94FB4A86E60E942B8E6B017C0104E09C
:10C9200010E0A7019601C701B6010E9434B3882325
:10C9300009F47DC00150110909F0E2C06FEB79E004
:10C9400086E292E10E94C84B66E272E1CE01019656
:10C950000E944E4C68ED7BE0CE0101960E945B4B3D
:10C9600060E272E10E94724BBC0180E292E10E949F
:10C97000DD4BCE0101960E94F24B83E090E0909354
:10C98000100C80930F0C64E670E080E090E00E9451
:10C990002B868091450C882309F4BEC060E273E0C9
:10C9A00080E090E00E942B86B7C00150110909F089
:10C9B0009BC06BE671E18AE192E10E94834B6AE1E0
:10C9C00072E1CE0101960E944E4C4AE050E060E0D8
:10C9D00070E0CE0101960E94BB8FCE0101960E94AD
:10C9E000F24B6AE579E0CE0101960E94564C6AE16D
:10C9F00072E1CE0101960E94724BBC0180E292E18D
:10CA00000E94DD4BCE0101960E94F24B80910F0CEB
:10CA10009091100C039721F41092100C10920F0CAF
:10CA200082E090E09093060280930502ACCF21E073
:10CA3000B701A601CE0107960E94F74B6DE07AE0A0
:10CA4000CE0101960E94564CBE01695F7F4FCE0118
:10CA500001960E94724BBC0186E292E10E94DD4B7E
:10CA6000CE0101960E94F24BCE0107960E94F24B36
:10CA700068ED7BE0CE0101960E94564C66E272E1C1
:10CA8000CE0101960E94724BBC018AE192E10E94A4
:10CA9000DD4BCE0101960E94F24B6AE172E1CE01BC
:10CAA00001960E944E4C4AE050E06FEF7FEFCE01BE
:10CAB00001960E946090CE0101960E94F24B66E7BB
:10CAC00079E0CE0101960E94564CCE0101960E945B
:10CAD000EF8DCE0101960E94F24B65E779E086E288
:10CAE00092E10E94FB4A30CF68EC70E080E090E079
:10CAF0000E942B868CE40E942B8E6B017C01BBCEA6
:10CB000068EC70E080E090E00E942B8686E60E9450
:10CB10002B8E6B017C0105CF2C960FB6F894DEBFEF
:10CB20000FBECDBFDF91CF911F910F91FF90EF907E
:10CB3000DF90CF90BF90AF9008952F923F924F9289
:10CB40005F926F927F928F929F92AF92BF92CF929D
:10CB5000DF92EF92FF920F931F93CF93DF93CDB7A6
:10CB6000DEB7C554D1090FB6F894DEBF0FBECDBFF6
:10CB70002B013C0169017A010E94878722966CAFE4
:10CB80007DAF8EAF9FAF229720E9421621E052067B
:10CB90006104710434F090E9492E55245394612CBA
:10CBA000712C30E1C31637E2D306E104F1042CF412
:10CBB000CDA6DEA6EFA6F8AA08C080E197E2A0E025
:10CBC000B0E08DA79EA7AFA7B8AB8091450C882396
:10CBD00021F0CDA6DEA6EFA6F8AA22966CAD7DAD1B
:10CBE0008EAD9FAD229728EE33E040E050E00E94EA
:10CBF000D7AF26962CAF3DAF4EAF5FAF269791E0F3
:10CC00009DAB19A61AA61BA61CA68E01035F1F4F7B
:10CC1000CC24DD247601C418D508E608F708C9AA93
:10CC2000DAAAEBAAFCAAC9A4DAA4EBA4FCA42DA559
:10CC30003EA54FA558A9C216D306E406F5060CF08A
:10CC40002BC3C701B6010E94ABAE20E030E04AE73B
:10CC500054E40E94FBB0AB01BC0123E0C8010E9478
:10CC6000F74BB8018AE192E10E940F4BC8010E9484
:10CC7000F24B8DA59EA5AFA5B8A90A97A105B10550
:10CC800084F426964CAD5DAD6EAD7FAD2697C801A0
:10CC900038D4B8018AE192E10E940F4BC8010E948A
:10CCA000F24BCE0101960E94125268E371E180E2DC
:10CCB00092E10E94834BDE0111961D01C12CD12C03
:10CCC0007601F10181909190A190B1901F01A50191
:10CCD0009401C501B4010E940AAF9B01AC01C701D8
:10CCE000B6010E9435B06B017C0123E0B501A401BF
:10CCF000C8010E94F74BB801CE0143960E944E4CEA
:10CD000068ED7BE0CE0143960E945B4BBC0180E264
:10CD100092E10E94094BCE0143960E94F24BC8015A
:10CD20000E94F24B0215130561F6C701B6010E947D
:10CD3000F3B26B017C01FDE24F16F1E05F06610486
:10CD400071042CF00E94DC3E60E080E0AFD323E071
:10CD5000B701A601CE0143960E94F74B68EF78E039
:10CD6000C8010E94564C6AE172E1C8010E94724BF0
:10CD700068E779E00E945B4BBE016D5E7F4F0E94C9
:10CD8000724B6DE779E00E945B4BBC0180E292E15F
:10CD90000E94094BC8010E94F24BCE0143960E94AB
:10CDA000F24B2DEC3CEC4CE45FE3C701B6010E9472
:10CDB000EAB129813A814B815C812DA33EA34FA327
:10CDC00058A718160CF0ACC12AE939E949E95FE324
:10CDD000C701B6010E94A5AE87FFA2C1CDA8CC2095
:10CDE00009F49EC189849A84AB84BC8420E030E03D
:10CDF000A901C501B4010E94A5AECD80DE80EF80FF
:10CE0000F884882309F12DA13EA14FA158A5CA019C
:10CE1000B9010E940AAF6EAB7FAB88AF99AFA70193
:10CE20009601C701B6010E940AAF9B01AC016EA931
:10CE30007FA988AD99AD0E9435B00E94F3B2A501DB
:10CE400094010E94A8B004C06BED7FE089EC9FE3E1
:10CE500020EE3EE245E652E40E940AAF6EAB7FABA5
:10CE600088AF99AF20E030E0A901C701B6010E9468
:10CE7000A5AE882309F12DA13EA14FA158A5CA0155
:10CE8000B9010E940AAF6AAF7BAF8CAF9DAFA5011D
:10CE90009401C501B4010E940AAF9B01AC016AADC7
:10CEA0007BAD8CAD9DAD0E9435B00E94F3B2A70161
:10CEB00096010E94A8B004C06BED7FE089EC9FE36F
:10CEC00020EE3EE245E652E40E940AAF6AAF7BAF35
:10CED0008CAF9DAF20E030E0A9016DA17EA18FA1B4
:10CEE00098A50E94A5AE8823F9F0A5019401C5017B
:10CEF000B4010E940AAF4B015C01A7019601C70172
:10CF0000B6010E940AAF9B01AC01C501B4010E94A9
:10CF100035B00E94F3B22DA13EA14FA158A50E94A9
:10CF2000A8B06B017C0108C08BEDC82E8FE0D82E15
:10CF300089ECE82E8FE3F82E69EF78E0C8010E94B3
:10CF4000564C6AE172E1C8010E94724B60E879E0D8
:10CF50000E945B4BBC0180E292E10E94DD4BC80164
:10CF60000E94F24B69EF78E0C8010E94564C6AE1DA
:10CF700072E1C8010E94724B6AE979E00E945B4B42
:10CF8000BC018AE192E10E94DD4BC8010E94F24B94
:10CF900021E04EA95FA968AD79ADCE014F960E9400
:10CFA000F74B21E04AAD5BAD6CAD7DADCE0149964E
:10CFB0000E94F74B20EE3EE245E652E4C701B6017F
:10CFC0000E940AAFAB01BC0121E0C8010E94F74BEF
:10CFD000B801CE0143960E944E4C68ED7BE0CE0135
:10CFE00043960E945B4BBE01675E7F4F0E94724B6F
:10CFF00068ED7BE00E945B4BBE01615E7F4F0E944B
:10D00000724BBC0184E192E10E94DD4BCE0143965C
:10D010000E94F24BC8010E94F24BCE0149960E9439
:10D02000F24BCE014F960E94F24B2DE2421621E0C8
:10D0300052066104710474F469A57AA58BA59CA5B8
:10D0400025E030E040E050E00E94D7AF672B682B2E
:10D05000692BC1F56AE172E1C8010E944E4C45E0BE
:10D0600050E06FEF7FEFC8010E946090C8010E94FE
:10D07000F24B63EA79E0C8010E94564C45E050E06B
:10D0800061EF7FEFC8010E94BB8FC8010E94F24B85
:10D090006FEB79E0C8010E94564CC8010E94EF8DE9
:10D0A000C8010E94F24B64E172E1C8010E944E4C3B
:10D0B00045E050E060E070E0C8010E94738DC80157
:10D0C0000E94F24B64E172E180E292E10E94094B1E
:10D0D0003FE1431651046104710434F4C9A4DAA495
:10D0E000EBA4FCA4F7FC11C060E272E1C8010E944D
:10D0F0004E4CC8010E940A71C8010E94F24B6FEBAE
:10D1000079E080E292E10E94C84BB201C30177FE50
:10D1100004C069A97AA98BA99CA90E942B86A9C0E1
:10D1200023E04DA15EA16FA178A5CE0143960E9498
:10D13000F74B69EF78E0C8010E94564C6AE172E152
:10D14000C8010E94724B65EA79E00E945B4BBE0108
:10D150006D5E7F4F0E94724B6EE779E00E945B4BE1
:10D16000BC018AE192E10E94DD4BC8010E94F24BB2
:10D17000CE0143960E94F24B49855A856B857C858A
:10D1800023E0CE0149960E94F74B4D815E816F816D
:10D19000788523E0C8010E94F74BB801CE01439681
:10D1A0000E944E4C6AEA79E0CE0143960E945B4BA6
:10D1B000BE01675E7F4F0E94724B6EE779E00E946E
:10D1C0005B4BBC0184E192E10E94DD4BCE014396B2
:10D1D0000E94F24BC8010E94F24BCE0149960E9478
:10D1E000F24B2DE2421621E052066104710474F400
:10D1F00069A57AA58BA59CA525E030E040E050E02C
:10D200000E94D7AF672B682B692BF1F46AE172E1BA
:10D21000C8010E944E4C4AE050E06FEF7FEFC8011A
:10D220000E946090C8010E94F24B64E172E1C80163
:10D230000E944E4C4AE050E060E070E0C8010E945D
:10D24000738DC8010E94F24B60E272E1C8010E9436
:10D250004E4CC801DFD7C8010E94F24B6FEB79E05A
:10D2600080E292E10E94C84BC301B2010E942B866A
:10D270001DAA0E9487876B017C0122962CAD3DADD3
:10D280004EAD5FAD2297C21AD30AE40AF50AC9A6C9
:10D29000DAA6EBA6FCA6C7CC6AE172E1CE010D9638
:10D2A0000E944E4C4AE050E06FEF7FEFCE010D96AA
:10D2B0000E94BB8FCE010D960E94F24BCDA8CC20D0
:10D2C000B1F163EA79E0CE010D960E94564C45E03B
:10D2D00050E061EF7FEFCE010D960E94BB8FCE0133
:10D2E0000D960E94F24B8091450C882391F060E3EB
:10D2F00071E1CE010D960E94464C45E050E060E0A1
:10D3000070E0CE010D960E94BB8FCE010D960E945B
:10D31000F24B6FEB79E0CE010D960E94564CCE0198
:10D320000D960E94EF8DCE010D960E94F24B64E1A6
:10D3300072E1CE010D960E944E4C4AE050E06FEF34
:10D340007FEFCE010D960E94738DCE010D960E9447
:10D35000F24BCB5BDF4F0FB6F894DEBF0FBECDBFF5
:10D36000DF91CF911F910F91FF90EF90DF90CF90C1
:10D37000BF90AF909F908F907F906F905F904F90F5
:10D380003F902F9008956DEB79E00C94E64C0F934D
:10D390001F93CF93DF93EC010E94B44C8C01CE011C
:10D3A000F2DF800F911FDF91CF911F910F910895B0
:10D3B000282F3091380D313208F04AC08091150D78
:10D3C0008111FCCF90912D1342E04093150D2093D5
:10D3D000140D2FEF2093130D1092120D3093110D99
:10D3E000E8E1FDE0A1EFBCE020E0321721F041913F
:10D3F0004D932F5FFACF1092F00C2091F00C990F03
:10D40000922B9093F00C9091EF0C913061F410926C
:10D41000EF0C9091F00C9093BB009091BC0093FDA9
:10D42000F8CF95EC01C095EE9093BC009091150D4E
:10D430009230E1F39091130D9F3F79F08091130D9D
:10D44000803241F08091130D803331F084E005C0CB
:10D4500081E003C082E001C083E01092170D1092BA
:10D46000380D1092160D089581E0A2CF682F8DEA35
:10D470009FE00C94445691E09093160D80932D13E9
:10D480001092170D1092380D0895CF93C82F682F62
:10D49000607F81E293E10E94725780E1C89FB001F2
:10D4A000112481E293E1CF910C947257CF93DF93D3
:10D4B000CDB7DEB728970FB6F894DEBF0FBECDBF4D
:10D4C00098E0EBE3F5E0DE01119601900D929A955C
:10D4D000E1F790912A13961710F46FEF690FFE0190
:10D4E0003196E60FF11DE60FF11D9081890F8068DE
:10D4F00028960FB6F894DEBF0FBECDBFDF91CF9157
:10D50000C4CF0F931F93CF93DF93CDB7DEB7A2970E
:10D510000FB6F894DEBF0FBECDBF8C01CB01BA01B0
:10D52000F8011182108213821282158214822AE07D
:10D53000AE014F5F5F4F0E9477AABE016F5F7F4FC2
:10D54000C8010E94C84BA2960FB6F894DEBF0FBE6A
:10D55000CDBFDF91CF911F910F9108950F931F932E
:10D56000CF93DF93EC010E94E64C8C01CE010BDFE0
:10D57000800F911FDF91CF911F910F910895CF924E
:10D58000DF92EF92FF92CF93DF936B017C0197FFC5
:10D5900015C06DE280E19FE00E94AD4CEC01442794
:10D5A0005527BA014C195D096E097F092AE080E10F
:10D5B0009FE00E94FB4CC80FD91F08C02AE0AB01B6
:10D5C000BC0180E19FE00E94FB4CEC0180E19FE008
:10D5D000DADE8C0F9D1FDF91CF91FF90EF90DF90EF
:10D5E000CF9008958F929F92AF92BF92CF92DF9289
:10D5F000EF92FF920F931F93CF93DF936B017C0108
:10D60000142F9B01AC010E9434B3882319F060EC05
:10D6100079E027C046015701E894B7F82FEF3FEFB4
:10D620004FE75FE7C501B4010E9434B381110DC01B
:10D630002FEF3FEF4FE75FE7C501B4010E94A5AEB2
:10D6400018161CF464EC79E00CC02FEF3FEF4FE7A5
:10D650005FE4C701B6010E94EAB1181694F468ECC1
:10D6600079E080E19FE0DF91CF911F910F91FF90D2
:10D67000EF90DF90CF90BF90AF909F908F900C94E1
:10D68000E64C2FEF3FEF4FE75FECC701B6010E947A
:10D69000A5AE87FDE4CF20E030E0A901C701B601C7
:10D6A0000E94A5AE87FF0BC06DE280E19FE00E9463
:10D6B000AD4CEC01F7FAF094F7F8F09402C0C0E03A
:10D6C000D0E000E060E070E080E09FE3101741F000
:10D6D00020E030E040E251E40E94FBB00F5FF6CF63
:10D6E000A70196010E9435B06B017C010E9499B19F
:10D6F0004B015C012AE0AB01BC0180E19FE00E948C
:10D70000FB4CC80FD91F1123C9F1C501B4010E94F8
:10D71000A9AE9B01AC01C701B6010E9434B06B01F8
:10D720007C016EE280E19FE00E94AD4CC80FD91FE2
:10D7300020E030E040E251E4C701B6010E940AAFA8
:10D740004B015C010E9499B16B01E12CF12C2AE0A4
:10D75000B701A60180E19FE00E94FB4CC80FD91FD2
:10D76000C701B6010E94A9AE9B01AC01C501B4017D
:10D770000E9434B06B017C011150D1F6CE01DF91D3
:10D78000CF911F910F91FF90EF90DF90CF90BF90BE
:10D79000AF909F908F9008952F923F924F925F92FB
:10D7A0006F927F928F929F92AF92BF92CF92DF92B1
:10D7B000EF92FF920F931F93CF93DF93CDB7DEB716
:10D7C00028970FB6F894DEBF0FBECDBFC0909F0C58
:10D7D000D090A00C4091A10C5091A20CC416D5067B
:10D7E0002CF43C2D2D2D6A01432F522FE3EAFCE04F
:10D7F00060E070E0CB01019111910417150754F41A
:10D800004A01550FAA08BB08680D791D8A1D9B1D8A
:10D81000A80115C0C016D10654F40D2C000CEE085A
:10D82000FF086C0D7D1D8E1D9F1D680108C0012E17
:10D83000000C220B330B600F711F821F931F2CE013
:10D84000EF3EF207C1F60E94ABAE20E030E048E1C7
:10D8500052E40E94FBB08B0188879F838FE9E82EFA
:10D860008CE0F82E812C912C5401D7016D917D9183
:10D870007D01072E000C880B990B0E94ABAE98011E
:10D8800048855F810E9434B09B01AC010E940AAFC1
:10D890009B01AC01C501B4010E9435B04B015C0194
:10D8A000EFEEFCE0EE15FF0501F720E030E04CE183
:10D8B00052E40E94FBB00E94F3B26B017C0120E0B5
:10D8C00030E040E85FE30E94EAB118160CF069C04E
:10D8D0002FE93CE03A832983212C312C412C512C17
:10D8E0003201A981BA818D919D91BA83A9839C014E
:10D8F000990F440B550B2B833C834D835E83CA01E8
:10D90000B9010E94ABAE980148855F810E9434B096
:10D910004B015C0120E030E0A9010E94EAB1181639
:10D9200024F0B7FAB094B7F8B094A7019601C501F6
:10D93000B4010E94A5AE87FF0BC08B819C81AD8195
:10D94000BE81480E591E6A1E7B1E9FEF291A390A96
:10D95000AFEEBCE0E981FA81AE17BF0711F620E017
:10D9600030E040EC5FE3C701B6010E940AAF6B01F3
:10D970007C01F5E02F1631040CF4AACFC301B201EB
:10D980000E94ABAE6B017C01B101330C880B990B8B
:10D990000E94ABAE9B01AC01C701B6010E94FBB077
:10D9A00003C0B80188859F816B017C01C701B60166
:10D9B00028960FB6F894DEBF0FBECDBFDF91CF9192
:10D9C0001F910F91FF90EF90DF90CF90BF90AF909D
:10D9D0009F908F907F906F905F904F903F902F908F
:10D9E00008954F925F926F927F928F929F92AF9223
:10D9F000BF92CF92DF92EF92FF921F93CF93DF936C
:10DA0000CDB7DEB728970FB6F894DEBF0FBECDBFF7
:10DA10004B015C0111E0612E712C9301220F331F29
:10DA2000220F331F3A832983F901ED57FD4FC08040
:10DA3000D180E280F380A5019401C701B6010E9464
:10DA4000A5AE87FF02C01F5FE6CFA5019401C70105
:10DA5000B6010E94A5AE49815A8145595D4F5E834A
:10DA60004D83811106C0FA016081718182819381A9
:10DA70004DC0F1E06F1AF0EC7F0AC301880F991FC7
:10DA8000880F991FFC01ED57FD4F208131814281A4
:10DA9000538129833A834B835C83FC01E559FD4F15
:10DAA0004080518062807380A3019201ED81FE81EC
:10DAB00060817181828193810E9434B06D837E8305
:10DAC0008F83988729813A814B815C81C501B4019C
:10DAD0000E9434B09B01AC016D817E818F8198855D
:10DAE0000E940AAF4B015C0129813A814B815C8124
:10DAF000C701B6010E9434B09B01AC01C501B4015D
:10DB00000E94FBB0A30192010E9435B028960FB687
:10DB1000F894DEBF0FBECDBFDF91CF911F91FF9074
:10DB2000EF90DF90CF90BF90AF909F908F907F90BD
:10DB30006F905F904F9008950F931F930E94878777
:10DB40006093DE0D7093DF0D8093E00D9093E10DF7
:10DB500086ED9DE00E948A4797FF1FC00E9487873D
:10DB60000091DE0D1091DF0D2091E00D3091E10D5F
:10DB7000DC01CB01801B910BA20BB30B0091DA0DE2
:10DB80001091DB0D2091DC0D3091DD0D8017910798
:10DB9000A207B307E8F28FEF9FEF1F910F9108954F
:10DBA000CF92DF92EF92FF92CF93DF93EC016A0165
:10DBB0007B01E889F98982E080834115514E610536
:10DBC0007105B1F060E079E08DE390E0A701960186
:10DBD0000E9403B0DA01C9010197A109B109B69504
:10DBE000A795979587959C01211580E13807A8F0A6
:10DBF000E889F989108260E874E88EE190E0A70175
:10DC000096010E9403B0DA01C9010197A109B10987
:10DC1000B695A795979587959C01EC85FD853083F2
:10DC2000EE85FF852083188EEC89FD8986E0808350
:10DC3000EA89FB89808180618083EA89FB89808110
:10DC400088608083EA89FB89808180688083EA8993
:10DC5000FB8980818F7D8083DF91CF91FF90EF9052
:10DC6000DF90CF9008950F931F93CF93DF931F9270
:10DC70001F92CDB7DEB70DE91CE0F80160818EED93
:10DC800093E09A838983CE0101960E940E3FF801AA
:10DC900061818FED93E09A838983CE0101960E9482
:10DCA0000E3FC8010F900F90DF91CF911F910F9100
:10DCB0000895EF92FF920F931F93CF93DF931F92DC
:10DCC0001F92CDB7DEB70AE111E18A5191417C0183
:10DCD000C701800F911FF80161918F019A83898399
:10DCE000CE0101960E940E3FF1E104321F0781F739
:10DCF0008AE191E10F900F90DF91CF911F910F91E9
:10DD0000FF90EF900895EF92FF920F931F93CF93A0
:10DD1000DF931F921F92CDB7DEB70BE810E18B584F
:10DD200090417C01C701800F911FF80161918F0123
:10DD30009A838983CE0101960E940E3FF1E1013161
:10DD40001F0781F78BE890E10F900F90DF91CF9143
:10DD50001F910F91FF90EF900895EF92FF920F9314
:10DD60001F93CF93DF931F921F92CDB7DEB70AE1C7
:10DD700011E18A5191417C01C701800F911FF80187
:10DD800061918F019A838983CE0101960E940E3F93
:10DD9000F2E104311F0781F78AE191E10F900F90C2
:10DDA000DF91CF911F910F91FF90EF9008958F9287
:10DDB0009F92AF92BF92CF92DF92EF92FF920F931A
:10DDC0001F93CF93DF938C01862F0B30110509F041
:10DDD0006FC090918712992309F0F89462E10E9434
:10DDE000B15020918712222309F07894009709F00E
:10DDF00072C0E0908212F09083126F2D70E080E08C
:10DE000090E00E94ABAE2DEC3CEC4CEC5DE30E944C
:10DE10000AAF4B015C016E2D70E080E090E00E9443
:10DE2000ABAE9B01AC01C501B4010E9435B060935B
:10DE30007A1270937B1280937C1290937D12C09122
:10DE40008412D09185126C2F6F7770E080E090E0A3
:10DE50000E94ABAE4B015C016D2F70E080E090E062
:10DE60000E94ABAE2DEC3CEC4CEC5DE30E940AAFA3
:10DE70009B01AC01C501B4010E9435B0C7FD09C0CA
:10DE800060937E1270937F12809380129093811220
:10DE90000BC0DC01CB01B05880937E1290937F12AF
:10DEA000A0938012B0938112FE0CCF0DCD0F71C0E4
:10DEB0000631110509F0B4C090918712992309F039
:10DEC000F89461E00E94B15020918712222309F05A
:10DED00078940097A9F040E050EC69E774EC409327
:10DEE0007A1250937B1260937C1270937D12409350
:10DEF0007E1250937F12609380127093811295C0AE
:10DF0000F0908312D09182126091821270918312EC
:10DF100076276727762780E090E00E94A9AE2DEC57
:10DF20003CEC4CEC5DE30E940AAF60937A12709374
:10DF30007B1280937C1290937D12E0908512C091A9
:10DF400084128C2F8F776E2D70E0782B80E090E01C
:10DF50000E94A9AE2DEC3CEC4CEC5DE30E940AAFB4
:10DF6000C7FD09C060937E1270937F128093801268
:10DF7000909381120BC0DC01CB01B05880937E12CC
:10DF800090937F12A0938012B0938112DF0DED0E5B
:10DF9000CE0D80918612C81346C0C0907A12D090E0
:10DFA0007B12E0907C12F0907D1220E030E048EC93
:10DFB00052E4C701B6010E94EAB118161CF0C0E095
:10DFC000D0E002C0CBEFDFEF20E030E0A901C701D5
:10DFD000B6010E94A5AE87FF02C0CAEFDFEFC09076
:10DFE0007E12D0907F12E0908012F090811220E09B
:10DFF00030E048EC52ECC701B6010E94A5AE87FFA5
:10E0000002C0C9EFDFEF20E030E040EF52E4C7018B
:10E01000B6010E94EAB11816ACF4C8EFDFEF12C0E7
:10E02000CFEFDFEF0FC08FEF9FEF8F3FFFEF9F0727
:10E0300009F4D3C0009709F4B0CF029609F4D9C00F
:10E04000CCEFDFEF0C30110509F0D6C08CE513DA08
:10E0500080E090E00BDA08DA65E08CE50E94A750DA
:10E06000C82FD0E02097A1F0C530D105A4F00EE272
:10E0700013E18DEA9FE00E94FC55F80180870F5F55
:10E080001F4FC8018E5293418C179D0794F306C011
:10E09000CEEFDFEFB1C0CDEFDFEFAEC0C0913613F2
:10E0A00000913713602F70E080E090E00E94ABAEEB
:10E0B0002DEC3CEC4CEC5DE30E940AAF6B017C0163
:10E0C0006C2F70E080E090E00E94ABAE9B01AC0151
:10E0D000C701B6010E9435B060932E1370932F13C1
:10E0E0008093301390933113D091381310913913DA
:10E0F0006D2F6F7770E080E090E00E94ABAE6B0117
:10E100007C01612F70E080E090E00E94ABAE2DECCE
:10E110003CEC4CEC5DE30E940AAF9B01AC01C701F3
:10E12000B6010E9435B0D7FF5BC0DC01CB01B0580F
:10E130008093321390933313A0933413B093351319
:10E140008C2F800FC82FCD0FC10F80913A13C813A9
:10E1500044C0C0902E13D0902F13E0903013F09055
:10E16000311320E030E048EC52E4C701B6010E94D0
:10E17000EAB118161CF0C0E0D0E002C0CBEFDFEF30
:10E1800020E030E040EA50E4C701B6010E94A5AEAD
:10E1900087FF02C0CAEFDFEFC0903213D090331375
:10E1A000E0903413F090351320E030E040EF51EC74
:10E1B000C701B6010E94A5AE87FF02C0C9EFDFEF1D
:10E1C00020E030E040EF52E4C701B6010E94EAB11E
:10E1D000181694F4C8EFDFEF0FC0CFEFDFEF0CC0DD
:10E1E00060933213709333138093341390933513E9
:10E1F000A7CFCEEFDFEF26CFCE01DF91CF911F91DA
:10E200000F91FF90EF90DF90CF90BF90AF909F90D5
:10E210008F900895CF93DF93FC0124813581232BC8
:10E2200089F0EC01BC0189E39DE0B1D86EE170E0BA
:10E2300080E090E00E942B86BE0180E19FE0DF91AC
:10E24000CF91A5C8DF91CF910895CF92DF92EF9241
:10E25000FF92CF93C091BA10C430DCF4C1300CF0FF
:10E260003FC0C11164C07FD720E030E040EA50E4F5
:10E270000E940AAF20E030EC4FE754E40E94FBB06C
:10E280002091BB103091BC104091BD105091BE1038
:10E290004BC0C43009F04BC066D720E030E040EA04
:10E2A00050E40E940AAF20E030EC4FE754E40E94B3
:10E2B000FBB020E030E040EA50E40E94FBB020E0F8
:10E2C00030E040E851E40E940AAF20E030E040E84E
:10E2D00050E40E9435B020E030E04AE754E424C026
:10E2E00042D72AE137E64CE950E40E940AAF209178
:10E2F000BB103091BC104091BD105091BE100E94D7
:10E3000034B06B017C01EC2FEE0FFF0BE955FA4F97
:10E3100060817181072E000C880B990B0E94ABAEB7
:10E320009B01AC01C701B6010E94FBB003C060E0D5
:10E3300070E0CB01CF91FF90EF90DF90CF900895E8
:10E340008F929F92AF92BF92CF92DF92EF92FF9205
:10E35000CF93DF93CDB7DEB72C970FB6F894DEBF1F
:10E360000FBECDBF66E472E1CE0101960E94464C1D
:10E370004CE251E06FEF7FEFCE0101960E94738D6A
:10E38000CE0101960E94F24B6091B7027091B802E3
:10E390008091290290912A020ADD84E1882E912C35
:10E3A000A12CB12CE12CF12C2FEFE21AF20AC501BD
:10E3B000B4010E942B866091B7027091B8028091DF
:10E3C000290290912A02F3DC23E0E216F10434F0F2
:10E3D0002AE0E216F10444F4892B49F084E1880E26
:10E3E000911CA11CB11CE0CF892B09F08BC180913D
:10E3F000290290912A028B309105C9F480917E12F6
:10E4000090917F12A0918012B091811280933F135E
:10E4100090934013A0934113B093421380917A12CA
:10E4200090917B12A0917C12B0917D121DC086311B
:10E43000910521F30C9701F58091321390913313DC
:10E44000A0913413B091351380933F1390934013F0
:10E45000A0934113B093421380912E1390912F13E8
:10E46000A0913013B091311380933B1390933C13E0
:10E47000A0933D13B0933E1340913F13509140132E
:10E48000609141137091421321E0CE0107960E94E2
:10E49000F74B6DE07AE0CE0101960E94564CBE012A
:10E4A000695F7F4FCE0101960E94724BBC0180E2F2
:10E4B00092E10E94DD4BCE0101960E94F24BCE010B
:10E4C00007960E94F24B40913B1350913C13609190
:10E4D0003D1370913E1321E0CE0107960E94F74B49
:10E4E00062E476E0CE0101960E94564CBE01695F5F
:10E4F0007F4FCE0101960E94724BBC0180E292E1F7
:10E500000E94094BCE0101960E94F24BCE01079664
:10E510000E94F24B64E076E080E292E10E94FB4AC6
:10E520006FEB79E0CE0101960E94564C44E150E039
:10E5300060E070E0CE0101960E94BB8FCE01019693
:10E540000E94F24BC0903F13D0904013E0904113D3
:10E55000F090421320E030E0A901C701B6010E940B
:10E56000EAB120E030E040E05FE387FD05C0C7018D
:10E57000B6010E9435B004C0C701B6010E9434B094
:10E580000E9494B1AB01BC01CE0101960E94816A48
:10E59000BE016F5F7F4F8AE192E10E940F4BCE0177
:10E5A00001960E94F24B60E087E00E94566A6AE1A1
:10E5B00072E181E293E10E94B44C6FED81E293E15C
:10E5C0000E94AD4C68E476E081E293E10E948D4DBB
:10E5D00060913B1370913C1380913D1390913E13D9
:10E5E0000E9494B14AE050E081E293E10E94434DE1
:10E5F00064E076E081E293E10E948D4D64E670E094
:10E6000080E090E00E942B86C0903F13D090401392
:10E61000E0904113F090421320E030E040EF51E4ED
:10E62000C701B6010E94EAB187FD03C067E372E14A
:10E6300054C020E030E040ED51E4C701B6010E9433
:10E64000EAB187FD1FC067E272E1CE0101960E9428
:10E65000464C4AE050E06FEF7FEFCE0101960E94FA
:10E66000738DCE0101960E94F24B80914702882360
:10E6700031F06CED75E080E090E00E942B8667E160
:10E6800072E12BC020E030E040EB51E4C701B6015D
:10E690000E94EAB187FD03C069E072E11EC06AEF23
:10E6A00071E1CE0101960E94464C4AE050E06FEFC6
:10E6B0007FEFCE0101960E94738DCE0101960E94DC
:10E6C000F24B80914702882331F06CED75E080E0D9
:10E6D00090E00E942B866CEE71E1CE0101960E94C3
:10E6E000464C4AE050E06FEF7FEFCE0101960E946A
:10E6F000738DCE0101960E94F24B62E370E080E0E0
:10E7000090E0DCC00E94DC3E6EE170E080E090E0D2
:10E710000E942B860E949A976B017C0164E670E050
:10E7200080E090E00E942B866DE07AE080E292E14A
:10E730000E94C84B21E0B701A601CE0101960E94BC
:10E74000F74BBE016F5F7F4F80E292E10E94094B61
:10E75000CE0101960E94F24B60E272E1CE01019679
:10E760000E944E4C4AE050E060E070E0CE0101961D
:10E770000E94BB8FCE0101960E94F24B80912E0524
:10E78000882379F080912D05882359F06FED81E27F
:10E7900093E10E94AD4C66E779E081E293E10E944B
:10E7A0008D4D65E779E080E292E10E94FB4AC092DC
:10E7B0003F13D0924013E0924113F092421320E0B5
:10E7C00030E040EF51E4C701B6010E94EAB187FD95
:10E7D00003C06CED71E154C020E030E040ED51E445
:10E7E000C701B6010E94EAB187FD1FC06CEC71E160
:10E7F000CE0101960E94464C4AE050E06FEF7FEF59
:10E80000CE0101960E94738DCE0101960E94F24BBB
:10E8100080914702882331F06CED75E080E090E054
:10E820000E942B866CEB71E12BC020E030E040EBC6
:10E8300051E4C701B6010E94EAB187FD03C06EEA48
:10E8400071E11EC06FE971E1CE0101960E94464C54
:10E850004AE050E06FEF7FEFCE0101960E94738D8A
:10E86000CE0101960E94F24B80914702882331F03D
:10E870006CED75E080E090E00E942B8661E971E12B
:10E88000CE0101960E94464C4AE050E06FEF7FEFC8
:10E89000CE0101960E94738DCE0101960E94F24B2B
:10E8A0006CE271E080E090E00E942B86809147024C
:10E8B000882331F068EE73E080E090E00E942B86C0
:10E8C0002C960FB6F894DEBF0FBECDBFDF91CF916F
:10E8D000FF90EF90DF90CF90BF90AF909F908F9080
:10E8E0000895DF92EF92FF920F931F93CF93DF93E0
:10E8F000CDB7DEB762970FB6F894DEBF0FBECDBFBF
:10E900008C01109243136FEB79E0CE010D960E94BB
:10E91000564CFF24F39480E19FE00E94AC47209185
:10E92000431318161906DCF5211139C080E19FE068
:10E930000E948A478A3041F08D3031F0682FCE0135
:10E940000D960E94E84A24C089899A89892B01F191
:10E95000F09243136CEC79E0CE0101960E94564C84
:10E96000BE01635F7F4FCE0101960E94724BBC01D6
:10E97000CE0107960E944E4CCE0107960E948F8FC3
:10E98000CE0107960E94F24BCE0101960E94F24BF7
:10E990006AE070E080E090E00E942B86BCCF2111FD
:10E9A00085C0E12CF12CDD24D39489E39DE00E9405
:10E9B000AC471816190614F589E39DE00E948A47B2
:10E9C0008A3079F08D3069F090914313911109C02C
:10E9D000682FCE010D960E94E84A8FEFE81AF80AD8
:10E9E00006C089899A89892B11F0D092431365E07A
:10E9F00070E080E090E00E942B86D7CF64E170E069
:10EA000080E090E00E942B86EF28D1F189899A89D5
:10EA1000892BB1F180919713882361F161E179E04D
:10EA2000CE0101960E94564CBE016F5F7F4FCE0112
:10EA30000D960E940685F82ECE0101960E94F24B9B
:10EA4000F11018C065ED79E080E19FE00E948D4DE6
:10EA5000BE01635F7F4FCE0101960E944E4CBE0106
:10EA60006F5F7F4F80E19FE00E94C769CE010196F2
:10EA70000E94F24B64E170E080E090E00E942B86FF
:10EA800080914313811112C089899A89892B71F46D
:10EA900064E670E080E090E00E942B860E94878709
:10EAA0006FEB79E0C8010E94564C51C089899A8960
:10EAB000019709F046C06BED75E0CE0107960E9404
:10EAC000564CBE01695F7F4FCE010D960E940685B0
:10EAD000811116C06EE577E0CE0101960E94564C7A
:10EAE000BE016F5F7F4FCE010D960E940685FF2409
:10EAF000F3948111F12CCE0101960E94F24B01C0DA
:10EB0000F12CCE0107960E94F24BFF20A1F040E0CD
:10EB100050E0BE01635F7F4FCE0101960E94273F08
:10EB2000BE016F5F7F4F8CE292E10E940F4BCE01DE
:10EB300001960E94F24B64E170E080E090E00E9458
:10EB40002B86BE01635F7F4FC8010E943E4CCE0101
:10EB50000D960E94F24BC80162960FB6F894DEBF84
:10EB60000FBECDBFDF91CF911F910F91FF90EF901E
:10EB7000DF900895DF92EF92FF920F931F93CF9350
:10EB8000DF93CDB7DEB72C970FB6F894DEBF0FBE7C
:10EB9000CDBF8C01109243136FEB79E0CE01079645
:10EBA0000E94564CE12CF12CDD24D39489E39DE0A6
:10EBB0000E94AC471816190614F580914313811171
:10EBC0001EC089E39DE00E948A478A3059F08D304B
:10EBD00049F0682FCE0107960E94E84A8FEFE81AA5
:10EBE000F80A06C08B859C85892B11F0D0924313BF
:10EBF0006FE070E080E090E00E942B86D7CF62E368
:10EC000070E080E090E00E942B86EF2851F089E3CD
:10EC10009DE00E944A4864E670E080E090E00E9437
:10EC20002B868091431381110AC08B859C85892B8B
:10EC300031F46FEB79E0C8010E94564C18C0809106
:10EC40009713882371F0BE01695F7F4FCE01019653
:10EC50000E944E4CCE010196DDDACE0101960E9453
:10EC6000F24BBE01695F7F4FC8010E943E4CCE014E
:10EC700007960E94F24BC8012C960FB6F894DEBF9F
:10EC80000FBECDBFDF91CF911F910F91FF90EF90FD
:10EC9000DF90089581E080932D0580912E058823D3
:10ECA00041F088E080932C1360E081E293E10C94C2
:10ECB0005F57089580912E0581110FC081E08093E8
:10ECC0002E0580932D0580912713982F94609093A3
:10ECD00027138C600E94456A18C080912D058823F7
:10ECE000A1F010922C1360E081E293E10E945F5743
:10ECF00010922D05809127138B7F809327138860B6
:10ED00000E94456A10922E050895C4CF2F923F921B
:10ED10004F925F926F927F928F929F92AF92BF922B
:10ED2000CF92DF92EF92FF920F931F93CF93DF93D7
:10ED3000CDB7DEB766970FB6F894DEBF0FBECDBF76
:10ED40001C0183E79EE00E940D8E40E855E260E0E2
:10ED500070E083E79EE00E94D06D64E670E080E0A2
:10ED600090E00E942B868CED95E0A0E0B0E08093CF
:10ED7000770E9093780EA093790EB0937A0E64E696
:10ED800070E080E090E00E942B868FEF8A8781E020
:10ED90008B8786E88C871D861E861F86188A198AAF
:10EDA00089E78A8BC101880F991F9E8B8D8BC12C9F
:10EDB000D12CE12CF12C412C512C320183E79EE027
:10EDC000E214F3046CF5ED89FE89CE16DF0644F5F6
:10EDD0000E947B4708974CF049E050E0BE01665F17
:10EDE0007F4F83E79EE00E94514765E070E080E03E
:10EDF00090E00E942B8600E010E0812C912C5401C1
:10EE000083E79EE00E94AC47892B31F4F4E08F1633
:10EE10009104A104B104ACF50230110594F535C09C
:10EE20000E940D8EE114F10409F47101C301B201D5
:10EE30000E94ABAE4B015C01B701FF0C880B990B34
:10EE40000E94ABAE9B01AC01C501B4010E94FBB0B6
:10EE500066960FB6F894DEBF0FBECDBFDF91CF919F
:10EE60001F910F91FF90EF90DF90CF90BF90AF90E8
:10EE70009F908F907F906F905F904F903F902F90DA
:10EE800008958FEFC81AD80A99CF83E79EE00E94B1
:10EE9000AC47892B69F083E79EE00E948A47E1E056
:10EEA000F0E0EC0FFD1FE00FF11F80830F5F1F4F9D
:10EEB00065E070E080E090E00E942B860230110552
:10EEC00069F599818A85981329C09A818C85981350
:10EED00025C0CE0103969C8B8B8B83E79EE00E941E
:10EEE000AC47892B31F494E089169104A104B10454
:10EEF0003CF509301105C1F48B8190E0982F8827EB
:10EF00002C81820F911D092E000CAA0BBB0B480E01
:10EF1000591E6A1E7B1EEFEFEE1AFE0AFFEF8F1AD4
:10EF20009F0AAF0ABF0A6CCF83E79EE00E948A4720
:10EF3000EB89FC898193FC8BEB8B0F5F1F4FCDCF4F
:10EF40000430110544F3D8CF2F923F924F925F9235
:10EF50006F927F928F929F92AF92BF92CF92DF92E9
:10EF6000EF92FF920F931F93CF93DF936C01CFEA41
:10EF7000D5E089E0882E82E0982E0BE810E1EE249F
:10EF8000E394F12C22E1222E312C33E1432E512C3B
:10EF900040E1642E712C51E1A52EB12C8091070225
:10EFA000909108028E159F050CF4CAC021E0C2168C
:10EFB000D10439F4F80182AD93ADF40191838083DB
:10EFC0000AC0F2E0CF16D10431F4F40180819181BE
:10EFD000F80193AF82AFF40180819181009739F4F9
:10EFE0008A819B819093BA028093B90222C08130BA
:10EFF000910539F48A819B819093B8028093B7027E
:10F0000018C08230910539F48A819B819093B602B1
:10F010008093B5020EC0039761F48A819B8190931F
:10F02000B4028093B3026FEB79E084E792E10E942F
:10F03000C84BF401819191914F018430910539F4CD
:10F040002A813B81309362022093610212C0853095
:10F05000910539F42A813B8130935A022093590259
:10F0600008C086309105C9F00EC08A30910509F4B8
:10F0700048C08531910589F42A813B8130935E0235
:10F0800020935D023EC08730910579F72A813B814C
:10F090003093600220935F020AC08631910539F4F3
:10F0A0002A813B8130935C0220935B022AC0873126
:10F0B000910539F52A813B812830310549F4709258
:10F0C000030260920202B0920102A092000219C0F3
:10F0D0002730310549F43092030220920202509207
:10F0E0000102409200020DC02630310551F421E0AA
:10F0F00030E030930302209302021092010210923A
:10F1000000029C012B5031092A30310590F42A81EC
:10F110003B813093B4022093B30239E1389FB001B0
:10F12000399F700D112465547D4F84E792E10E9450
:10F13000C84B8FEFE81AF80A22960E5F1F4F2ECFAA
:10F14000DF91CF911F910F91FF90EF90DF90CF90C3
:10F15000BF90AF909F908F907F906F905F904F90F7
:10F160003F902F9008954F925F926F927F929F925F
:10F17000AF92BF92CF92DF92EF92FF920F931F93C5
:10F18000CF93DF93982E8EE0A82EB12CEE24EA9434
:10F1900093E0F92ECFEFD3E0C12CD12C00E010E0AA
:10F1A000412C512C3201892D0E94E1850817190745
:10F1B00028F0C816D90618F46C0101C08C018C1710
:10F1C0009D0728F08E159F0518F47C0101C0EC0105
:10F1D000BC0180E090E00E94A9AE9B01AC01C3019C
:10F1E000B2010E9435B02B013C0165E070E080E087
:10F1F00090E00E942B8681E0A81AB108A1F6B60122
:10F200006E0D7F1D600F711FC60FD71FBE0180E0FE
:10F2100090E00E94A9AE9B01AC01C301B2010E9423
:10F2200034B020E030E040E251E40E94FBB0DF91D6
:10F23000CF911F910F91FF90EF90DF90CF90BF90F3
:10F24000AF909F907F906F905F904F9008954F92F6
:10F250005F926F927F92AF92BF92CF92DF92FF92B6
:10F260000F931F93CF93DF9300D000D0CDB7DEB7BD
:10F270005C0183E79EE00E940D8E40E052EC61E06D
:10F2800070E083E79EE00E94D06D8CED95E0A0E0F9
:10F29000B0E08093770E9093780EA093790EB093A0
:10F2A0007A0E64E670E080E090E00E942B86C12C2C
:10F2B000D12CF12CCA14DB040CF051C065E070E0D5
:10F2C00080E090E00E942B8600E010E0412C512C61
:10F2D0003201F1100FC083E79EE00E94AC47892BFA
:10F2E00031F485E148165104610471041CF40330C3
:10F2F000110554F08FEFC81AD80A64E670E080E078
:10F3000090E00E942B86D6CF83E79EE00E94AC4718
:10F31000892B69F083E79EE00E948A47E1E0F0E0F4
:10F32000EC0FFD1FE00FF11F80830F5F1F4F65E0A3
:10F3300070E080E090E00E942B86023011054CF0D6
:10F3400089818B3B31F4FF24F3948A818A3A09F056
:10F35000F12C8FEF481A580A680A780ABACF8F2D15
:10F3600026960FB6F894DEBF0FBECDBFDF91CF91CA
:10F370001F910F91FF90DF90CF90BF90AF907F9043
:10F380006F905F904F9008951F93CF93DF93182F46
:10F39000CFE9DCE0812F0E94E185899399936CE3AA
:10F3A00070E080E090E00E942B868CE0CF3ED80792
:10F3B00089F70E94CC6B20E030E040EA50E40E94E4
:10F3C0000AAF20E030E040E85AE30E940AAFDF9144
:10F3D000CF911F9108954F925F926F927F928F927B
:10F3E0009F92AF92BF92CF92DF92EF92FF92CF9314
:10F3F000DF93CDB7DEB768970FB6F894DEBF0FBEC8
:10F40000CDBF6B017C010E948787698B7A8B8B8BC8
:10F410009C8B86ED9DE00E940D8E61E08091020242
:10F420000E94A58560E0809100020E94A5850E944F
:10F430009A970E94E05B0E94FD5B6D877E878F87B5
:10F44000988B0E9406864B015C016AE070E080E0C8
:10F4500090E00E942B866CED79E080E292E10E94C0
:10F46000C84B20E030E04AE754E4C701B6010E94EF
:10F470000AAF6D8B7E8B8F8B988F412C512C320174
:10F48000C12CD12C7601C701B6010E94ABAE2D89EB
:10F490003E894F89588D0E94A5AE87FF85C10E9485
:10F4A000878729893A894B895C89621B730B840B96
:10F4B000950B0E94A9AE20E030E04AE754E40E9498
:10F4C000FBB0AB01BC0123E0CE0101960E94F74BDB
:10F4D000BE016F5F7F4F8AE192E10E940F4BCE0128
:10F4E00001960E94F24B0E94FD5B6B017C010E9421
:10F4F00006869B01AC01281939094A095B094901B3
:10F500005A0131ED831637E09306A104B1040CF4DF
:10F5100041C020E030E0A901C701B6010E94EAB174
:10F5200018165CF426EA3BE944EC5BE3C701B6013C
:10F530000E94A5AE87FF0BC02DC026EA3BE944EC34
:10F540005BEBC701B6010E94EAB118161CF1C501B8
:10F55000B40128EE33E040E050E00E94D7AFCA018A
:10F56000B9010E94ABAE4B015C012D853E854F85F4
:10F570005889C701B6010E9434B020E030E04AE764
:10F5800054E40E940AAFA50194010E94FBB04B0114
:10F590005C0103C0812C912C54016AE172E1CE011F
:10F5A00001960E944E4C6BED75E0CE0101960E94D3
:10F5B0005B4BBC018AE192E10E94DD4BCE010196DA
:10F5C0000E94F24B23E0B701A601CE0101960E94F2
:10F5D000F74BBE016F5F7F4FCE0107960E944E4CE6
:10F5E00068EC78E0CE0107960E945B4BBC0184E199
:10F5F00092E10E94DD4BCE0107960E94F24BCE01B4
:10F6000001960E94F24B22E0B501A401CE010796BB
:10F610000E94F74B69EF78E0CE0101960E94564CAC
:10F620006AE172E1CE0101960E94724B6AEF79E0C5
:10F630000E945B4B64E172E10E94724B6EED75E0DB
:10F640000E945B4BBE01695F7F4F0E94724B69ED68
:10F6500075E00E945B4BBC0180E292E10E94094B85
:10F66000CE0101960E94F24BCE0107960E94F24B0A
:10F6700020E030E0A901C501B4010E94EAB187FD94
:10F6800006C068ED7BE084E192E10E94FB4A22E043
:10F69000B501A401CE0101960E94F74BBE016F5F38
:10F6A0007F4FCE0107960E944E4C69ED75E0CE016A
:10F6B00007960E945B4BBC0184E192E10E94094BDA
:10F6C000CE0107960E94F24BCE0101960E94F24BAA
:10F6D00060E272E1CE0101960E944E4CCE0101968D
:10F6E0000E940A71CE0101960E94F24BC301B20141
:10F6F00025E030E040E050E00E94D7AF672B682B58
:10F70000692B21F56CE772E1CE0101960E94464C0F
:10F7100045E050E060E070E0CE0101960E94BB8FB2
:10F72000CE0101960E94F24B64E172E1CE01019696
:10F730000E944E4C45E050E06FEF7FEFCE01019606
:10F740000E94738DCE0101960E94F24B6FEB79E01F
:10F7500080E292E10E94C84B65E070E080E090E0BA
:10F760000E942B860E9487876B017C0129893A8938
:10F770004B895C89C21AD30AE40AF50A0E94FD5B30
:10F780006D877E878F87988B0E9406864B015C0170
:10F790006AE070E080E090E00E942B863FEF431A21
:10F7A000530A630A730A6FCE60E0809102020E94DE
:10F7B000A58568960FB6F894DEBF0FBECDBFDF916A
:10F7C000CF91FF90EF90DF90CF90BF90AF909F9040
:10F7D0008F907F906F905F904F9008954F925F92BF
:10F7E0006F927F92AF92BF92CF92DF92EF92FF9291
:10F7F0000F931F93CF93DF93CDB7DEB7EA970FB682
:10F80000F894DEBF0FBECDBFF82E6FEB79E0CE01CE
:10F81000C5960E94564C8E010B5E1F4F6F2DC8017E
:10F820000E94345718870F831D821E82198289E037
:10F830008A8381E08B838C831C8A1B8ACE0101968C
:10F840000E944154CE0101960E94D553CE010196EB
:10F850000E9406530E8110E00330110509F46EC1B9
:10F8600062E772E1CE01C5960E94834B6FEB79E0AF
:10F8700080E292E10E94C84BBE016B5C7F4FCE01DB
:10F8800083960E944E4C4AE050E060E070E0CE016A
:10F8900083960E94BB8FCE0183960E94F24B61E05B
:10F8A00080E00E94566A6DE07AE0CE01C5960E9423
:10F8B000C84B81E1A82E8CE0B82ECC24C394D12C67
:10F8C000E12CF12CE016F1060CF0EEC06E2DCE010D
:10F8D00001960E949752F5012191319141915191E8
:10F8E0005F010E9435B02B013C0120E030E04CEF7D
:10F8F00052EC0E94A5AE87FF24C0B601CE018996C6
:10F900000E947C506AEA77E0CE0183960E94564CB2
:10F91000BE01675D7F4FCE0183960E94724B6EEFF2
:10F9200079E00E945B4BBC0180E292E10E94094BAE
:10F93000CE0183960E94F24BCE0189960E94F24B33
:10F9400048C022E0B301A201CE018F960E94F74B7E
:10F95000B601CE0189960E947C506AEA77E0CE011A
:10F9600083960E94564CBE01675D7F4FCE01839601
:10F970000E94724B64ED7AE00E945B4BBE01615DB8
:10F980007F4F0E94724BBC0184E192E10E94DD4BEB
:10F99000CE0183960E94F24BCE0189960E94F24BD3
:10F9A000CE018F960E94F24B64E172E1CE01839604
:10F9B0000E944E4C68ED7BE0CE0183960E945B4B2B
:10F9C000BC0180E292E10E94094BCE0183960E9425
:10F9D000F24B0130110559F4E114F10409F05DC056
:10F9E00060E272E1CE01C5960E94DD4B56C0023046
:10F9F000110511F522E0B301A201CE0183960E9408
:10FA0000F74BBE016D5D7F4FCE0189960E944E4C33
:10FA100068ED7BE0CE0189960E945B4BBC01CE0174
:10FA2000C5960E94094BCE0189960E94F24BCE01E9
:10FA300083960E94F24B31C00330110571F164E1ED
:10FA400072E1CE0183960E944E4C44E150E06FEF8C
:10FA50007FEFCE0183960E94738DCE0183960E9424
:10FA6000F24B66E779E0CE0183960E94564CCE01B8
:10FA700083960E94EF8DCE0183960E94F24B809177
:10FA80002E05882351F080912D05882331F060EDFB
:10FA900077E080E090E00E942B86FFEFEF1AFF0AEC
:10FAA0008FEFC81AD80A0ECFCE01C5960E94484AD9
:10FAB00080E292E10E94484A01151105C9F46FE500
:10FAC00072E180E292E10E94834B64E572E1CE0133
:10FAD00083960E94464C4AE050E06FEF7FEFCE01E4
:10FAE00083960E94738DCE0183960E94F24BEBC0E9
:10FAF000043011050CF000C1BE016B5C7F4FCE01DC
:10FB000083960E944E4C4AE050E06FEF7FEFCE01AB
:10FB100083960E94738DCE0183960E94F24B66E716
:10FB200079E0CE0183960E94564CCE0183960E94C6
:10FB3000EF8DCE0183960E94F24BDEC06AE07AE040
:10FB4000CE01C5960E94C84BBE016B5C7F4FCE01B3
:10FB500083960E944E4C4AE050E060E070E0CE0197
:10FB600083960E94BB8FCE0183960E94F24B6FEB6F
:10FB700079E080E292E10E94C84B60E272E1CE013E
:10FB8000C5960E94DD4B00E010E0602FCE0101968B
:10FB90000E9497526B017C0122E0AB01BC01CE01B7
:10FBA00083960115110551F40E94F74BBE016D5D5E
:10FBB0007F4F81E293E10E94B44C18C00E94F74B42
:10FBC000BE016D5D7F4FCE0189960E944E4C68ED5F
:10FBD0007BE0CE0189960E945B4BBC01CE01C596AD
:10FBE0000E94094BCE0189960E94F24BCE0183966A
:10FBF0000E94F24B22E0B701A601CE0183960E943B
:10FC0000F74BBE016D5D7F4FCE0189960E944E4C31
:10FC100068ED7BE0CE0189960E945B4BBC0180E2DF
:10FC200092E10E94094BCE0189960E94F24BCE01CF
:10FC300083960E94F24B0F5F1F4F0330110509F0AE
:10FC4000A4CFCE01C5960E94484ABE016B5C7F4F8F
:10FC5000CE0183960E944E4C4AE050E06FEF7FEF5A
:10FC6000CE0183960E94738DCE0183960E94F24B43
:10FC700066E779E0CE0183960E94564CCE018396CA
:10FC80000E94EF8DCE0183960E94F24B80E292E1BA
:10FC90000E94484A60E17AE0CE0183960E94564C69
:10FCA00060E272E1CE0183960E94724B6AE17AE0D3
:10FCB0000E945B4BBC0180E292E10E94DD4BCE01D1
:10FCC00083960E94F24BCE01C5960E94F24BEA96B3
:10FCD0000FB6F894DEBF0FBECDBFDF91CF911F915D
:10FCE0000F91FF90EF90DF90CF90BF90AF907F90FB
:10FCF0006F905F904F9008956AE17AE080E292E120
:10FD00000E94FB4AE0CFAF92BF92CF92DF92EF9278
:10FD1000FF920F931F93CF93DF93CDB7DEB7A497D6
:10FD20000FB6F894DEBF0FBECDBF80914413882379
:10FD300019F01092441377C58091421290914312AA
:10FD4000049708F03FC060EF77E0CE0101960E9473
:10FD5000564CBE016F5F7F4F88E392E157D6182F54
:10FD6000CE0101960E94F24B112361F161E070E037
:10FD70008EE392E10E94A84A80330CF4845E6AE22A
:10FD800070E0681B710987FD7395CE0101960E9492
:10FD90007C50BE016F5F7F4F8EE392E10E940F4B5C
:10FDA000CE0101960E94F24B6EE372E18CE292E189
:10FDB0000E94DD4B8EE392E10E943D4ACB010E94FE
:10FDC000D70A31C561E577E0CE0101960E94564C15
:10FDD000BE016F5F7F4F88E392E118D6182FCE01E6
:10FDE00001960E94F24B112309F482C36DE27AE07E
:10FDF000CE0101960E94564CCE0101960E940A71D6
:10FE0000CE0101960E94F24B69E37AE0CE0107969B
:10FE10000E94564C65E173E1CE0107960E94724B39
:10FE2000BC01CE0101960E944E4CCE0101960E946B
:10FE30000A71CE0101960E94F24BCE0107960E94F4
:10FE4000F24B60914302709144028091450290917F
:10FE500046020E94ABAE20E030E048EC52E40E9443
:10FE6000FBB0AB01BC0122E0CE0107960E94F74B2C
:10FE70006FE47AE0CE010D960E94564CBE01695F98
:10FE80007F4FCE010D960E94724B62E578E00E9492
:10FE90005B4BBC01CE0101960E944E4CCE010196F7
:10FEA0000E940A71CE0101960E94F24BCE010D967E
:10FEB0000E94F24BCE0107960E94F24B40913F0206
:10FEC00050914002609141027091420224E0CE01C3
:10FED00007960E94F74B64E67AE0CE010D960E94E9
:10FEE000564CBE01695F7F4FCE010D960E94724B4A
:10FEF000BC01CE0101960E944E4CCE0101960E949B
:10FF00000A71CE0101960E94F24BCE010D960E941D
:10FF1000F24BCE0107960E94F24B40913302509172
:10FF20003402609135027091360222E0CE010796CC
:10FF30000E94F74B40912B0250912C0260912D02B0
:10FF400070912E0223E0CE010D960E94F74B409156
:10FF50003702509138026091390270913A0222E0E2
:10FF6000CE0143960E94F74B40912F0250913002F0
:10FF7000609131027091320223E0CE0149960E94D5
:10FF8000F74B61E87AE0CE014F960E94564CBE01D5
:10FF9000675E7F4FCE014F960E94724B66E97AE012
:10FFA0000E945B4BBE016D5E7F4F0E94724B69E900
:10FFB0007AE00E945B4BBE01635F7F4F0E94724BF1
:10FFC00066E97AE00E945B4BBE01695F7F4F0E9449
:10FFD000724B6FE97AE00E945B4BBC01CE01019647
:10FFE0000E944E4CCE0101960E940A71CE010196EC
:10FFF0000E94F24BCE014F960E94F24BCE014996E1
:020000021000EC
:100000000E94F24BCE0143960E94F24BCE010D9618
:100010000E94F24BCE0107960E94F24B6BEA72E10E
:10002000CE0149960E94464CF090BA100F2D0F2C2D
:10003000000C110B01151105A1F52091BB10309199
:10004000BC104091BD105091BE1060E070E080EA9D
:1000500090E40E94FBB0AB01BC0122E0CE0101960E
:100060000E94F74B65E878E0CE0107960E94564C57
:10007000BE016F5F7F4FCE0107960E94724B64ED09
:1000800078E00E945B4BBC01CE0149960E94094B6F
:10009000CE0107960E94F24BCE0101960E94F24BD0
:1000A00009C00130110531F46DE972E1CE014996C4
:1000B0000E94B94AC8010297029738F58F2D9AE03D
:1000C0008902B0011124CE0101960E947C5064EA9D
:1000D0007AE0CE0107960E94564CBE016F5F7F4FBB
:1000E000CE0107960E94724B6DEC78E00E945B4B4C
:1000F000BC01CE0149960E94094BCE0107960E9491
:10010000F24BCE0101960E94F24B0430110519F416
:100110006BE872E105C00530110534F063E872E167
:10012000CE0149960E94B94ABE01675E7F4FCE015B
:1001300001960E944E4CCE0101960E940A71CE019A
:1001400001960E94F24B60EB7AE0CE0149960E9444
:10015000C84B8091B7106091B8107091B91083307E
:100160000CF04FC3CE0101960E947C506BEA7AE0FE
:10017000CE0107960E94564CBE016F5F7F4FCE01A5
:1001800007960E94724B62EB7BE00E945B4BBC01C6
:10019000CE0149960E94094BCE0107960E94F24B70
:1001A000CE0101960E94F24BBE01675E7F4FCE01E9
:1001B00001960E944E4CCE0101960E940A71CE011A
:1001C00001960E94F24B4091BF105091C010609177
:1001D000C1107091C21022E0CE0107960E94F74B29
:1001E00060EC7AE0CE010D960E94564CBE01695F2C
:1001F0007F4FCE010D960E94724B66ED7AE00E9411
:100200005B4BBC01CE0101960E944E4CCE01019683
:100210000E940A71CE0101960E94F24BCE010D960A
:100220000E94F24BCE0107960E94F24B4091D510EE
:100230005091D6106091D7107091D81022E0CE0165
:1002400007960E94F74B6DED7AE0CE010D960E9465
:10025000564CBE01695F7F4FCE010D960E94724BD6
:100260006DEC75E00E945B4BBC01CE0101960E94D3
:100270004E4CCE0101960E940A71CE0101960E9459
:10028000F24BCE010D960E94F24BCE0107960E94D2
:10029000F24B89E0C82E82E0D82E01E010E099E10F
:1002A000F92E8091070290910802801791070CF4B3
:1002B0004DC0F601A190B1906F01B501CE01079636
:1002C0000E947C50B801CE010D960E947C5060EFD8
:1002D0007AE0CE0143960E94564CBE01635F7F4F89
:1002E000CE0143960E94724B68EF7AE00E945B4B0E
:1002F000BE01695F7F4F0E94724B6BEF7AE00E94F4
:100300005B4BFA9CB001FB9C700D112465547D4F32
:100310000E945B4BBC01CE0101960E944E4CCE0167
:1003200001960E940A71CE0101960E94F24BCE0105
:1003300043960E94F24BCE010D960E94F24BCE01E5
:1003400007960E94F24B0F5F1F4FABCF80910111B8
:1003500090910211892B71F461E07BE0CE0101964E
:100360000E94564CCE0101960E940A71CE01019660
:100370000E94F24B8091011190910211019771F44A
:1003800060E17BE0CE0101960E94564CCE010196C1
:100390000E940A71CE0101960E94F24B80910111D8
:1003A00090910211029771F46AE17BE0CE0101960F
:1003B0000E94564CCE0101960E940A71CE01019610
:1003C0000E94F24B6091290270912A02CE01079699
:1003D0000E947C506CE27BE0CE010D960E94564C50
:1003E000BE01695F7F4FCE010D960E94724BBC012A
:1003F000CE0101960E944E4CCE0101960E940A71D8
:10040000CE0101960E94F24BCE010D960E94F24B56
:10041000CE0107960E94F24B40915002509151023A
:10042000609152027091530222E0CE0107960E9421
:10043000F74B69E47BE0CE010D960E94564CBE015D
:10044000695F7F4FCE010D960E94724B6BED75E098
:100450000E945B4BBC01CE0101960E944E4CCE0126
:1004600001960E940A71CE0101960E94F24BCE01C4
:100470000D960E94F24BCE0107960E94F24B4091DE
:10048000550250915602609157027091580222E035
:10049000CE0107960E94F74B69E57BE0CE010D96F1
:1004A0000E94564CBE01695F7F4FCE010D960E949F
:1004B000724B6BED75E00E945B4BBC01CE01019667
:1004C0000E944E4CCE0101960E940A71CE01019607
:1004D0000E94F24BCE010D960E94F24BCE01079680
:1004E0000E94F24B10925402CE0149960E94F24BA8
:1004F00080914212909143128330910508F06FC1B0
:100500008130910541F460E070E08EE392E10E9459
:10051000A84AE82E57C0029709F054C060EF77E070
:10052000CE0101960E94564CBE016F5F7F4F88E35B
:1005300092E16CD2182FCE0101960E94F24B11234A
:1005400009F440C061E070E08EE392E10E94A84AA5
:10055000682FCE0101960E94264CBE016F5F7F4F2F
:100560008CE292E10E940F4BCE0101960E94F24B69
:1005700060E070E08EE392E10E94A84AE82E80914C
:1005800097138823F9F069E67BE0CE0101960E947B
:10059000564C6EE372E1CE0101960E94724B68EDFB
:1005A0007BE00E945B4BBC0180E19FE00E94B44C69
:1005B000CE0101960E94F24B6CE272E180E19FE075
:1005C0000E94C7698E2DEE0C990B0E94C7B5892B2E
:1005D000B1F00E944A760E94DC3E68ED7BE0CE01DD
:1005E00001960E94564C4AE050E060E070E0CE0177
:1005F00001960E946090CE0101960E94F24B6EE33C
:1006000072E1CE0107960E944E4C60E070E0CE0190
:1006100007960E94A84A823409F474C0D4F4803347
:1006200009F490C07CF4833209F483C08A3209F063
:10063000A9C062E87BE08EE392E10E94C84B8FEF95
:100640009FEF8EC0813309F48EC0813409F44FC00E
:1006500099C0813609F44BC034F4833409F45DC089
:10066000843449F08FC0833609F457C00CF44AC073
:10067000843609F087C08091301290913112892B15
:1006800009F49FC061E070E0CE0107960E94A84A7D
:10069000182F80919713882361F06FE67BE080E14B
:1006A0009FE00E948D4D6CE272E180E19FE00E942C
:1006B000C76910330CF4145E6AE270E0611B7109C3
:1006C00017FD7395CE0101960E947C50BE016F5FAD
:1006D0007F4F8CE292E10E940F4BCE0101960E9467
:1006E000F24B8CE292E10E943D4ACB0139C066E7B1
:1006F0007BE08EE392E10E94C84B8091090C9091BF
:100700000A0C2EC069E77BE08EE392E10E94C84BA1
:100710001092450C8CEF9FEF23C06CE77BE08EE3DB
:1007200092E10E94C84B81E08093450C8DEF9FEFD2
:1007300017C06FE77BE08EE392E10E94C84B8EEF1B
:100740009FEF0EC068E579E08CE292E10E94C84B11
:1007500068E579E08EE392E10E94C84B80E090E08A
:100760000E94D70A2EC063E87BE08CE292E10E94EF
:10077000C84B63E87BE08EE392E10E94C84B81E0C6
:1007800090E0EECFBE01695F7F4F8CE292E10E9464
:10079000DD4B60E070E08CE292E10E94A84A082EF6
:1007A000000C990BC0970A9738F48CE292E10E94F2
:1007B0003D4ACB010E94D70A64E670E080E090E0F9
:1007C0004AD2CE0107960E94F24BA1D360933B0C14
:1007D00070933C0C80933D0C90933E0C02C00E94A1
:1007E000962495D360933B0C70933C0C80933D0C06
:1007F00090933E0C6FEB79E08EE392E10E94C84B40
:1008000012C0CE0101960E947C5065E87BE0CE01CB
:1008100007960E94564CBE016F5F7F4FCE01079630
:100820000E94724BB4CCA4960FB6F894DEBF0FBEF4
:10083000CDBFDF91CF911F910F91FF90EF90DF908F
:10084000CF90BF90AF90089590E0FC013197E231D6
:10085000F10508F04EC08827E855FF4F8F4F0C94E4
:100860006FB3809180008F7703C0809180008F7D6F
:1008700080938000089580918000877FF9CF84B5B0
:100880008F7702C084B58F7D84BD08958091B000BC
:100890008F7703C08091B0008F7D8093B000089562
:1008A000809190008F7707C0809190008F7D03C06A
:1008B00080919000877F8093900008958091A000A0
:1008C0008F7707C08091A0008F7D03C08091A0002A
:1008D000877F8093A0000895809120018F7707C0C3
:1008E000809120018F7D03C080912001877F8093BC
:1008F00020010895CF93DF93FC0124813581232BC0
:1009000071F0FB01DC01CD91DC9160817181CE0140
:100910000E941EB6009719F08C1B9D0B02C08FEF32
:100920009FEFDF91CF9108950F931F93CF93DF93A4
:10093000FC01C481D581209719F4FB01108211C0FC
:10094000415051094C175D0708F4EA018B01FC0185
:1009500060817181AE01C8010E940FB6C00FD11F26
:100960001882DF91CF911F910F910895AF92BF929E
:10097000CF92DF92EF92FF920F931F93CF93DF936B
:10098000FC0124813581FB01448155818901041BCF
:10099000150B4115510551F12115310539F1241778
:1009A000350720F10217130718F0890101501109CA
:1009B0007B01FC01A080B180C501DFEFCFEF6501B5
:1009C000C00ED11EC816D906A0F0F7016081718152
:1009D0000E941EB6009769F09C012A193B09021774
:1009E000130710F0D22FC32F0196ECCF8FEF9FEF9C
:1009F00002C08D2F9C2FDF91CF911F910F91FF90FF
:100A0000EF90DF90CF90BF90AF900895FB014481AD
:100A10005581FC01248135812417350778F08081C8
:100A20009181009759F0FB01608171816115710519
:100A300029F00E9401B621E0892B09F020E0822FE5
:100A40000895CF93DF93C0913812D0913912209737
:100A500051F08881882339F0082E000C990B0E94F0
:100A6000E0B58993F6CFDF91CF910895FC01A0897D
:100A7000B1898C91A689B78982FD0FC09C91818D27
:100A80008F5F8F73228D821749F0218DDF01A20FB6
:100A9000B11D5D969C93818F08958C910895CF939D
:100AA000DF93282F30E0F901EA56FC4E8491F901DA
:100AB000E05BFC4ED491F901E65FFC4EC491CC237F
:100AC00089F08111C1DEEC2FF0E0EE0FFF1FE05145
:100AD000FD4EA591B491EC91ED2381E090E021F4DD
:100AE00080E002C080E090E0DF91CF9108951F93F5
:100AF000CF93DF93282F30E0F901EA56FC4E849122
:100B0000F901E05BFC4ED491F901E65FFC4EC49123
:100B1000CC23B9F0162F811197DEEC2FF0E0EE0F09
:100B2000FF1FEA52FD4EA591B4919FB7F8941111A1
:100B300004C08C91D095D82302C0EC91DE2BDC93BD
:100B40009FBFDF91CF911F910895CF93DF9390E0E6
:100B5000FC01E05BFC4E2491FC01E65FFC4E8491BD
:100B6000882361F190E0880F991FFC01E454FD4E49
:100B7000C591D491FC01EA52FD4EA591B491611149
:100B800009C09FB7F8948881209582238883EC91CF
:100B90002E230BC0623061F49FB7F8948881322F06
:100BA000309583238883EC912E2B2C939FBF06C016
:100BB0008FB7F894E8812E2B28838FBFDF91CF91D8
:100BC0000895863308F0865390917B00282F287073
:100BD000977F922B90937B0020912C0590E4299F86
:100BE000900111248770822B80937C0080917A0081
:100BF000806480937A0080917A0086FDFCCF80919A
:100C000078002091790090E0922B08953FB7F894F6
:100C10008091491390914A13A0914B13B0914C13BA
:100C200026B5A89B05C02F3F19F00196A11DB11D47
:100C30003FBFBA2FA92F982F8827820F911DA11D82
:100C4000B11DBC01CD0142E0660F771F881F991FBF
:100C50004A95D1F708958F929F92AF92BF92CF920B
:100C6000DF92EF92FF926B017C01D0DF4B015C01C0
:100C7000C114D104E104F104E9F0C8DFDC01CB01C7
:100C800088199909AA09BB09883E9340A105B105B5
:100C900078F321E0C21AD108E108F10888EE880E45
:100CA00083E0981EA11CB11CC114D104E104F1041D
:100CB00021F7DECFFF90EF90DF90CF90BF90AF9005
:100CC0009F908F900895FF920F931F93CF93DF9380
:100CD000CDB7DEB72B970FB6F894DEBF0FBECDBFF2
:100CE00083E79EE09AD740E855E260E070E083E752
:100CF0009EE00E94D06D64E670E080E090E0ABDFA3
:100D00008CED95E0A0E0B0E08093770E9093780EA4
:100D1000A093790EB0937A0E64E670E080E090E0E4
:100D20009ADF8FEF898381E08A8386E88B831C8238
:100D30001D821E821F82188689E7898783E79EE0CD
:100D40000E944A4862E370E080E090E084DF83E73D
:100D50009EE00E947B4708974CF049E050E0BE01BE
:100D60006F5F7F4F83E79EE00E94514762E370E030
:100D700080E090E070DF83E79EE00E94AC47892B23
:100D800001F183E79EE00E947B47089784F465E0C9
:100D900070E080E090E05FDF00E010E0F12C83E79E
:100DA0009EE00E94AC4702301105A4F50CC049E05A
:100DB00050E0BE016F5F7F4F83E79EE00E94514786
:100DC000E6CFF12C27C083E79EE00E94AC47892B39
:100DD00099F465E070E080E090E03DDF02301105BD
:100DE000F1F69A8589819813DACF9B858B819813C8
:100DF000D6CFFF24F394D3CF83E79EE00E948A47A7
:100E0000EAE0F0E0EC0FFD1FE00FF11F80830F5FC1
:100E10001F4FDFCF62E370E080E090E01CDF83E7EC
:100E20009EE0FBD68F2D2B960FB6F894DEBF0FBE3B
:100E3000CDBFDF91CF911F910F91FF900895CF9378
:100E4000DF930E944A501092261380912A13823019
:100E500018F098E09093261390912B13992339F072
:100E6000813029F48091261384608093261362E3F5
:100E700070E080E090E0EFDE60912C1381E293E17E
:100E80000E945F5768EE73E080E090E0E4DE60E38C
:100E900081E293E10E947257CBE4D6E4CE01019740
:100EA000F1F760E381E293E10E9472572197F1F735
:100EB00060E381E293E10E94725783E592E001973B
:100EC000F1F760E281E293E10E947257809126136C
:100ED00080620E94456A84E0809327138CE00E9420
:100EE000456A81E00E94456ACBE3DFE1CE010197CC
:100EF000F1F782E08093281386E00E94456A82E041
:100F00000E94456A2197F1F7DF91CF9108952FB79D
:100F1000F894609145137091461380914713909116
:100F200048132FBF08952F923F924F925F926F9276
:100F30007F928F929F92AF92BF92CF92DF92EF9269
:100F4000FF920F931F93CF93DF93CDB7DEB76697D2
:100F50000FB6F894DEBF0FBECDBF7C016D8B7E8BCC
:100F60005C8B4B8B19016FEB79E00E94564C8EE144
:100F7000882E912C8E010F5F1F4F2101032C000C36
:100F800066087708CD88DE88A12CB12CA214B304A2
:100F90000CF07BC0B501CE010D960E947C50BE01C5
:100FA000635F7F4FCE0107960E944E4C66E177E06B
:100FB000CE0107960E945B4B6B897C890E94724B25
:100FC000B6010E94724BBC01C8010E944E4C40ED1C
:100FD00057E060E070E0C80186D5C8010E94F24B7E
:100FE000CE0107960E94F24BCE010D960E94F24B65
:100FF00044E150E061E070E0C8010E94EA540E153F
:101000001F0521F0B801C7010E940F4BC8010E94C3
:10101000F24BF70184819581892BA9F160E070E0A2
:10102000C7010E94A84A082E000C990BC0970A9786
:1010300040F4C7010E943D4A641575058605970571
:101040004CF066E779E0F701808191810E94F1B56B
:10105000892B59F481E0FFEFAF1ABF0A96E0C90E61
:10106000D11C882309F492CF15C06CED73E1C8013F
:101070000E94464C40ED57E060E070E0C80133D577
:10108000C8010E94F24B80E0E6CFE1E08E1A9108A1
:1010900009F078CFC70166960FB6F894DEBF0FBE91
:1010A000CDBFDF91CF911F910F91FF90EF90DF9017
:1010B000CF90BF90AF909F908F907F906F905F90F8
:1010C0004F903F902F900895CF93DF93EC014830DD
:1010D00085E058076105710509F441C108F08DC02C
:1010E000493481E058076105710509F43BC1E0F519
:1010F000443481E058076105710509F424C1E8F41E
:10110000413481E058076105710509F413C138F4D1
:10111000403451406105710509F409C135C14234BB
:1011200081E058076105710509F407C14334514056
:101130006105710509F404C127C1463481E05807EF
:101140006105710509F405C108F400C1473481E067
:1011500058076105710509F4FFC048345140610525
:10116000710509F4FCC010C1423085E058076105E3
:10117000710509F4E2C0E8F4443781E058076105DD
:10118000710509F4F5C038F4423751406105710525
:1011900009F4F1C0F9C0411585E0580761057105F2
:1011A00009F4C5C0413055406105710509F4C2C05C
:1011B000EBC0453085E058076105710509F4C6C0EC
:1011C00070F4433085E058076105710509F4B8C033
:1011D000443055406105710509F4B5C0D5C04630AD
:1011E00085E058076105710509F4B3C047305540E3
:1011F0006105710509F4B0C0C7C04D3B82E45807D2
:101200008FEF6807710509F4BCC008F045C04F3E78
:1012100080E158078FEF6807710509F49DC0E8F475
:10122000423385E058076105710509F4A4C038F41C
:10123000493055406105710509F494C0A5C0443397
:1012400085E058076105710509F492C04D3F524091
:101250006F4F710509F48FC097C04D3D82E258076A
:101260008FEF6807710509F483C038F4473E584191
:101270006F4F710509F46AC087C04F3C80E358077F
:101280008FEF6807710509F45EC0473C58436F4F04
:10129000710509F464C078C0473988E658078FEFB4
:1012A0006807710509F446C000F54D3A82E5580714
:1012B0008FEF6807710509F461C030F4453B5A446B
:1012C0006F4F7105A1F160C0453A8AE558078FEF6D
:1012D0006807710509F446C04D3952466F4F7105D4
:1012E00009F052C066E779E051C0473588EA5807EF
:1012F0008FEF68077105C9F168F445388AE7580728
:101300008FEF6807710529F1473658496F4F71050E
:10131000A1F03AC04F3480EB58078FEF6807710592
:1013200079F04D33524C6F4F710529F12DC068E5AE
:1013300079E02CC063E87BE029C060E87BE026C050
:101340006DE77BE023C06AE77BE020C067E77BE0D6
:101350001DC06BEB79E01AC06EE87BE017C060E956
:101360007BE014C062E97BE011C060EF77E00EC063
:1013700060E476E00BC06DEC78E008C061E179E0F4
:1013800005C064E97BE002C06FEB79E0CE010E940A
:10139000564CCE01DF91CF9108954F925F926F929C
:1013A0007F928F929F92AF92BF92EF92FF920F9394
:1013B0001F93CF93DF93CDB7DEB762970FB6F89444
:1013C000DEBF0FBECDBF7C015B018DE593E10E94C6
:1013D000E61D892B31F46FEB79E0C7010E94564C72
:1013E00028C1409161135091621360916313709111
:1013F0006413CE01079668DE80919713882359F114
:1014000066E97BE0CE0101960E94564CBE01695F01
:101410007F4FCE0101960E94724B66E177E00E94F9
:101420005B4BBC0180E19FE00E94B44CCE01019671
:101430000E94F24B409161135091621360916313CB
:101440007091641320E180E19FE00E94FB4C80E1F9
:101450009FE00E94C36960E070E0CE0107960E94A1
:10146000A84A182F8A3211F01092441350DD60936D
:101470003B0C70933C0C80933D0C90933E0C6FEBB7
:1014800079E0CE010D960E94564C812F110F990BD9
:10149000C0970A9708F05CC0CE0107960E943D4AAB
:1014A00063307105810591050CF094C001E010E0F6
:1014B00082E0982E0A151B050CF08CC06CE271E0DE
:1014C00080E090E0C8DB9092B90F1092BC0F412CE5
:1014D000512C32018DE493E10E94E61D892B41F4E9
:1014E0008EE1481651046104710409F08CC01CC0DF
:1014F0008EE14816510461047104B1F0409151131A
:10150000509152136091531370915413CE01019670
:10151000DBDDBE016F5F7F4FCE010D960E940F4B4A
:10152000CE0101960E94F24B89899A89892B39F064
:10153000BE01635F7F4FCE0107960E94094B0F5F8C
:101540001F4F6FEB79E0CE010D960E94C84BB2CFD2
:101550006CE271E080E090E07EDB82E08093B90F86
:101560001092BC0F812C912C54018DE493E10E94C8
:10157000E61D892B41F48EE188169104A104B10483
:1015800009F04CC01CC08EE188169104A104B1047E
:10159000B1F04091511350915213609153137091D7
:1015A0005413CE01019690DDBE016F5F7F4FCE01D7
:1015B0000D960E940F4BCE0101960E94F24B898935
:1015C0009A89892B39F0BE01635F7F4FCE01079660
:1015D0000E94094B64E670E080E090E03CDB82E032
:1015E0008093B90F1092BC0FBE01695F7F4FC70196
:1015F0000E943E4CCE010D960E94F24BCE01079602
:101600000E94F24B16C06EE170E080E090E023DBB8
:101610008FEF481A580A680A780A5CCF6EE170E0CA
:1016200080E090E018DB8FEF881A980AA80AB80AC1
:101630009CCFC70162960FB6F894DEBF0FBECDBF38
:10164000DF91CF911F910F91FF90EF90BF90AF90DE
:101650009F908F907F906F905F904F900895AF9282
:10166000BF92CF92DF92EF92FF920F931F93CF938F
:10167000DF93CDB7DEB72C970FB6F894DEBF0FBE61
:10168000CDBF7C015B010E94FA97182F811106C023
:101690006FEB79E0C7010E94564C99C08A3211F075
:1016A0001092441334DC60933B0C70933C0C809399
:1016B0003D0C90933E0C612FCE0107960E94264C64
:1016C000812F012E000C990BC0970A9750F5CE017F
:1016D00007960E943D4A63307105810591050CF023
:1016E0004BC001E010E00A151B050CF045C062E399
:1016F00070E080E090E0AFDA0E94FA97C12CD12C24
:10170000811152C08FEFC81AD80A85E1C816D104DA
:1017100099F16EE170E080E090E09DDA0E94FA9726
:10172000EFCF612FCE0101960E94264CBE016F5F64
:101730007F4FCE0107960E940F4BCE0101960E946B
:10174000F24B62E370E080E090E085DA0E94FA9765
:1017500000E010E08823D9F0682FCE0101960E94A6
:10176000264CBE016F5F7F4FCE0107960E94094B4A
:10177000CE0101960E94F24BBE01695F7F4FC70107
:101780000E943E4CCE0107960E94F24B20C00F5F94
:101790001F4F0F31110581F36EE170E080E090E0A2
:1017A0005ADA0E94FA97D6CF682FCE0101960E948E
:1017B000264CBE016F5F7F4FCE0107960E94094BFA
:1017C000CE0101960E94F24B0F5F1F4F8CCFC701D5
:1017D0002C960FB6F894DEBF0FBECDBFDF91CF9130
:1017E0001F910F91FF90EF90DF90CF90BF90AF903F
:1017F00008954F925F926F927F928F929F92AF92D5
:10180000BF92CF92DF92EF92FF92CF93DF93CDB74B
:10181000DEB72C970FB6F894DEBF0FBECDBF0E9487
:10182000DC3E0E94C8952B013C010E949A974B0117
:101830005C01609143027091440280914502909155
:1018400046020E94ABAE6B017C010E94C8950E94CB
:10185000ABAEA70196010E94FBB021E03EED42E451
:101860005EE30E94A3B29B01AC0160E070E080E8FF
:101870009FE30E9434B020E03AE24DE257E40E9438
:101880000AAF6B017C01C301B2010E94ABAE20E044
:1018900030E048EC52E40E94FBB0AB01BC0122E016
:1018A000CE0101960E94F74BBE016F5F7F4F84E12E
:1018B00092E10E940F4BCE0101960E94F24B62E52D
:1018C00078E084E192E10E94FB4A64E172E18AE1FE
:1018D00092E10E94DD4B6EE478E0CE0101960E9419
:1018E000564C64E172E1CE0101960E94724BBC013C
:1018F00084E192E10E94DD4BCE0101960E94F24B01
:101900006DE07AE080E292E10E94C84B21E0B501EF
:10191000A401CE0101960E94F74BBE016F5F7F4F7D
:1019200080E292E10E94094BCE0101960E94F24BA7
:101930006BE97BE080E292E10E94FB4A21E0B70183
:10194000A601CE0101960E94F74BBE016F5F7F4F4B
:10195000CE0107960E944E4C67EF75E0CE010796C8
:101960000E945B4BBC0180E292E10E94094BCE01D8
:1019700007960E94F24BCE0101960E94F24B64E161
:1019800072E1CE0101960E944E4C68ED7BE0CE01E3
:1019900001960E945B4B60E272E10E94724BBC01B7
:1019A00080E292E10E94DD4BCE0101960E94F24B53
:1019B00021E0B501A401CE0101960E94F74BBE01C2
:1019C0006F5F7F4F86E292E10E940F4BCE0101963E
:1019D0000E94F24B66E272E1CE0101960E944E4CEB
:1019E0004AE050E060E070E0CE010196C4D2CE0142
:1019F00001960E94F24B65E070E080E090E02BD908
:101A000066E779E0CE0101960E94564CCE01019620
:101A1000E6D0CE0101960E94F24B6AE172E1CE015E
:101A200001960E944E4C4AE050E06FEF7FEFCE01EE
:101A3000019659D0CE0101960E94F24B20E0B701E9
:101A4000A601CE0101960E94F74BBE016F5F7F4F4A
:101A5000CE0107960E944E4C67EF75E0CE010796C7
:101A60000E945B4BBC0186E292E10E94DD4BCE01FD
:101A700007960E94F24BCE0101960E94F24B66E25D
:101A800072E1CE0101960E944E4C4AE050E064EFB4
:101A90007FEFCE01019627D0CE0101960E94F24B36
:101AA00065E070E080E090E0D6D88091450C882316
:101AB00029F068E572E080E090E0CDD82C960FB672
:101AC000F894DEBF0FBECDBFDF91CF91FF90EF90B6
:101AD000DF90CF90BF90AF909F908F907F906F904E
:101AE0005F904F9008958F929F92AF92BF92EF9226
:101AF000FF920F931F93CF93DF9320912E05222304
:101B000009F462C020912D05222309F45DC08A01E9
:101B1000EB017C0177FF18C0C095D09561E08C2F58
:101B20000E94566AB70181E293E10E94B44C6AEFC9
:101B300073E181E293E10E94C24CF701848161E08C
:101B40008C0F0E94566A31C0E2D980908F1390901A
:101B50009013A0909113B090921324E6820E911CE2
:101B6000A11CB11C86169706A806B90668F561E0A7
:101B70008C2F0E94566AB70181E293E10E94B44C17
:101B800069EE73E181E293E10E94C24CF701848126
:101B900061E08C0F0E94566ABAD960938F137093DC
:101BA00090138093911390939213B801110F880BA7
:101BB000990BDF91CF911F910F91FF90EF90BF9004
:101BC000AF909F908F9047C8DF91CF911F910F9159
:101BD000FF90EF90BF90AF909F908F900895CF931C
:101BE000DF9320912E052223A9F020912D05222399
:101BF00089F0EC016FED81E293E10E94AD4C8C81A4
:101C00009D81892B39F0BE0181E293E1DF91CF9173
